:020000040002F8
:10600000B0BF0020DD630200E5630200598C02008E
:10601000E9630200EB630200ED6302000000000090
:10602000000000000000000000000000EF6302001C
:10603000F163020000000000F3630200F563020058
:10604000BD9B0200F763020065C7020049B1020070
:106050005DB10200F7630200598B02002DAA020015
:10606000F7630200F7630200F7630200F7630200C0
:10607000F7630200F7630200F7630200F7630200B0
:1060800091CA02009DA50200F7630200F7630200B7
:10609000F7630200F7630200D5B10200F763020064
:1060A000F7630200F7630200F7630200F763020080
:1060B000B99C0200F763020000000000000000002D
:1060C000F7630200F7630200F763020071B1020098
:1060D000B5A50200F7630200F763020000000000AC
:1060E00000000000000000000000000000000000B0
:1060F00000000000000000000000000000000000A0
:10610000000000000000000000000000000000008F
:10611000000000000000000000000000000000007F
:10612000000000000000000000000000000000006F
:10613000000000000000000000000000000000005F
:10614000000000000000000000000000000000004F
:10615000000000000000000000000000000000003F
:10616000000000000000000000000000000000002F
:10617000000000000000000000000000000000001F
:10618000000000000000000000000000000000000F
:1061900000000000000000000000000000000000FF
:1061A00000000000000000000000000000000000EF
:1061B00000000000000000000000000000000000DF
:1061C00000000000000000000000000000000000CF
:1061D00000000000000000000000000000000000BF
:1061E00000000000000000000000000000000000AF
:1061F000000000000000000000000000000000009F
:10620000DFF80CD000F0FCFC0048004765F003000C
:10621000B0BF002000B583B002900091019244F21B
:10622000010071466A460AF099F903B000BD00000A
:1062300030B450E8012F93B2C48923448489A34227
:1062400028BF1B1B0489A34202BFBFF32F8F00206E
:1062500007E0C3EA020340E80134002CE9D14FF023
:1062600001000A6030BC704750E8012FC2EA0242C8
:1062700040E801210029F7D1704730B450E8022FDF
:106280001FFAA2F3C488A34202BFBFF32F8F0020DE
:106290000DE0C48923448489A34228BF1B1BC2EAA2
:1062A000034340E80234002CE8D14FF001000A60BB
:1062B00030BC704750E8022FC2EA224240E8022177
:1062C0000029F7D17047034653E8022FD988B2EB73
:1062D000324F4FF0000017BF92B241EA014142EA4B
:1062E000014104E05A68B2EB324F08BF012043E895
:1062F0000212002AE8D1704730B4044654E8000F77
:106300000D4644E80053002BF8D1156030BC7047AF
:1063100030B4044654E8000F40EA010544E8005355
:10632000002BF7D1156030BC704730B4044654E8F8
:10633000000F00EA010544E80053002BF7D1156077
:1063400030BC704730B4044654E8000F80EA0105C1
:1063500044E80053002BF7D1156030BC704730B4CF
:10636000044654E8000F00EB010544E80053002BFD
:10637000F7D1156030BC704730B4044654E8000FC4
:10638000A0EB010544E80053002BF7D1156030BCA9
:10639000704770B404464FF0000054E8006F0D6879
:1063A000AE4207BF44E80023012044E800630E60CA
:1063B000002B1CBF0020F0E770BC704730B40446CF
:1063C00054E8000F88422CBF451A054644E80053A4
:1063D000002BF5D1156030BC70470000064880479F
:1063E00006480047FEE7FEE7FEE7FEE7FEE7FEE7BA
:1063F000FEE7FEE7FEE7FEE7B1BE02000162020033
:106400002DE9F05F0546002092469B4688460646E9
:10641000814640241BE0284641464746224600F07C
:10642000CFFA53465A46C01A914110D31146184626
:10643000224600F016F82D1A67EB01084F46224657
:106440000120002100F00DF817EB00094E41201E3D
:10645000A4F10104DFDC484631462A464346BDE844
:10646000F09F202A04DB203A00FA02F10020704756
:106470009140C2F1200320FA03F319439040704782
:1064800040EA01039B0703D009E008C9121F08C0B6
:10649000042AFAD203E011F8013B00F8013B521E36
:1064A000F9D27047D2B201E000F8012B491EFBD2AD
:1064B00070470022F6E710B513460A46044619460F
:1064C000FFF7F0FF204610BD421C10F8011B002909
:1064D000FBD1801A704710B5002200E0521C835C8B
:1064E0008C5CA34201D1002BF8D1D8B2E1B2401AA2
:1064F00010BD30B504460020034600E05B1C93420B
:1065000003D2E05CCD5C401BF8D030BD034611F8EF
:10651000012B00F8012B002AF9D1184670472DE90C
:10652000FE4F804681EA0300C00F0C46009021F028
:10653000004123F00045B8EB0200A94105D24046D6
:10654000214690461C460B46024623F0004010436D
:1065500047D0270DC7F30A00C3F30A510290401A2F
:10656000019040286BDAC3F3130040F4801B0098BD
:10657000924620B10023D2EB030A63EB0B0B019888
:106580005946C0F140025046FFF76BFF06460D46E4
:1065900050465946019A00F023FA10EB0800614179
:1065A000002487EA115284EAE7731A4340D0009A24
:1065B00062B3019A012A4FEA075215DC001B61EB16
:1065C00002014FF0004202EA0752CDE90042001CEE
:1065D00041F5801132462B4600F05AFA03B0BDE86F
:1065E000F08F40462146F9E7001B61EB0201001CD9
:1065F00041F5801300185B412018A2F5001747EB06
:10660000030140EAD570B6196D4111E06D084FEAFB
:10661000360645EAC0754FEA0752001B61EB0201DE
:10662000001C41F5801149084FEA30000019514122
:1066300032462B4603B0BDE8F04F00F01ABA00987E
:10664000012240000023D0EB020263EBE0730098CC
:1066500021464FEAE074B8EB000061EB0401E9E782
:1066600083F000435BE781F0004158E72DE9FE4FDE
:1066700081EA030404F0004421F0004100944FF04B
:10668000000B23F0004350EA01045ED052EA0304F9
:106690005BD0C3F30A54C1F30A552C44A4F2F3347B
:1066A0000194A0FB0254C1F3130141F48011C3F320
:1066B000130343F4801301FB024400FB034E840ADE
:1066C000970A44EA815447EA8357A4FB0768029576
:1066D0008D0A05FB07854FEA932C04FB0C54270514
:1066E000029D4FEA065847EA1637B5EB08056EEBF0
:1066F000070C870E920E47EA811742EA8312A7FB26
:106700000201B6EB0B0164EB00042B0D43EA0C33E2
:106710005E1844EB1C50DA465146E7FB0201C5F314
:1067200013044FEA0B3343EA14534FEA0432019C3B
:1067300043EA0603A4F10C040294009CCDE900B4E2
:1067400000F0A6F903B0BDE8F08F00200146F9E79C
:106750002DE9F04D81EA030404F0004B21F00045DF
:1067600014464FF0000A23F0004150EA050220D001
:1067700054EA01021DD0C5F30A570246C5F31303BC
:10678000C1F31300C1F30A5640F4801543F480139B
:10679000A7EB0608101BD64608F2FD3873EB050080
:1067A00002D308F1010801E092185B41B8F1000F33
:1067B00003DA00200146BDE8F08D00204FF480117F
:1067C000064684460EE0171B73EB050705D3121B24
:1067D00063EB050306434CEA010C49084FEA30001D
:1067E00092185B4150EA0107EDD152EA030012D042
:1067F00082EA040083EA0501084305D0101BAB417F
:1068000006D20122002306E000224FF0004302E0FE
:106810006FF0010253101AEB06004CEB085110EB1D
:106820000A0041EB0B01BDE8F04D00F022B9F0B4D5
:10683000CA17CB0F50405140C61841F100054FEA2E
:10684000C372314628004FF0960303D0B623F0BC44
:1068500000F0E1B830460021F9E70EB5C10F80EA3B
:10686000E0700844CA07002140F233438DE80E006F
:106870000A460B4600F00CF903B000BD0EB540F21D
:10688000334102910021CDE900110A460B4600F088
:10689000FFF803B000BD70B5C1F30A5201F0004526
:1068A0000024C1F3130140F2FF3341F480119A42F6
:1068B00001DA002070BD40F233439A42A2F2334223
:1068C00003DC524200F07CF800E090402C43F1D011
:1068D000404270BDC1F30A5210B5C1F3130140F23A
:1068E000FF3341F480119A4201DA002010BD40F2DA
:1068F00033439A42A2F2334203DC524200F060F882
:1069000010BD904010BD00F0004230F000400AD0B1
:10691000C10D01F56071C0F3160042EA0151C208D1
:1069200040071143704700200146704730B5041EF0
:1069300071F1000404DB4FF00044404264EB0101BC
:10694000141E73F1000405DB1C464FF00043524255
:1069500063EB0403994208BF904230BD01F000434D
:1069600030B421F0004150EA010206D00A0DA2F530
:106970006072C1F31301002A02DC30BC00207047B2
:10698000440F44EAC104C100E01830BC00EBC2501F
:1069900000F038B830B50B46014600202022012413
:1069A00009E021FA02F59D4205D303FA02F5491BDD
:1069B00004FA02F52844151EA2F10102F1DC30BDF3
:1069C000202A04DB203A21FA02F00021704721FA44
:1069D00002F3D040C2F120029140084319467047AB
:1069E000202A06DBCB17203A41FA02F043EAE07393
:1069F00006E041FA02F3D040C2F120029140084380
:106A0000194670470029A8BF7047401C490008BFBD
:106A100020F00100704710B4B0FA80FC00FA0CF0CE
:106A200050EA010404BF10BC704749B1CCF1200406
:106A300021FA04F411FA0CF118BF01212143084393
:106A4000A3EB0C01CB1D4FEA00614FEA102042BFBF
:106A5000002010BC704700EBC35010440029A4BFB5
:106A600010BC7047401C490008BF20F0010010BC5A
:106A7000704710B5141E73F1000408DA401C41F190
:106A8000000192185B411A4301D120F0010010BDB2
:106A90002DE9F04D92469B4611B1B1FA81F202E028
:106AA000B0FA80F220329046FFF7DBFC04460F4636
:106AB00040EA0A0041EA0B0153465A46084313D004
:106AC000114653EA010019D0C8F140025046FFF7C1
:106AD00077FF05460E46504659464246FFF7C1FC31
:106AE000084305D0012004E020463946BDE8F08D7A
:106AF0000020054346EAE0762C4337430A986305B5
:106B0000E40AA0EB08000022FD0A44EA47540A30D8
:106B100002D500200146E9E7010510196941DDE9C8
:106B2000084500196941BDE8F04DA2E72DE9F04D97
:106B300000231A461B1A8A4103DB00200146BDE8E8
:106B4000F08DC1F30A52C1F3130141F480154FF0E7
:106B5000000BD10702D100186D41521E00270446D8
:106B600040F2FF11384601EB620A3E46804602467B
:106B700000204FF48011FFF723FFC2197141BB18A9
:106B800046EB0100B4EB030C75EB000C04D3E41AE4
:106B900065EB000517460E46241908F101006D410A
:106BA00080463428E3DDF91946EB0600091BA841AD
:106BB00003D24FF0FF32134601E0002213461BEBD5
:106BC000070046EB0A51BDE8F04DFFF752BFC1F395
:106BD0000A52C1F3130140F2FF3341F480119A428B
:106BE00002DA00200146704740F233439A42A2F293
:106BF000334202DC5242FFF7E3BEFFF732BC000033
:106C0000064C074D06E0E06840F0010394E80700F9
:106C100098471034AC42F6D3FFF7F6FAECAC040018
:106C20000CAD040070B58C1810F8015B15F007036B
:106C300001D110F8013B2A1106D110F8012B03E015
:106C400010F8016B01F8016B5B1EF9D12B0705D41D
:106C50000023521E0DD401F8013BFAE710F8013B66
:106C6000CB1A921C03E013F8015B01F8015B521E82
:106C7000F9D5A142D8D3002070BD000010B51CF09A
:106C800043F900200149086010BD0000F4400020D5
:106C900010B500F00DF810BD38B504460020009086
:106CA0006946204600F0F8F8BDF9000038BD000044
:106CB0002DE9F84F00265F480068009006208DF807
:106CC00002006C465C4F04B95C4C394620461CF00F
:106CD0002FF8054600BF0DB14FF0FF3600248FE0BE
:106CE000574850F83400FF287DD0554800EBC400C9
:106CF0004068FF28F8D0524A52F8340000210022A0
:106D000013461746944600BF4FF0A049C84642EAD2
:106D1000430949EA810949EA072949EA0C4A08F581
:106D2000E06949F820A000BF00BF0020444901EB02
:106D3000C401496801EBC101424A5054404901EB8A
:106D4000C401496801EBC101114448703C4901EBA1
:106D5000C401496801EBC10111448870384901EB55
:106D6000C401496801EBC1011144C87002203449D3
:106D700001EBC401496801EBC10111440871002015
:106D80002F4901EBC401496801EBC101114448716D
:106D90002B4901EBC401496801EBC1011144887121
:106DA000274800EBC4000079401C254901EBC401D1
:106DB000496801EBC1011144C8710020204901EB71
:106DC000C401496801EBC101114408721C4A02EB7D
:106DD000C402526802EBC2021A4BD118184A02EBE5
:106DE000C402107900E00AE01BF00AFF05460DB16D
:106DF0004FF0FF3614480068401C13490860641CBB
:106E0000082CFFF66DAF1048006848B10E480088A6
:106E100081B20E481BF094FE05460DB14FF0FF36CF
:106E2000701C20B90A4A0BA1002003F007FABDE844
:106E3000F88F0000D4A3040015ED0200D0A30400D5
:106E4000B04000202C7C0020F4400020747C002006
:106E5000E93F03006273705F6164635F696E697428
:106E60005F70726F636573730000000010B50721D7
:106E70001F2000F06BF804211C2000F067F8FFF7DA
:106E800017FF034805F022FF024804F0EFF910BD98
:106E9000B7540300AD5403002DE9FC4706460F46E6
:106EA0004FF0030923A103C9CDE900014FF0000809
:106EB0000020224908702248006810B90520BDE86A
:106EC000FC871CF009F805460DB10720F7E709E03B
:106ED000B9F10000A9F1010902D01AF009FF01E09F
:106EE0000620ECE7154800780028F1D000240DE0DA
:106EF00004EBC40013490844C07930B1E0B20DF886
:106F0000080008F1010000F0FF08641C082CEFDB0A
:106F1000002408E01DF80400B04203D10A4830F80C
:106F200014003880641C064800688442F2D30020B4
:106F3000C5E70000FFFFFFFFFFFFFFFFF04000205D
:106F4000F44000202C7C0020747C002002460B467C
:106F500000211EE0114850F83100904201D101207B
:106F600070470E4800EBC1004068984201D10220F2
:106F7000F6E7FF2A0CD0094850F83100FF2807D166
:106F8000064840F8312000EBC10043600020E7E7ED
:106F9000491C0829DEDB0320E2E70000B0400020A6
:106FA0002DE9F04106460F4614469846069DB0EE80
:106FB000000A84ED000A95ED020AB1EE400A84ED64
:106FC000010A95ED010A84ED020A95ED020A84EDAD
:106FD000030AB0EE000A84ED040A95ED000AB1EE52
:106FE000400A84ED050A95ED010AB1EE400A84EDF0
:106FF000060A95ED000A84ED070AB0EE000A84ED5A
:10700000080A4146204616F0FFFBB0EE000A84ED68
:10701000000A95ED020A84ED010A95ED010AB1EE30
:10702000400A84ED020A95ED020AB1EE400A84EDB1
:10703000030AB0EE000A84ED040A95ED000A84ED1F
:10704000050A95ED010A84ED060A95ED000AB1EEF8
:10705000400A84ED070AB0EE000A84ED080A3A46B9
:107060004146204619F01FF8242239462046FFF7F2
:1070700007FA3A463146204619F015F824223946D7
:107080003046FFF7FDF9BDE8F081000010B5054A74
:1070900005A1002003F0D2F8074A08A1012003F05F
:1070A000CDF810BD21710200424C455F436C69650B
:1070B0006E745F527800000021730200424C455FFD
:1070C000436C69656E745F547800000030B5034608
:1070D000104A1068002900DC30BD002214E00D4C7D
:1070E0002468601C0C4CA04201D3A4F580600B4CBA
:1070F0002468A04206D09C5C064D2D682C70054C7F
:10710000206000E002E0521C8A42E8DB00BF00BFC2
:10711000E2E70000D03F002040560020D43F00208E
:1071200070B565E03348007810B101285BD12BE0E1
:1071300000F090FC032800D270BD002000F05AFC43
:10714000AA2803D0012000F0B5FC1CE0022000F0CA
:1071500051FC0446E043C4B2012000F04BFC264938
:10716000087008460078844209D10846007805284E
:1071700005DB20480078401C1E49087002E0012011
:1071800000F098FC00BF32E000F064FC1A49097876
:10719000884200D2D0E70025002406E0204600F017
:1071A00029FC2844C5B2601CC4B213480078401EB4
:1071B000A042F3DC10490978491E88B200F01AFC9D
:1071C000A84208D10C48007803F0C4F80A480078B7
:1071D00000F070FC02E0012000F06CFC002005498A
:1071E000087000BF03E000200249087000BF00BF24
:1071F00098E70000E03F0020E13F002010B5024684
:1072000010480068112802D34FF0FF3010BD0E481F
:107210000C4B1B6800EB0310C1600B48094B1B684B
:1072200000EB031002700948074B064C246803EB7F
:107230000413586003480068401C024B186000208B
:10724000E4E70000D83F00204056002050570020BF
:107250002DE9F047C0B08046894616460025002437
:10726000701D00F0FF0AFA2E03DD601E40B0BDE87D
:10727000F087AA200DF804002046611CCCB21DF84E
:1072800000002844C5B20DF804A02046611CCCB211
:107290001DF800002844C5B26FEA0A00C0B20DF81C
:1072A00004002046611CCCB21DF800002844C5B281
:1072B0000DF804802046611CCCB21DF80000284463
:1072C000C5B200270CE019F807000DF804002046AD
:1072D000611CCCB21DF800002844C5B2781CC7B2AE
:1072E000B742F0DB2046611CCCB20DF800502146BD
:1072F000684620F017FEB9E708490AE00A688242AA
:1073000004D100234376136A0B6001E002F12001EF
:1073100000BF0A68002AF1D170470000DC3F00205E
:1073200070B5002600251E48046831E0E06800289A
:107330002BD004F00DFF1B490968451A04F008FF23
:107340001849086005B90125E068A84203D3E06840
:10735000401BE06001E00020E060E068A8B9207A0E
:1073600000280ADD207A401E20726068E060227EDC
:10737000207C6169FFF76CFF07E02046FFF7BCFF48
:10738000E06910B12046E1698847607E0643246ABF
:10739000002CCBD13146AFF2770002F02BFF70BD4D
:1073A000DC3F0020E43F00202DE9F0410446884600
:1073B00015461E4613480768ECB184F810806561D5
:1073C00026766068E0602078002803DD2078401E83
:1073D000207201E0002020720120607604E0A742C4
:1073E00001D1BDE8F0813F6A002FF8D1054800685F
:1073F000206204480460324629464046FFF728FFD1
:1074000000BFEEE7DC3F002010B5054A05A10020D3
:1074100002F014FF064A07A1012002F00FFF10BD81
:10742000C9740200424C455F486F73745F52780024
:10743000D9760200424C455F486F73745F54780000
:107440002DE9F04104460D461B480668052D01DA7A
:10745000BDE8F0816778A078C04300F0FF0820788D
:10746000AA280CD147450AD1AF4208D1E0780528B7
:1074700005DAE9B22046114A1268904719E0002067
:1074800014E00D4909684E1C0D498E4201D3A1F547
:1074900080660C4909688E4206D0215C064A126853
:1074A000117005490E6000E002E0401CA842E8DBD4
:1074B00000BF00BFCCE70000E83F0020F03F002005
:1074C000505C0020EC3F002070B565E03348007848
:1074D00010B101285BD12BE000F0CCFA032800D2D8
:1074E00070BD002000F096FAAA2803D0012000F019
:1074F00005FB1CE0022000F08DFA0446E043C4B214
:10750000012000F087FA2649087008460078844276
:1075100009D108460078052805DB20480078401C82
:107520001E49087002E0012000F0E8FA00BF32E0D6
:1075300000F0A0FA1A490978884200D2D0E7002565
:10754000002406E0204600F065FA2844C5B2601C1D
:10755000C4B213480078401EA042F3DC10490978F9
:10756000491E88B200F056FAA84208D10C480078AB
:1075700002F030FF0A48007800F0C0FA02E0012073
:1075800000F0BCFA00200549087000BF03E00020AD
:107590000249087000BF00BF98E70000FC3F0020D0
:1075A000FD3F002010B5024610480068112802D3A4
:1075B0004FF0FF3010BD0E480C4B1B6800EB031062
:1075C000C1600B48094B1B6800EB031002700948AF
:1075D000074B064C246803EB04135860034800680B
:1075E000401C024B18600020E4E70000F43F00203C
:1075F000505C0020605D00200146024801600020D0
:1076000070470000F03F00202DE9F047C0B08046F1
:107610008946164600250024701D00F0FF0AFA2E48
:1076200002DD40B0BDE8F087AA200DF80400204636
:10763000611CCCB21DF800002844C5B20DF804A0AE
:107640002046611CCCB21DF800002844C5B26FEA88
:107650000A00C0B20DF804002046611CCCB21DF82F
:1076600000002844C5B20DF804802046611CCCB24D
:107670001DF800002844C5B200270CE019F80700E7
:107680000DF804002046611CCCB21DF8000028440F
:10769000C5B2781CC7B2B742F0DB2046611CCCB241
:1076A0000DF800502146684620F056FC00BFB8E7B0
:1076B00008490AE00A68824204D100234376136A2B
:1076C0000B6001E002F1200100BF0A68002AF1D13D
:1076D00070470000F83F002070B5002600251E48C6
:1076E000046831E0E06800282BD004F031FD1B492C
:1076F0000968451A04F02CFD1849086005B90125F0
:10770000E068A84203D3E068401BE06001E000208D
:10771000E060E068A8B9207A00280ADD207A401EDF
:1077200020726068E060227E207C6169FFF76CFF58
:1077300007E02046FFF7BCFFE06910B12046E16991
:107740008847607E0643246A002CCBD13146AFF2D5
:10775000770002F04FFD70BDF83F00200040002090
:107760002DE9F0410446884615461E461348076831
:10777000ECB184F81080656126766068E06020785E
:10778000002803DD2078401E207201E000202072D6
:107790000120607604E0A74201D1BDE8F0813F6A94
:1077A000002FF8D105480068206204480460324682
:1077B00029464046FFF728FF00BFEEE7F83F0020CC
:1077C00010B50446002116E00F4850F82100A042F1
:1077D00002D14FF0FF3010BD0B4850F8210048B9DE
:1077E0000A480078401C094A1070074840F82140B8
:1077F0000020F0E7491C0329E6DB05A1002003F087
:107800005BFA6FF00100E6E7A8840020C44700207F
:10781000626C655F6576745F526567697374202D6D
:107820003E20746F6F206D616E79210A00000000A8
:1078300010B50446002116E00F4850F82100A04280
:1078400002D14FF0FF3010BD0B4850F8210048B96D
:107850000A480078401C094A1070074840F8214047
:107860000020F0E7491C1029E6DB05A1002003F009
:1078700023FA6FF00100E6E7108200208A41002021
:10788000626C655F6576745F526567697374202DFD
:107890003E20746F6F206D616E79210A0000000038
:1078A00030B52DED048B83B0B0EE408AF0EE608AE7
:1078B0003148007800285CD018EE900AFFF723F8D2
:1078C00041EC190B9FED2D0B53EC102BFFF72EF80D
:1078D00004D3F4EEC88AF1EE10FA04D2032003B008
:1078E000BDEC048B30BDB1EE0E0AB4EEC08AF1EEF1
:1078F00010FA01D20320F2E79FED220A28EE800A57
:10790000DFED210A80EE201ABCEEC10A10EE100A4B
:1079100080B2ADF806009FED1B0A28EE000ADFEDED
:107920001A0A80EE201ABCEEC10A10EE100A80B2CC
:10793000ADF804004FF4C870ADF80A000020ADF8AF
:1079400008001249088901A975DF0446082C0ED0E9
:10795000112C0CD05CB100BF25463DB100BF0CA27C
:1079600040F287212846FEF755FC00BF00BF2046A5
:10797000B5E70120B3E70000BA470020000000008F
:10798000003B9F4000007A4400409C4490820020CD
:107990002E2E5C2E2E5C2E2E5C626C655F636667FD
:1079A0005C686F73742E63009FED0E2AC0EE022A8E
:1079B0009FED0D2A22EE822AB0EE421A9FED0B2A8D
:1079C00021EE022A22EE202ADFED092A82EE223A57
:1079D000F0EE431A90ED002A32EE212A80ED002AC3
:1079E0007047000000803B45CDCC8C3F00007A44BE
:1079F000000061450246054800688118044881423C
:107A000001D3A1F58061087870470000D43F0020C1
:107A1000405600200246054800688118044881420B
:107A200001D3A1F58061087870470000EC3F002089
:107A3000505C0020024605480068811804488142D5
:107A400001D3A1F580610878704700001C40002038
:107A500060620020054B1A68054B19688A4201D301
:107A6000501A02E002F58063581A7047D03F002098
:107A7000D43F0020054B1A68054B19688A4201D390
:107A8000501A02E002F58063581A7047E83F002060
:107A9000EC3F0020054B1A68054B19688A4201D358
:107AA000501A02E002F58063581A7047184000200F
:107AB0001C40002018E0411E88B20D4909680D4A9B
:107AC0001268914200D1704709490968491C0A4A65
:107AD000914204D3A2F58061054A116004E0044993
:107AE0000968491C024A11600028E4D100BFEAE796
:107AF000D43F0020D03F00204056002018E0411E17
:107B000088B20D4909680D4A1268914200D1704748
:107B100009490968491C0A4A914204D3A2F58061C7
:107B2000054A116004E004490968491C024A1160D1
:107B30000028E4D100BFEAE7EC3F0020E83F002046
:107B4000505C002018E0411E88B20D4909680D4ABA
:107B50001268914200D1704709490968491C0A4AD4
:107B6000914204D3A2F58061054A116004E0044902
:107B70000968491C024A11600028E4D100BFEAE705
:107B80001C40002018400020606200200849095C69
:107B900001290CD1002206490A54891F498C31B1B0
:107BA0000349891F498C491E014A921F518470471D
:107BB0003E4F0020004870475C4F002001460020E7
:107BC0000DE000EB8002074B03EBC20292F8252088
:107BD00022B900EB800203EBC2021162401C0228B2
:107BE000EFDB7047A0FF002001460348405C0128FE
:107BF00000D170470020FCE73E4F002010B5002167
:107C0000064802F0F7FA0120054908703220488042
:107C100001208880072001F05DFD10BD9D7E0200DF
:107C2000384F002010B51A48408800282ED0012176
:107C3000184802F0DFFA1648808868B914480078BE
:107C400018B901201249087002E00020104908709C
:107C500001200F49888014E00D48007818B90E49BA
:107C6000072001F003FD0A480078012804D14FF0F5
:107C70007F41072001F0FAFC05488088401E044936
:107C8000888003484088401E0149488010BD00009C
:107C9000384F00209D7E020000106FFF70B5044633
:107CA000241F10A1002003F007F84FF40070B0EB80
:107CB000145F04D01B49002002F0FEFF70BD0834A1
:107CC0000121194880F84D1080F84C1020222146DF
:107CD0002830FEF7D5FB2546A869C01EA86100BF65
:107CE000ECE700000D0A2D2D2D2D2D2D2D2D2D2DE8
:107CF0002D2D2D2D2D2D2D4552524F52202D2D2D18
:107D00002D2D2D2D2D2D2D2D2D2D2D2D2D2D0D0AE6
:107D1000486172644661756C745F48616E646C653D
:107D2000720D0A0030AB0400A0FF00200649095C78
:107D3000012908D0012204490A54891F498C491C91
:107D4000014A921F518470473E4F0020F0B5BFB0EA
:107D500006460F46002400253846FEF7B5FB85B2DF
:107D6000F82D02D9601E3FB0F0BD1148007930B146
:107D700000222046611CCCB20DF8002005E0012253
:107D80002046611CCCB20DF800202046611CCCB20C
:107D90000DF800600DEB04002A463946FEF770FB33
:107DA0006019C4B222466946AD20FFF751FADAE7FE
:107DB000945100200120024981F8250070470000FD
:107DC000A0FF002010B524211348FEF772FB01200C
:107DD0001149087032204880012088800F4A10A184
:107DE000C82002F02BFA144A14A1642002F026FAEB
:107DF0001C49AD20FFF7D6FB50221BA1002002F04A
:107E00005BFF242223492448FEF73AFB21492248FC
:107E10001DF0DAFD10BD0000384F00209D7E0200ED
:107E2000457863657074696F6E5F4C65645F50720E
:107E30006F63657373000000097F02004578636516
:107E40007074696F6E5F556E6B6F776E5265736598
:107E5000745F496E666F5F53656E645F50726F63E7
:107E600065737300EB4F0300457863657074696F49
:107E70006E5F496E6974202D2073697A656F66287C
:107E80006E6F5F696E69745F64617461293A25641D
:107E90000D0A0000005200205C4F002000B589B0A0
:107EA00000200BF067FD012811DB01AA0021084624
:107EB0000BF056FDBDF80400ADF81C00BDF806003F
:107EC000ADF81E00BDF80800ADF8200001E009B0D3
:107ED00000BDBDF9200040F2DC51884206DB0848B5
:107EE000408C002802DDFFF79DFE06E0BDF9200072
:107EF0000449884201DCFFF781FE00BFE7E700008C
:107F0000384F002024FAFFFF30B5C9B0FC210AA881
:107F1000FEF7CFFAFC210AA8FEF7CBFA00248EE088
:107F200004EB8400484901EBC00090F825000128CB
:107F300071D104EB840001EBC00090F8240010B173
:107F400001286AD117E004EB84003F4901EBC0002F
:107F5000026A3EA10AA805F097F80AA91120FFF7C6
:107F6000F5FE38B9002004EB8401374A02EBC10169
:107F700081F825005AE02A22364B04EB840032496E
:107F800001EBC000C16904EB84002F4D05EBC0007C
:107F90008069C01E05AD0BC5089204EB84002A4918
:107FA00001EBC000406904EB8401274A02EBC101E8
:107FB000096904EB8402244B03EBC202D26804EB90
:107FC0008403214D05EBC3039B68CDE90132CDE964
:107FD000031004EB8400294601EBC00040680090C8
:107FE00004EB840051F8303004EB840001EBC00056
:107FF000026A19490AA805F047F80AA91120FFF7F3
:10800000A5FE38B9002004EB84012A4602EBC10129
:1080100081F825000AE011E0FFE7002004EB84016D
:10802000094A02EBC10181F8250000BF00BF04EB43
:108030008400054901EBC00090F82400641C022C68
:10804000FFF66EAF49B030BDA0FF002069643A254D
:10805000640D0A000101010074AB0400704770B5A3
:108060000025002600240CE04FF4E82000EB043645
:1080700030461FF063F905460DB1032070BD601C4A
:10808000C4B2022CF0DB0020F8E770B50025002612
:1080900000240CE04FF4EC2000EB043630461FF0D7
:1080A0004DF905460DB1032070BD601CC4B2022C11
:1080B000F0DB0020F8E710B504461C2221464FF4FF
:1080C000E62011F0B3FB10BD7CB500240020019028
:1080D000F24817F014FBF248FFF7EDFF06461923AC
:1080E0003246F0A1002002F0E7FDED48007E0528B1
:1080F00013DBFFF7B4FFFFF7C8FF0020E84908765D
:1081000000F032FB18B1F6A10820FFF71FFEF9A11D
:10811000002002F0D1FD04F0E3FFE148007E401CA6
:10812000DF49087600F020FB18B1EDA10820FFF729
:108130000DFE002436E004EB4401F84A52F8210019
:10814000FEF7C2F9054604EB4400F44A52F8201049
:1081500001AB2A46D1481CF045FF08BB04EB4400A4
:10816000EE4901EB8000007A9DF80410884217D197
:1081700004EB4401E94A52F82100FEF7A5F905464F
:1081800001A8009004EB4400E44A02EB800043683D
:1081900004EB440052F820102A46C0481CF0DEFED2
:1081A000601C84B2192CC6DBDD48DEA10268002009
:1081B00002F082FDDA480068E04988426BD0D84876
:1081C000DFA10268002002F077FDFFF748FFFFF70C
:1081D0005CFF9021D248FEF76CF9D848D04908607E
:1081E00001200871AE480068D449884259D1002561
:1081F00000BF0DE0AA48001D415DC948401D415522
:10820000A7480A30415DC64832304155681CC5B2A6
:10821000062DEFDBD7A1002002F04EFD002508E07F
:108220009F48001D425DD7A1002002F045FD681C5B
:10823000C5B2062DF4DBD5A1002002F03DFDD4A18E
:10824000002002F039FD002508E095480A30425D23
:10825000CCA1002002F030FD681CC5B2062DF4DB75
:10826000CAA1002002F028FD8D480169AC48C16216
:108270008B48818AAA4801868948807DA84981F86F
:1082800028008748C07D08718548808A009084480E
:108290000369827D00E098E0C1A1002002F00CFD9E
:1082A0000AE01C217E48FEF704F900F05DFA18B1DF
:1082B0008BA10820FFF74AFD00241EE004EB4401D7
:1082C000964A52F82100FEF7FFF8054604EB4400F9
:1082D000924901EB8000007A009004EB44000A46CA
:1082E00002EB8000436804EB440052F820102A4659
:1082F0006A481CF06BFD601C84B2192CDEDB002088
:1083000087490860002436E004EB4401834A52F8B0
:108310002100FEF7D9F8054604EB44007F4A52F8E5
:10832000201001AB2A465D481CF05CFE08BB04EB44
:1083300044007A4901EB8000007A9DF804108842DD
:1083400017D104EB4401754A52F82100FEF7BCF83E
:10835000054601A8009004EB4400704A02EB80003F
:10836000436804EB440052F820102A464B481CF0A6
:10837000F5FD601C84B2192CC6DB694896A1026821
:10838000002002F099FC664800686C49884208D0D9
:1083900099A1002002F090FC9DA10820FFF7D6FCD7
:1083A0007CBD5F48A0A10268002002F085FC00258A
:1083B00007E04FF4FA7018F059FF11F05DF9681CEE
:1083C000C5B2062DF5DB04F08BFE002455E104EB6D
:1083D0004401524A52F82100FEF776F8054604EBB4
:1083E00044004E4A52F8201001AB2A462B481CF09C
:1083F000F9FDE0BB04EB4400484901EB8000007A42
:108400009DF80410884218D104EB4401434A52F805
:108410002100FEF759F8054601A8009004EB44003E
:108420003E4A02EB8000436804EB440052F82010FF
:108430002A461A481CF092FD1DE104EB4401374A1C
:1084400052F82100FEF740F8054604EB4400334A99
:1084500052F820102A4611481CF05AFD04EB440142
:108460002E4A52F82100FEF72FF8054600E0E5E01D
:1084700004EB4400294901EB8000007A009004EBF2
:1084800044000A4602EB8000436804EB440052F8C3
:1084900020102A4601481CF099FCECE0983F00208F
:1084A00024520020466C6173685F476574426163C3
:1084B0006B75702028266D4261636B7570293A25B3
:1084C000642C4D41585F6D666C6173685F706172BA
:1084D000616D5F4C454E4754483A25640A000000E0
:1084E00073617665206261636B7570206661696C8B
:1084F000000000006D4261636B75702E4572726FF3
:10850000725374617274466C6167203E3D20352160
:10851000212121212121212121210A0010A2040051
:1085200094510020466C6173682068656164207214
:108530006561642825303458292E0A00AA5555AAA9
:10854000466C61736820666972737420696E697421
:108550002825303458292C777269746520696E6635
:108560006F6D6174696F6E20746F20666C617368E3
:108570002E0A00004261636B206D61634164647286
:108580005F4C3A00253032583A0000000D0A0000D6
:108590004261636B206D6163416464725F523A00B3
:1085A0004261636B20446174613A6966636F6E6611
:1085B00069673A25642C686172645665723A25646D
:1085C0002C6261636B75702E736F6674766572735F
:1085D000696F6E3A25640A00466C617368206865AD
:1085E0006164207365636F6E642072656164282521
:1085F000303458292E0A0000466C61736820777267
:108600006974652068656164206661696C2E0A0082
:10861000466C61736820777269746520686561646F
:10862000206661696C00000053797374656D207277
:10863000657365742E2E2E0A0000000004EB4401C1
:108640002E4A52F82100FDF73FFF054604EB440097
:108650002A4901EB8000007A009004EB44000A46AE
:1086600002EB8000436804EB440052F820102A46D5
:1086700023481CF0ABFB601C84B2192CFFF6A7AE9C
:10868000204A21A1002002F017FB23A1002002F0C4
:1086900013FB01201B49393908710321102019F0FF
:1086A00077F8642018F0E2FD102000BF4FF0A042E0
:1086B000114600BFD1F81025C24002F00102114856
:1086C000393802710079012804D10121102019F0F4
:1086D0005FF803E00021102019F05AF809483938F2
:1086E000007920B110A1002002F0E6FA03E016A103
:1086F000002002F0E1FA00BF52E6000010A20400E0
:10870000983F0020CD51002065727220636F646530
:10871000203A25730A000000466C61736820696E78
:108720006974206F6B2E0A003D3D3D3D3D3D3D206F
:108730004C656674202073686F6F65203D3D3D3D3C
:108740003D3D3D200A0000003D3D3D3D3D3D3D207D
:1087500052696768742073686F6F65203D3D3D3DC9
:108760003D3D3D200A00000070B500250026104860
:108770001049086000240CE04FF4E62000EB0436BA
:1087800030461EF0DBFD05460DB1032070BD601CB8
:10879000C4B2012CF0DB072206494FF4E6201EF09C
:1087A0000BFE05460DB10220F0E70020EEE70000C9
:1087B000AA5555AA24520020F8B5002500242CE023
:1087C00004EB4401174A52F82100FDF77DFE0646EE
:1087D00004EB4400134901EB8000007A009004EBA5
:1087E00044000A4602EB8000436804EB440052F860
:1087F000201032460C481CF066FD05465DB104EBC6
:108800004400084951F820202B4608A1002002F01E
:1088100053FA0220F8BD601CC4B2192CD0DB002032
:10882000F8E7000010A20400983F0020466C617336
:10883000685F53617665496E666F6D6174696F6ECE
:10884000206661696C206E616D652025732C7265F0
:1088500073756C742025640D0A000000F8B5064697
:108860000F46144633212548FDF723FE01202349F6
:10887000383981F83800012E0CD06FF48050304424
:1088800078B1B0F5405F1CD06FF440510844002827
:1088900029D10DE032221AA11848401CFDF7F0FD45
:1088A00028E032221CA11548401CFDF7E9FD21E01B
:1088B000254620A11148401CD5E9003204F0E4FB14
:1088C00018E025462868009021A10C48401CD5E9F5
:1088D000013204F0D9FB094B5B1C22A10020AA68DD
:1088E00002F0EAF906E03A4624A10448401C04F0EC
:1088F000CBFB00BF00BFFFF75FFFF8BDCC510020EE
:1089000053443A20415353455254494F4E20464117
:10891000494C45440D0A000053443A20494E564103
:108920004C4944204D454D4F5259204143434553F6
:10893000530D0A00415353455254494F4E2046416E
:10894000494C45442025733A25750D0A0000000066
:108950006572726F723A25752C25733A25750D0A6A
:10896000000000003E3E3E3E3E65727220636F6432
:1089700065203A25642C257300000000554E4B4EAF
:108980004F574E204641554C5420307825303858AA
:108990000A000000FEB55348406AB0F5006F7DD272
:1089A00009F074F8074609F077F83D184FF07F405A
:1089B00000EA05604FF47F0101EA052108434FF406
:1089C0007F4101EA1521084340EA156002904648BC
:1089D000007801280ED1FFF758FB28B143A10B20E6
:1089E000FFF7B4F90220FEBD00213E48416200209D
:1089F0003D4908703B48406A00902A463FA100204C
:108A0000029B02F059F93749496A4FF4EC2202EB14
:108A10008100012202A91EF0CFFC06460EB1022001
:108A2000E1E73048406A401C2E49486208464169E7
:108A3000C16181690162FFF7BFFE18B138A108204A
:108A4000FFF784F904240020019044E004EB440182
:108A5000394A52F82100FDF737FD074604EB440080
:108A6000354A52F8201001AB3A4634481CF0BAFAA5
:108A700078BB04EB4400304901EB8000007A9DF89C
:108A80000410884225D104EB44012B4A52F82100FE
:108A9000FDF71AFD074601A8009000E01EE004EB78
:108AA0004400254A02EB8000436804EB440052F87E
:108AB00020103A4621481CF051FA50B90948436940
:108AC00004EB44001C4951F820201DA1002002F0B5
:108AD000F3F8601CC4B2052CB8DB01E0022082E789
:108AE000002080E794510020B43F0020636C656152
:108AF000722073746570206661696C0073746570B0
:108B00002025642C666C6173685F646174613A252A
:108B1000642C737465705F6E756D3A25640A00008D
:108B20007361766520696E666F726D6174696F6ED0
:108B3000206661696C00000010A20400983F0020CC
:108B40003E3E3E3E3E3E3E3E25732076616C756560
:108B50003A25640A000000002DE9F84F00260020A5
:108B600000904FF480770125002410E0384618F07B
:108B7000C1FF40B100BF25480068284018B1384601
:108B800018F0AAFF2E436D00381D87B2641C082C14
:108B9000ECD34FF4BE7018F0ADFF50B14FF4BE707F
:108BA00018F09AFF46F000466A460121002018F0AE
:108BB00085FEF0B210B3012500241DE005EA060091
:108BC000C0B100BF124850F82400C0F30420814611
:108BD00000BF0F4850F82400C0F3014082462046F1
:108BE0000CF00AFD8046B8F1000F02D0514648460D
:108BF000C04700BF6D00641C082CDFD306F00040A6
:108C000010B168461CF098FBBDE8F88F0463004083
:108C10001065004000200F49096891ED070AF6EE43
:108C2000000A30EE200ABCEEC00A10EE101AC8B2DC
:108C30000A2806DD0A2190FBF1F000EB80014906CD
:108C4000080E642801DD642002E0002800DC00201A
:108C5000704700004440002000BFEFF308808046CA
:108C600000BFEFF3098000BF4046FFF717F80A2462
:108C700004B90DE000BF4FF47A7505B904E0134E56
:108C8000AF013846B04700BF601E041EF3D100BFDD
:108C900000BF00BF00BF00BF00BFBFF34F8F00BFCA
:108CA00000BF00BF0A48006800F4E06009490843BB
:108CB000001D0749086000BF00BF00BFBFF34F8F12
:108CC00000BF00BF00BF00BF00BFFDE791A10400CF
:108CD0000CED00E00000FA0510B500210C2018F0A2
:108CE000AEFE012019F080FC00210D2018F0A7FE37
:108CF000012019F079FC01210C2018F0A0FE0120C0
:108D000019F072FC00210C2018F099FE10BD1CB562
:108D10000020009003460122114601900C2018F01B
:108D2000B7FC0C2018F0ACFD0C2018F010FE002051
:108D3000009003460122114601900D2018F0A8FC76
:108D40000D2018F09DFD0D2018F001FE1CBD10B582
:108D500000210C2018F073FE01210D2018F06FFE89
:108D6000012019F041FC01210C2018F068FE0120BF
:108D700019F03AFC00210C2018F061FE10BD2DE91D
:108D8000F04107460E4615469846002400F084F848
:108D9000384600F057F800F0AFF810B90020BDE8F1
:108DA000F081304600F04EF800F0A6F808B9002037
:108DB000F5E700F071F8791CC8B200F043F800F054
:108DC0009BF808B90020EAE7002406E000F012F85A
:108DD0002855FFF781FF601CC4B2A8F10100A04232
:108DE000F4DC00F007F82855FFF7B1FF00F06CF84D
:108DF0000120D4E770B5002501210D2018F01FFED9
:108E000000BF17E06006040E00210C2018F017FECA
:108E1000052019F0E9FB01210C2018F010FE0520B7
:108E200019F0E2FB0D2018F07AFD08B144F00104BE
:108E3000681CC5B2082DE5DB00210C2018F0FFFDF1
:108E4000204670BD70B50446002500BF1DE000211E
:108E50000C2018F0F4FD052019F0C6FB04F080008A
:108E600020B101210D2018F0EAFD03E000210D20C2
:108E700018F0E5FD6006040E01210C2018F0DFFD5E
:108E8000052019F0B1FB681CC5B2082DDFDB0021FD
:108E90000C2018F0D4FD70BD10B501210D2018F084
:108EA000CEFD01210C2018F0CAFD052019F09CFB15
:108EB00000210D2018F0C3FD052019F095FB0021BD
:108EC0000C2018F0BCFD10BD10B500210C2018F0CE
:108ED000B6FD00210D2018F0B2FD052019F084FB2D
:108EE00001210C2018F0ABFD01210D2018F0A7FD89
:108EF000052019F079FB10BD10B5002401210D20CB
:108F000018F09DFD012019F06FFB01210C2018F0D5
:108F100096FD0BE0601CC0B20446322803DBFFF76D
:108F2000D3FF002010BD012019F05EFB0D2018F0CA
:108F3000F6FC0028EED100210C2018F080FD012065
:108F4000F0E72DE9F04180460D4616461F46002405
:108F5000FFF7A2FF4046FFF775FFFFF7CDFF10B9FF
:108F60000020BDE8F0812846FFF76CFFFFF7C4FF43
:108F700008B90020F5E7002409E0305DFFF762FF43
:108F8000FFF7BAFF08B90020EBE7601CC4B2BC428F
:108F9000F3DBFFF799FF0120E3E7000010B5054878
:108FA000007828B1044B054A0549064800F0E8F866
:108FB00010BD0000D047002055CB0300E44700203F
:108FC000D44700204A8600200120014908707047DC
:108FD000D04700200020014908707047D04700208A
:108FE0002DE9FC5F05460E4617469846DDE90CB9AB
:108FF000DDF838A04448007868B15B4642463946FF
:109000003046CDE9009A1CF07DFE4049A1F15000A8
:1090100012F074FB0CE05B46424639463046CDE91F
:10902000009A0CF047FF3949A1F150000CF0F4FE12
:10903000304617F085F90446002C62D034A1002098
:1090400001F03AFECDB33048007828B12F495039AD
:1090500034481CF081FF54E0334890F850302B48DE
:10906000503890F85010304A0CF0FEFE2F49A1F114
:1090700050000CF0E5FE2D485038B0F85200401C6E
:109080002A495039A1F85200084690F8521090F839
:109090005000401C254A503A11541046B0F8520076
:1090A0000012114691F850105054104690F850306C
:1090B000042100201EF09EFF23E0FFE713485038F4
:1090C000B0F85200401C11495039A1F8520008462E
:1090D00090F8521090F85000401C0C4A503A11542D
:1090E0001046B0F852000012114691F8501050543A
:1090F000104690F85000801CC3B2042100201EF0DE
:1091000079FFBDE8FC9F0000D0470020F2850020D9
:109110004E4545445F53454E445F444154412E2ED5
:109120002E2E0A00D44700204E85002046860020BF
:1091300070B504460D46E07804281AD16278211DE6
:109140000C48FDF79DF96078C01F0A4981F850006E
:109150006078801E215C6078C01E205C41EA00209F
:109160000449A1F852000448007810B103481CF0EB
:10917000F3FE70BD4E850020D0470020E44700205C
:109180002DE9F04104460E4615461F466548007815
:1091900010B101280CD10CE06889002808DD0120FD
:1091A0006049087028461DF057F830461DF054F805
:1091B000B5E008E004F1540128461CF00DFFB4F8B6
:1091C000A60059490880688971898842F2DC68895B
:1091D000002867DD04F1540128461CF0FDFE5248CA
:1091E0000088401C50490880B4F8A60009888842CD
:1091F00059D000BF4D480088401C4C4908804A485F
:109200000088401C48490880214630461CF0E4FE96
:10921000B4F852004449098888423BD1214630467F
:109220001CF0DAFE94F8A43094F8501004F15402C3
:109230002046B8473E49A1F1500012F071FA3C486F
:109240005038B0F85200401C39495039A1F852004A
:10925000084690F8521090F85000401C344A503A9A
:1092600011541046B0F852000012114691F85010F7
:1092700050541146B1F8520000EBD0714910A0EBE8
:10928000410131B9104690F85030042100201EF001
:10929000B1FE07E07089002803DC00202149087036
:1092A00000E0A7E73AE0214630461CF095FE94F82E
:1092B000A43094F8501004F154022046B8471C49D9
:1092C000A1F1500012F02CFA19485038B0F85200B1
:1092D000401C17495039A1F85200084690F8521026
:1092E00090F85000401C124A503A11541046B0F801
:1092F00052000012114691F8501050541146B1F826
:10930000520000EBD0714910A0EB410131B9104679
:1093100090F85030042100201EF06CFE00BF00BF0A
:10932000BDE8F081F4470020F64700207A3F002096
:109330004686002070B505460C4600202649086088
:10934000264800210160416081602548016041603C
:1093500081604FF4A2712348FDF7ABF82248002149
:109360000160416081602148016041608160204866
:1093700001604160816024211E48FDF79AF8242194
:109380001D48FDF796F86C211C48FDF792F84FF444
:10939000A2711B48FDF78DF824211A48FDF789F8C2
:1093A00024211948FDF785F824211248FDF781F89A
:1093B00024211148FDF77DF8144890ED000A21465C
:1093C000114813F047FA24220F491148FDF758F8C5
:1093D00000201049086070BD744900206C91002085
:1093E00078910020A08D0020E48E00205491002070
:1093F00060910020F08E0020148F0020388F002014
:10940000A48F0020E89000200C9100206C490020DF
:1094100030910020984900202DE9F0412DED048B7A
:1094200086B005460027002618216846FDF741F85A
:10943000B0460024288810FB00F06A8812FB020066
:10944000AA8812FB020000EE100AB8EEC00A10EE65
:10945000101A0846FDF757FA41EC190BB0EE490A0D
:10946000F0EE690A04F064FBB0EE408AF0EE608A28
:1094700051EC180BFDF70FFA064627480078012833
:109480000CD100202449087000BF04E0234840F8B4
:109490002460601CC4B2062CF8DB0DE0002407E059
:1094A0001E49601C51F8200041F82400601CC4B221
:1094B000052CF5DB19484661182218496846FCF767
:1094C000DFFF002119E0002011E05DF82030421C90
:1094D0005DF82220934208DD421C5DF822805DF891
:1094E00020304DF822304DF82080421CD0B2C1F11E
:1094F00005028242E9DC481CC1B20529E3DB009980
:109500000598401AB0F57A7F00DB0127384606B08F
:10951000BDEC048BBDE8F0814C4000202474002099
:1095200010B500210E2018F050FA002001490870F3
:1095300010BD00005C40002010B5012001F04EFE7F
:10954000FF231A461946122001F04EFE032001F0B7
:109550005BFE00F0D3FF00231A4660210F4800F0A5
:10956000D1FF0F4908600E2018F029F901210E20C3
:1095700018F02BFA112018F022F90021112018F010
:1095800024FA084A08A1052000F058FE094801F015
:109590006DFE094803F09AFB10BD00004C740020DA
:1095A00058400020BD9502004C45445F50726F63E7
:1095B00065737300C9510300DB51030010B500242B
:1095C0002348007810B101283BD126E021480078DB
:1095D00010B300201F49087007240DE01E4810F842
:1095E0003400002806DD1C4901EBC401486803F083
:1095F0006FFA03E0601EC4B2002CEFDC00BF24B998
:1096000000210E2018F0E1F906E001210E2018F0EB
:10961000DCF901200E49087017E00E48007848B1C7
:1096200000200B490870AFF26B020CA1052000F07E
:1096300005FE05E0012204210B48006801F0EAFD67
:1096400003E000200249087000BF00BF10BD000009
:109650005D4000205C4000200C7500204C45445FBC
:1096600050726F63657373005840002070B50446F4
:109670000D46082C00DB70BD0F4810F8340001289F
:1096800006D10D4800EBC4004068A84200D1F2E7C3
:109690000120094901F83400084600EBC400456088
:1096A0000120064908702B46224605A1002001F042
:1096B00003FB00BFDFE700000C7500205C400020CA
:1096C0004C45445F53746172743A25642C25580AE2
:1096D00000000000082800DB7047074911F830102F
:1096E00001B9F9E70021044A02F830100121034AC8
:1096F000117000BFF0E700000C7500205C400020F6
:1097000010B50021082018F0AFF9012018F078FFFB
:109710000021072018F0A8F9012018F071FF01219D
:10972000082018F0A1F9012018F06AFF0021082094
:1097300018F09AF910BD1CB50020009003460122D4
:1097400011460190082017F0B7FF082018F0A7F87D
:10975000082018F007F90020062103460122CDE970
:1097600000101146072017F0A7FF072018F097F800
:10977000072018F0F7F8092018F045F80121092012
:1097800018F072F9062018F03EF81CBD10B5002143
:10979000082018F069F90121072018F065F9012067
:1097A00018F02EFF0121082018F05EF9012018F0B2
:1097B00027FF0021082018F057F910BD2DE9F041CE
:1097C00007460E4615469846002400F084F83846B1
:1097D00000F057F800F0BDF810B90020BDE8F081A6
:1097E000304600F04EF800F0B4F808B90020F5E774
:1097F00000F071F8791CC8B200F043F800F0A9F845
:1098000008B90020EAE7002406E000F012F8285525
:10981000FFF776FF601CC4B2A8F10100A042F4DC9F
:1098200000F007F82855FFF7B1FF00F06CF80120B1
:10983000D4E770B500250121072018F015F900BF05
:1098400017E06006040E0021082018F00DF905202D
:1098500018F0D6FE0121082018F006F9052018F0AE
:10986000CFFE072018F067F808B144F00104681C27
:10987000C5B2082DE5DB0021082018F0F5F82046D8
:1098800070BD70B50446002500BF1DE00021082012
:1098900018F0EAF8052018F0B3FE04F0800020B1BB
:1098A0000121072018F0E0F803E00021072018F05C
:1098B000DBF86006040E0121082018F0D5F8052019
:1098C00018F09EFE681CC5B2082DDFDB00210820C1
:1098D00018F0CAF870BD10B50121072018F0C4F8BF
:1098E0000121082018F0C0F8052018F089FE002199
:1098F000072018F0B9F8052018F082FE0021082092
:1099000018F0B2F810BD10B50021082018F0ACF81E
:109910000021072018F0A8F8052018F071FE012199
:10992000082018F0A1F80121072018F09DF8052063
:1099300018F066FE10BD10B5082017F01DFF0720B7
:1099400017F01AFF092017F017FF062017F014FF71
:1099500010BD10B500240121072018F085F8012062
:1099600018F04EFE0121082018F07EF80BE0601C74
:10997000C0B20446322803DBFFF7C5FF002010BD4C
:10998000012018F03DFE072017F0D5FF0028EED18A
:109990000021082018F068F80120F0E72DE9F041D7
:1099A00080460D4616461F460024FFF794FF4046AA
:1099B000FFF767FFFFF7CDFF10B90020BDE8F0818A
:1099C0002846FFF75EFFFFF7C4FF08B90020F5E760
:1099D000002409E0305DFFF754FFFFF7BAFF08B934
:1099E0000020EBE7601CC4B2BC42F3DBFFF78BFF47
:1099F0000120E3E77CB506F009FEF8B1002512F07E
:109A0000A3FC4042C6B20E48058800242A12214613
:109A1000641C0DF80120EAB22146641C0DF80120F7
:109A20002146641C0DF8016023466A46032100208C
:109A3000FDF7BAFC00200249088000BF7CBD000091
:109A40007A3F00200348006808B1012070470020D9
:109A5000FCE70000044000202DE9F0410220012134
:109A60000A4600242346254600BF4FF0A0473E4645
:109A700041EA420747EA840747EA032747EA054CD9
:109A800006F5E06747F820C000BF00BF002117F0CF
:109A90007FFF642000F01EF8084802F0BDFB084A72
:109AA00008A1002000F0CAFB0121054800F0A2FB3C
:109AB0000749A420FDF7A2FBBDE8F081159B020039
:109AC000B99B02004D545F70726F63657373000041
:109AD000A54D030010B50446224608A1002001F060
:109AE000EBF84CB1094804600121022017F050FF47
:109AF0000121074800F07EFB10BD00004D54204DB1
:109B0000545F52756E3A2564200A0000044000201C
:109B1000B99B020010B5044623480068002842D0D3
:109B20002148006868B320480068401E1E4908604C
:109B30001E480068082809D00121022017F028FFDC
:109B40001A480068401C194908600CE01848006871
:109B5000022808D016480068401C154908600021FA
:109B6000022017F015FF11480068082810D110488E
:109B7000006802280CD100200D4908600B490860DC
:109B800006E00020084908600949086007490860A4
:109B90000548006838B90021022017F0F9FE0021BD
:109BA000044800F027FB10BD044000200C400020BA
:109BB00008400020B99B02007047000010B54FF428
:109BC000807017F02EFB80B14FF4807017F032FBDD
:109BD000012017F039FB2048407930B901201E4997
:109BE000487108460168002088474FF4827017F0DA
:109BF00018FB50B14FF4827017F01CFB022017F0D5
:109C000023FB15480168012088474FF4887017F03E
:109C100008FB50B14FF4887017F00CFB102017F0C0
:109C200013FB0D480168022088474FF4867017F037
:109C3000F8FA80B10020094908604FF4867017F0E7
:109C4000F9FA082017F000FB002003498871084644
:109C500001680320884710BD904A0020340C004062
:109C60002DE9F0411FF0B0FE0FF006FD1521032095
:109C7000002213461446154600BF0F073E4642EA2F
:109C8000430747EA800747EA042747EA054C06F5F9
:109C9000E06747F821C000BF00BF00F017F8FFF7EA
:109CA0004BFCFFF7D9FEFEF70FFAFEF78BF81FF01B
:109CB0005BFDBDE8F081000010B50249024813F0D9
:109CC000D7FE10BDA04A002000C0014010B5034AD5
:109CD00003A142F2107000F0B1FA10BDA99D02007C
:109CE0005057525F50726F63657373002DE9F041F6
:109CF0001321084602F0E0FCFFF712FC09F00CFE0D
:109D00000220002161B900BF00BF4FF0A0421346FE
:109D1000012505FA00F2C3F80C2500BF00BF0CE0D6
:109D200000BF00BF4FF0A0421346012505FA00F224
:109D3000C3F8082500BF00BF00BF00BFC82017F050
:109D4000ADFA19200021022200231D461E4600BF45
:109D50004FF0A04C674643EA450C4CEA810C4CEAB4
:109D6000062C4CEA024C07F5E06848F820C000BF1A
:109D700000BF33DF0446FEF74DFF054623462A4663
:109D800002A1002000F098FFBDE8F081706F7765B8
:109D900072206F66662E2E2E4241543A25642C4561
:109DA00052523A25640A000010B5FEF733FF00282E
:109DB0003FD105F045FB01283BD1FEF72BFF0446C0
:109DC00022461CA1002000F077FF1FA1002000F018
:109DD00073FFFEF7DFFD18B11FA10D20FDF7B6FFE1
:109DE000242221492148FCF74BFB002020494876DA
:109DF000FEF7BAFC18B11FA10D20FDF7A7FFFEF773
:109E0000DBFC18B121A10D20FDF7A0FF4FF47A7003
:109E1000FFF760FE0FF030FC002406E005F0E8FCE0
:109E2000642017F03BFA601CC4B20A2CF6DBFFF783
:109E30005DFF10BD4261747465727950657273651F
:109E40006E743A25640A0000706F776572206F6641
:109E5000662E2E2E0A0000007361766520737465ED
:109E600070206661696C00005C4F00200052002089
:109E700024520020707772207361766520626163DE
:109E80006B7570206661696C000000007361766517
:109E900020696E666F726D6174696F6E20666169AC
:109EA0006C00000010B52DED048BF0EE408AB0EE92
:109EB000608A9FED9F0AB0EE409A9E48006890F835
:109EC000210020B1012833D0022830D183E0B3EE45
:109ED000040AB4EEC08AF1EE10FA1BDD02209549A7
:109EE000096881F82100B0EE680A0BF0BFFC9148C8
:109EF000006880ED050A8F480068D0ED050AB0EED5
:109F0000600AF0EE490A15F0A1F88A48006880ED71
:109F1000060A0CE0B0EE680A02F05CFD85480068B5
:109F200080ED050A01208349096881F82100F7E0E6
:109F3000B3EE040AB4EEC08AF1EE10FA19DD022085
:109F40007C49096881F821009FED7B0A7948006807
:109F500080ED030A77480068D0ED050AB0EE600A8C
:109F6000F0EE490A15F072F87248006880ED060AB2
:109F700030E0B0EE680A02F02DFD6E48006880ED1A
:109F8000040A6C48006890ED050A6A480068D0ED44
:109F9000040AB4EEE00AF1EE10FA07DD6548006845
:109FA00090ED040A6348006880ED050A0BF0BEFCE2
:109FB00080B16048006890ED050ADFED600AB4EEFC
:109FC000E00AF1EE10FA05DD9FED5D0A59480068E0
:109FD00080ED050AA4E0B3EE040AB4EEC08AF1EE07
:109FE00010FA22D201205349096881F82100B2EE0B
:109FF000040AC8EE800A4F480068C0ED000A4D48C8
:10A00000006890ED050ADFED4F0AB4EEE00AF1EECC
:10A0100010FA09DD0BF08AFC002805D09FED480AF4
:10A020004448006880ED050A79E0F7EE000A4148EF
:10A0300000681830B0EE480AFDF7B6FC3D480068ED
:10A04000D0ED060AB0EE600AF0EE490A02F0B6FC66
:10A050003848006880ED020AB0EE680A0BF006FC92
:10A060003448006880ED040A9FED370AC8EE000A04
:10A0700030480068C0ED030A2E48006890ED030ADE
:10A08000F7EE000AB4EEE00AF1EE10FA05DDB7EEE5
:10A09000000A2848006880ED030A2648006890ED11
:10A0A000030AF7EE000A30EEC00A22480068D0ED3D
:10A0B000040A20EE200A1F480068D0ED030A1D485C
:10A0C000006890ED021A00EE810A1A48006880EDDF
:10A0D000040A1848006890ED050A16480068D0ED9B
:10A0E000040AB4EEE00AF1EE10FA07D21148006853
:10A0F00090ED040A0F48006880ED050A0D480068DD
:10A1000090ED050ADFED0E0AB4EEE00AF1EE10FA6A
:10A1100005DD9FED0E0A0748006880ED050A00BFC7
:10A1200000BF0448006890ED050ABDEC048B10BD2B
:10A130000000AF4344400020000000000000BE4289
:10A140000000C8423333C64200007A44CDCCC74237
:10A1500070B50025002400BF33E02046FDF72EFD3A
:10A16000224800EB0410007B00B928E01F4800EBF8
:10A170000410806810B31D4800EB0410408828B913
:10A180001A4901EB04118868804717E001F0E0FFED
:10A19000164901EB04114968401A144901EB0411F6
:10A1A000498888420AD301F0D3FF104901EB04111A
:10A1B00048600E4901EB04118868804700BF601CAD
:10A1C000C4B20B4800788442C7DB002407E007488C
:10A1D00000EB0410007800B10125601CC4B20448F3
:10A1E00000788442F3DB284670BD0000784B0020E5
:10A1F000D63D002010B50246002014E00D4B03EBC5
:10A2000000139B6893420CD10A4B03EB00131B789D
:10A210008B4205D001F00103064C04EB00142370BF
:10A2200010BD431CD8B2044B1B789842E6DB00BF3C
:10A23000F6E70000784B0020D63D00202DE9F041E4
:10A2400005460F461646002419E0234800EB04108B
:10A250008068B04211D101201F4901EB041108733D
:10A260001D4800EB0410458001F072FF1A4901EB14
:10A27000041148600120BDE8F081601CC4B2174899
:10A2800000788442E1DB154800783C2802DB4FF07F
:10A29000FF30F0E710481149097800EB01108660A3
:10A2A00001210D480D4A127800EB021001730A4893
:10A2B0000A49097800EB0110458001F049FF064981
:10A2C000064A127801EB0211486004480078401CED
:10A2D000024908700020CEE7784B0020D63D0020D0
:10A2E0000146002011E00C4A02EB001292688A42FB
:10A2F00009D10022084B03EB00131A73064B03EB42
:10A3000000131A707047421CD0B2044A127890426F
:10A31000E9DB00BFF6E70000784B0020D63D0020C7
:10A32000024600200CE0094B03EB00139B689342AC
:10A3300004D1064B03EB001359807047431CD8B27D
:10A34000034B1B789842EEDB00BFF6E7784B00200A
:10A35000D63D00202DE9F04105460320FDF74AFBDC
:10A360000746052D01DABDE8F081002426E01748F4
:10A3700000EB04100078B8421FD1144800EB041021
:10A38000C068D0B1002609E0311D88B2FDF732FB6C
:10A390000E4901EB041149688855761C681FB042CC
:10A3A000F2DC0A4901EB04110872084A02EB0410BE
:10A3B00002EB0412D168884704E0641C044800687A
:10A3C0008442D4D300BF00BFCDE700004056002038
:10A3D000D83F0020F0B5C1B005460320FDF71AFBB9
:10A3E0000746052F12DA002406E0211D88B2FDF78A
:10A3F00011FB01A90855641C681FA042F5DCC3B21B
:10A4000001AA39460020FDF7ABF900BF052D01DA9E
:10A4100041B0F0BD002426E0164800EB041000789F
:10A42000B8421FD1134800EB0410C068D0B1002619
:10A4300009E0311D88B2FDF7EDFA0E4901EB041178
:10A4400049688855761C681FB042F2DC094901EB67
:10A4500004110872074A02EB041002EB0412D168DF
:10A46000884704E0641C044800688442D4D300BFD9
:10A4700000BFCDE7505C0020F43F00202DE9F04103
:10A4800005460320FDF7D6FA0746052D01DABDE89B
:10A49000F081002426E0174800EB04100078B84251
:10A4A0001FD1144800EB0410C068D0B1002609E0A9
:10A4B000311D88B2FDF7BEFA0E4901EB041149685F
:10A4C0008855761C681FB042F2DC0A4901EB041182
:10A4D0000872084A02EB041002EB0412D1688847A4
:10A4E00004E0641C044800688442D4D300BF00BF69
:10A4F000CDE70000606200202040002010B500F091
:10A5000025F810BD2DE9F04107460C4615461E46BC
:10A510000848807A30B1002000F070FE00F00EF89C
:10A52000FFF7ECFF0448076084808560C660BDE8E3
:10A53000F08100009C4000201C7C002010B50248E7
:10A5400018F0EEF910BD00009440002070B5002511
:10A55000084809490268094818F016F9044604B188
:10A560006D1E681C20B9064A06A10020FFF766FE92
:10A5700070BD0000A84000209C40002094400020B6
:10A58000194003006273705F70776D5F696E697464
:10A590005F70726F636573730000000010B5034A4B
:10A5A0001068034A1168884710BD0000E84A00207F
:10A5B000E44A002010B504220021024813F0FCF9FF
:10A5C00010BD0000004002402DE9F0472DED068B44
:10A5D00086B005460E4617464FF00008C146C246F3
:10A5E000002005E035F9101003AA42F82010401CA5
:10A5F0000328F7DB0598002801DB014600E0414213
:10A600008846002004E036F910104DF82010401C58
:10A610000328F8DB0298002801DB014600E04142F4
:10A620008946EE48007803280CDBED484068EC4989
:10A6300008600846806848600220E84908700120E8
:10A64000E8490860E54801780078401CE34A10704A
:10A65000E34840F82180E448007803280CDBE34815
:10A660004068E24908600846806848600220DE4988
:10A6700008700120DB490860DB4801780078401C45
:10A68000D94A1070D94840F82190D9480078032859
:10A690000CDBD8484088D749088008468088488025
:10A6A0000220D34908700120CE490860B888404292
:10A6B00001B2CF4802780078401CCD4B1870CD48CD
:10A6C00020F81210C748006801287DD1C44880686E
:10A6D000C3494968401A12D4C748008820B9C04805
:10A6E0008068C649086011E0BD488068C3490968B0
:10A6F00088420BDDBA488068C049086006E0BE4861
:10A70000008818B9B6488068BD490860B7488068B5
:10A71000B6494968401A12D4BA48008820B9B348EB
:10A720008068B949086011E0B0488068B649096896
:10A7300088420BDDAD488068B349086006E0B14847
:10A74000008818B9A9488068B0490860A4488068A2
:10A75000AB490968401A40F69801884212DD012091
:10A76000A54908809E488068A5490968401AA849FB
:10A770000968884206DD9A488068A1490968401A3C
:10A78000A349086099488068A0490968401A40F6C2
:10A790009801884212DD01209A4908809348806818
:10A7A0009A490968401A9B490968884206DD8F4822
:10A7B000806896490968401A964908608848806808
:10A7C0008F490968401A00E0EEE040F2DC5188420F
:10A7D00028DD8F480068FCF740F841EC1A0B9FED2C
:10A7E0008E0B53EC102BFBF741FF41EC180B7C490F
:10A7F0008968824A1268501AFCF72FF841EC190B4D
:10A8000053EC182BFCF792F813D275488068744902
:10A810004968441A002C01DB204600E06042B0F594
:10A82000C87F06DA00207449088040F6980078490D
:10A8300008606E48806875490968401A40F2DC512A
:10A84000884228DD73480068FCF707F841EC1A0BD2
:10A850009FED710B53EC102BFBF708FF41EC180B2D
:10A8600062498968684A1268501AFBF7F6FF41ECA2
:10A87000190B53EC182BFCF759F813D25B4880687E
:10A880005A494968441A002C01DB204600E0604226
:10A89000B0F5C87F06DA00205A49088040F69800D3
:10A8A0005C4908605648006810B900205249088089
:10A8B0005648006810B9002052490880584800885E
:10A8C00038BB5848B0F90000B0F5967F05DA554816
:10A8D0000088401C00B2534908800020524908807B
:10A8E00045480088012803D04648008801280AD13D
:10A8F0004C48B0F90000082805DB4FF0010A0120A0
:10A900004749088062E04FF0000A0020444908806F
:10A910005CE04FF0000A4448B0F90000B0F5967FC3
:10A9200005DA41480088401C00B23F4908800020F9
:10A930003C4908803C4BB3F90030062B30DB2E4BF2
:10A940001B886BBB2B4BB3F90030A3F5FA62002ACE
:10A9500001DB134600E05342B3F5967F19DC254B2B
:10A96000B3F90230A3F5FA61002901DB0B4600E0E0
:10A970004B42B3F5967F0CDC1E4BB3F90430A3F5C4
:10A98000FA60002801DB034600E04342B3F5967FFE
:10A9900006DD1C4B1B881BB900202149088015E0EF
:10A9A00001201F49088011E04FF0000A0C48806820
:10A9B000134908600A488068104908600B4880689D
:10A9C00012490860094880680F4908600AF0FF00D2
:10A9D00006B0BDEC068BBDE8F0870000DC49002026
:10A9E000AC950020E8490020DD490020B895002002
:10A9F000E4490020EC490020C6490020D04900204D
:10AA0000CC490020C8490020D8490020D449002062
:10AA1000F4490020F84900209A9999999999D93FC9
:10AA2000E2490020E0490020DE490020FEB54FF455
:10AA3000827017F011FB002837D04FF4827017F0A6
:10AA400015FB6C4890F82E0018B16A4890F82F005A
:10AA500058B300208DF800006648406801906548B2
:10AA60000189ADF80810C06818B900206149087460
:10AA700012E06048008B5F4948830846C068486020
:10AA80000846008B08810020C860084690F82E0018
:10AA900010B9002017F00CFB56480168684688473B
:10AAA0000020544981F82F0000BF524890F82E0032
:10AAB000002852D04FF4807017F0CEFA00284CD006
:10AAC0004FF4807017F0D2FA4A48408B494991F808
:10AAD0002D10884216DD4748408B464991F82D10CD
:10AAE000401A444948830A4612890B465B8BD21AA6
:10AAF0000B465B6803EB42000A4692F82D1017F0F4
:10AB000097FA23E03B48408B3A4991F82D10884250
:10AB10000FD13848C06860B10120364981F82F0054
:10AB2000002048830A4692F82D10D06817F080FA6A
:10AB30000CE03048408B2F4991F82D10884205D108
:10AB400001202C4981F82F00002048834FF48270A7
:10AB500017F08CFA042017F0ABFA4FF4887017F056
:10AB60007BFA70B14FF4887017F080FA0020214909
:10AB7000087402208DF8000008460168684688477E
:10AB800000BF4FF48A7017F067FA38B14FF48A703B
:10AB900017F06CFA0020174908742AE01548456937
:10ABA00024E0B5FA85F64FF00040F0408543B00050
:10ABB00000F58C74204617F04FFAB8B1204617F014
:10ABC00055FA01208DF80000A4F58C70C0F3C70081
:10ABD0008DF80400A4F58C70012121EA90018DF814
:10ABE0000510044801686846884700BF002DD8D189
:10ABF00000BFFEBD0C9A0020F8B504460D4616466F
:10AC000000BF0B48007808B902F088F800BF0020A8
:10AC10000090684607F04FF932462946204600F07A
:10AC200009F807469DF8000007F04CF93846F8BDD2
:10AC3000E09C00202DE9F047074688461646C246AC
:10AC400007EB47011B4800EBC109D9F8140020B1FC
:10AC5000012811D0022826D11EE0484602F096F8BD
:10AC60000546B54201D2002405E03446324651463D
:10AC7000484602F0E2F918E0484602F087F8054637
:10AC8000B54201D2284600E03046044622465146ED
:10AC9000484602F0D2F908E032465146484602F0F2
:10ACA00091F9044601E0002400BF00BF2046BDE842
:10ACB000F0870000F89C00200FB438B5044606A8C1
:10ACC00000906A462046059900F007F805460020E6
:10ACD0000090284638BC5DF814FB2DE9F04F99B080
:10ACE00082460D46144603A814904020159000207B
:10ACF0001690CDF860A0179000BF2E786D1C06B995
:10AD0000DDE0252E79D100274FF0010900BF2E7814
:10AD1000232E12D02B2E0CD02D2E02D0302E10D15F
:10AD200003E047F001076D1C0EE047F002076D1CC1
:10AD30000AE047F004076D1C06E047F008076D1CA9
:10AD400002E04FF0000900BF00BFB9F1000FDED1F3
:10AD50004FF0000800BF2E78302E01DB392E00DDC9
:10AD600007E06D1CA6F1300008EB880100EB4108FC
:10AD7000F1E700BF002013902E782E2E12D16D1C0B
:10AD800000BF2E78302E01DB392E00DD09E06D1C6E
:10AD9000A6F13000139901EB810100EB4100139003
:10ADA000EFE700BF2E7800BF6C2E01D0682E02D1D5
:10ADB0006D1C2E7800E000E0F6E700BF702E5DD03D
:10ADC00008DC252E6AD0582E35D0632E09D0642E8B
:10ADD00069D113E0732E3CD0752E1DD0782E62D130
:10ADE00028E02168081D2060D1F8009009F0FF0BD1
:10ADF000594614A802F0C4F856E058E02168081D2E
:10AE00002060D1F80090CDE900870A22494614A8B5
:10AE1000139B01F0C9FF47E02168081D2060D1F8AD
:10AE20000090CDE900870A22494614A8139B02F03E
:10AE300031F839E000BF2168081D2060D1F800908A
:10AE4000CDE900871022494614A8139B02F022F88E
:10AE50002AE02168081D2060D1F800B000BF9BF8EF
:10AE600000600BF1010B06B906E0314614A802F0B0
:10AE700087F817980028F2DA00BF15E02168081D4E
:10AE80002060D1F80090002008210B461022CDE967
:10AE90000010494614A801F0FDFF05E0252114A883
:10AEA00002F06EF800E000BF00BF6D1C03E0314609
:10AEB00014A802F065F817980028BFF61EAF00BF6F
:10AEC000179800280ADD169820B103A95046169A53
:10AED000FFF792FEDDE9161008441790179819B095
:10AEE000BDE8F08F0246002106E00548405C904234
:10AEF00001D100207047491C0029F6D00220F9E753
:10AF000008A4040070B505460C462846FFF7EAFF82
:10AF1000061E01D0304670BD012C04D10121284607
:10AF200016F070FD04E01CB90021284616F06AFDF9
:10AF30000020F0E710B5002409E00D49085D01216B
:10AF4000FFF7E0FF0A49085D16F00AFC641C002CBC
:10AF5000F3D0084816F093FA062016F001FC0720FB
:10AF600016F0FEFB082016F0FBFB002010BD0000D1
:10AF700008A40400D8A304007FB50025174B0FCB0D
:10AF80008DE80F0006208DF8020007208DF80100E3
:10AF900008208DF8000000208DF80C004FF00040D4
:10AFA000029006208DF8040000230D4A69460D48E2
:10AFB00016F008FA064606B16D1E002404E00A49A0
:10AFC000085D16F014FC641C002CF8D0681C20B935
:10AFD000064A07A10020FFF731F97FBD0CA4040049
:10AFE000E9910400D8A3040008A40400A9400300C8
:10AFF0006273705F737069305F696E69745F7072DD
:10B000006F63657373000000F8B506460F4614467B
:10B010001D462346002239463046009500F04EF882
:10B02000F8BDF8B506460F4614461D4623460122D4
:10B0300039463046009500F041F8F8BD2DE9F84F4B
:10B0400005460E4617469846DDF8289042F2107ADB
:10B050002846FFF747FF041E02D02046BDE8F88FC0
:10B0600000212846FFF74EFF002012490870434692
:10B070003A4631461048CDF8009016F0E7F90446FC
:10B080000CB10120EAE70AE0BAF10000AAF1010AD6
:10B0900005D101212846FFF735FF0120DEE70548ED
:10B0A00000780028F0D001212846FFF72BFF002070
:10B0B000D4E70000F8400020D8A304002DE9FC47A5
:10B0C00081460D4690461E460A9C4846FFF70AFFF9
:10B0D000071E02D03846BDE8FC87812C01D9032029
:10B0E000F9E7B8F1000F16D145F080000190601C1F
:10B0F000C0B2144B012201A900904846FFF79EFF01
:10B1000007460FB13846E6E722460E49491C30464D
:10B11000FBF7B6F913E00B48057022463146401C98
:10B12000FBF7AEF900200090601CC2B20023054975
:10B130004846FFF783FF07460FB13846CBE70020AC
:10B14000C9E70000847C002010B50249024812F0D3
:10B15000E1FC10BD549A00200030004010B50349B6
:10B160004FF0402012F0D6FC10BD0000789A00206D
:10B1700010B50249024812F0CDFC10BD9C9A002087
:10B180000030024070B50A4816F021F8044600BFAE
:10B19000254635B100BF07A262212846FBF73AF8E1
:10B1A00000BF00BF0CB1062070BD0020FCE700000E
:10B1B000C88200202E2E5C2E2E5C2E2E5C626C65CA
:10B1C0005F6366675C686F73742E630010B516F07A
:10B1D00026F810BD10B517F0BFF810BD0149487131
:10B1E000704700009C40002030B5034D2870697006
:10B1F000AA70EB7030BD00009C40002001498872AD
:10B20000704700009C400020014908817047000001
:10B210009C40002070B504460D46164633462A462B
:10B220002146024817F03AFB70BD00009440002010
:10B2300001480078704700008D41002010B50024BF
:10B240000BE0084850F8240028B1064850F82410B4
:10B250004FF47A708847601CC4B203480078844277
:10B26000EFDB10BD4C4B0020D43D002010B5044650
:10B27000002117E0104850F82100A04202D14FF001
:10B28000FF3010BD0C4850F8210048B90B48007839
:10B29000401C0A4A1070084840F821400020F0E79E
:10B2A000481CC1B20529E5DB05A10020FFF704FD1C
:10B2B0006FF00100E5E700004C4B0020D43D00207A
:10B2C000536C6565705F52656769737420746F6F46
:10B2D000206D616E79210A0002460020002100BF26
:10B2E00027E0411C22E000EBC0030B4402EB830388
:10B2F000D3ED000A01EBC103034402EB830393ED9A
:10B30000001A70EE810AB6EE001A20EE810A00EBF8
:10B31000C0030B4402EB830383ED000A01EBC1037E
:10B32000034402EB830383ED000A491C0929DADB9D
:10B33000401C0928D5DB704790ED031AD0ED061AA2
:10B3400001EE801A80ED031A90ED041AD0ED071A71
:10B3500001EE801A80ED041A90ED051AD0ED081A5E
:10B3600001EE801A80ED051A90ED0C1AD0ED0F1A3F
:10B3700001EE801A80ED0C1A90ED0D1AD0ED101A26
:10B3800001EE801A80ED0D1A90ED0E1AD0ED111A13
:10B3900001EE801A80ED0E1A90ED151AD0ED181AF4
:10B3A00001EE801A80ED151A90ED161AD0ED191ADB
:10B3B00001EE801A80ED161A90ED171AD0ED1A1AC8
:10B3C00001EE801A80ED171A90ED1B1AD0ED361A97
:10B3D00001EE801A80ED1B1A90ED1C1AD0ED371A81
:10B3E00001EE801A80ED1C1A90ED1D1AD0ED381A6E
:10B3F00001EE801A80ED1D1A90ED241AD0ED3F1A4F
:10B4000001EE801A80ED241A90ED251AD0ED401A35
:10B4100001EE801A80ED251A90ED261AD0ED411A22
:10B4200001EE801A80ED261A90ED2D1AD0ED481A03
:10B4300001EE801A80ED2D1A90ED2E1AD0ED491AEA
:10B4400001EE801A80ED2E1A90ED2F1AD0ED4A1AD7
:10B4500001EE801A80ED2F1A90ED1E1AD0ED391AE8
:10B4600001EE801AD0ED211A90ED3C2A42EE001A2E
:10B4700000EE211A80ED1E1A90ED1F1AD0ED3A1A37
:10B4800001EE801AD0ED221A90ED3D2A42EE001A0C
:10B4900000EE211A80ED1F1A90ED201AD0ED3B1A14
:10B4A00001EE801AD0ED231A90ED3E2A42EE001AEA
:10B4B00000EE211A80ED201A90ED271AD0ED421AE5
:10B4C00001EE801AD0ED2A1A90ED452A42EE001ABC
:10B4D00000EE211A80ED271A90ED281AD0ED431ABC
:10B4E00001EE801AD0ED2B1A90ED462A42EE001A9A
:10B4F00000EE211A80ED281A90ED291AD0ED441A99
:10B5000001EE801AD0ED2C1A90ED472A42EE001A77
:10B5100000EE211A80ED291A90ED301AD0ED4B1A69
:10B5200001EE801AD0ED331A90ED4E2A42EE001A49
:10B5300000EE211A80ED301A90ED311AD0ED4C1A40
:10B5400001EE801AD0ED341A90ED4F2A42EE001A27
:10B5500000EE211A80ED311A90ED321AD0ED4D1A1D
:10B5600001EE801AD0ED351A90ED502A42EE001A05
:10B5700000EE211A80ED321A90ED211AD0ED3C1A1E
:10B5800001EE801AD1ED021A61EE801A90ED1C2AAC
:10B5900001EE821AD1ED011A61EE801A90ED1D2A9A
:10B5A00001EEC21A80ED211A90ED221AD0ED3D1A5B
:10B5B00001EE801AD1ED021A61EE801A90ED1B2A7D
:10B5C00001EEC21AD1ED001A61EE801A90ED1D2A2B
:10B5D00001EE821A80ED221A90ED231AD0ED3E1A68
:10B5E00001EE801AD1ED011A61EE801A90ED1B2A4E
:10B5F00001EE821AD1ED001A61EE801A90ED1C2A3C
:10B6000001EEC21A80ED231A90ED2A1AD0ED451AE8
:10B6100001EE801AD1ED021A61EE801A90ED252A12
:10B6200001EE821AD1ED011A61EE801A90ED262A00
:10B6300001EEC21A80ED2A1A90ED2B1AD0ED461AAF
:10B6400001EE801AD1ED021A61EE801A90ED242AE3
:10B6500001EEC21AD1ED001A61EE801A90ED262A91
:10B6600001EE821A80ED2B1A90ED2C1AD0ED471ABC
:10B6700001EE801AD1ED011A61EE801A90ED242AB4
:10B6800001EE821AD1ED001A61EE801A90ED252AA2
:10B6900001EEC21A80ED2C1A90ED331AD0ED4E1A3D
:10B6A00001EE801AD1ED021A61EE801A90ED2E2A79
:10B6B00001EE821AD1ED011A61EE801A90ED2F2A67
:10B6C00001EEC21A80ED331A90ED341AD0ED4F1A04
:10B6D00001EE801AD1ED021A61EE801A90ED2D2A4A
:10B6E00001EEC21AD1ED001A61EE801A90ED2F2AF8
:10B6F00001EE821A80ED341A90ED351AD0ED501A11
:10B7000001EE801AD1ED011A61EE801A90ED2D2A1A
:10B7100001EE821AD1ED001A61EE801A90ED2E2A08
:10B7200001EEC21A80ED351A90ED091AD1ED021A18
:10B7300061EE211A90ED361A01EE801AD0ED121A40
:10B7400091ED012A61EE821A01EEC01A80ED361ADF
:10B7500090ED0A1AD1ED021A61EE211A90ED371A16
:10B7600001EE801AD0ED131A91ED012A61EE821AD2
:10B7700001EEC01A80ED371A90ED0B1AD1ED021AC6
:10B7800061EE211A90ED381A01EE801AD0ED141AEC
:10B7900091ED012A61EE821A01EEC01A80ED381A8D
:10B7A00090ED001AD1ED021A61EE211A90ED3F1AC8
:10B7B00001EEC01AD0ED121A91ED002A61EE821A44
:10B7C00001EE801A80ED3F1A90ED011AD1ED021AB8
:10B7D00061EE211A90ED401A01EEC01AD0ED131A55
:10B7E00091ED002A61EE821A01EE801A80ED401A76
:10B7F00090ED021AD1ED021A61EE211A90ED411A74
:10B8000001EEC01AD0ED141A91ED002A61EE821AF1
:10B8100001EE801A80ED411A90ED001AD1ED011A67
:10B8200061EE211A90ED481A01EE801AD0ED091A46
:10B8300091ED002A61EE821A01EEC01A80ED481ADD
:10B8400090ED011AD1ED011A61EE211A90ED491A1D
:10B8500001EE801AD0ED0A1A91ED002A61EE821AEB
:10B8600001EEC01A80ED491A90ED021AD1ED011ACD
:10B8700061EE211A90ED4A1A01EE801AD0ED0B1AF2
:10B8800091ED002A61EE821A01EEC01A80ED4A1A8B
:10B8900090ED391AD0ED3C1A00EE211AD0ED0C1AB9
:10B8A00091ED022A61EE821A01EE801AD0ED151A8E
:10B8B00091ED012A61EE821A01EEC01A80ED391A6B
:10B8C00090ED3A1AD0ED3D1A00EE211AD0ED0D1A86
:10B8D00091ED022A61EE821A01EE801AD0ED161A5D
:10B8E00091ED012A61EE821A01EEC01A80ED3A1A3A
:10B8F00090ED3B1AD0ED3E1A00EE211AD0ED0E1A53
:10B9000091ED022A61EE821A01EE801AD0ED171A2B
:10B9100091ED012A61EE821A01EEC01A80ED3B1A08
:10B9200090ED421AD0ED451A00EE211AD0ED031A1F
:10B9300091ED022A61EE821A01EEC01AD0ED151ABD
:10B9400091ED002A61EE821A01EE801A80ED421A12
:10B9500090ED431AD0ED461A00EE211AD0ED041AEC
:10B9600091ED022A61EE821A01EEC01AD0ED161A8C
:10B9700091ED002A61EE821A01EE801A80ED431AE1
:10B9800090ED441AD0ED471A00EE211AD0ED051AB9
:10B9900091ED022A61EE821A01EEC01AD0ED171A5B
:10B9A00091ED002A61EE821A01EE801A80ED441AB0
:10B9B00090ED4B1AD0ED4E1A00EE211AD0ED031A7D
:10B9C00091ED012A61EE821A01EE801AD0ED0C1A77
:10B9D00091ED002A61EE821A01EEC01A80ED4B1A39
:10B9E00090ED4C1AD0ED4F1A00EE211AD0ED041A4A
:10B9F00091ED012A61EE821A01EE801AD0ED0D1A46
:10BA000091ED002A61EE821A01EEC01A80ED4C1A07
:10BA100090ED4D1AD0ED501A00EE211AD0ED051A16
:10BA200091ED012A61EE821A01EE801AD0ED0E1A14
:10BA300091ED002A61EE821A01EEC01A80ED4D1AD6
:10BA400090ED0F1AD1ED021A61EE211A90ED3C1A19
:10BA500001EE801AD0ED181A91ED012A61EE821ADA
:10BA600001EEC01AD1ED021A61EE801A90ED372A6C
:10BA700001EE821AD1ED011A61EE801A90ED382A9A
:10BA800001EEC21A80ED3C1A90ED101AD1ED021AA7
:10BA900061EE211A90ED3D1A01EE801AD0ED191ACF
:10BAA00091ED012A61EE821A01EEC01AD1ED021A5F
:10BAB00061EE801A90ED362A01EEC21AD1ED001A1D
:10BAC00061EE801A90ED382A01EE821A80ED3D1A5F
:10BAD00090ED111AD1ED021A61EE211A90ED3E1A85
:10BAE00001EE801AD0ED1A1A91ED012A61EE821A48
:10BAF00001EEC01AD1ED011A61EE801A90ED362ADE
:10BB000001EE821AD1ED001A61EE801A90ED372A0B
:10BB100001EEC21A80ED3E1A90ED061AD1ED021A1E
:10BB200061EE211A90ED451A01EEC01AD0ED181AF7
:10BB300091ED002A61EE821A01EE801AD1ED021A0F
:10BB400061EE801A90ED402A01EE821AD1ED011AC1
:10BB500061EE801A90ED412A01EEC21A80ED451A7D
:10BB600090ED071AD1ED021A61EE211A90ED461AF6
:10BB700001EEC01AD0ED191A91ED002A61EE821A79
:10BB800001EE801AD1ED021A61EE801A90ED3F2A83
:10BB900001EEC21AD1ED001A61EE801A90ED412A31
:10BBA00001EE821A80ED461A90ED081AD1ED021AC4
:10BBB00061EE211A90ED471A01EEC01AD0ED1A1A63
:10BBC00091ED002A61EE821A01EE801AD1ED011A80
:10BBD00061EE801A90ED3F2A01EE821AD1ED001A33
:10BBE00061EE801A90ED402A01EEC21A80ED471AEC
:10BBF00090ED061AD1ED011A61EE211A90ED4E1A60
:10BC000001EE801AD0ED0F1A91ED002A61EE821A32
:10BC100001EEC01AD1ED021A61EE801A90ED492AA8
:10BC200001EE821AD1ED011A61EE801A90ED4A2AD6
:10BC300001EEC21A80ED4E1A90ED071AD1ED011AED
:10BC400061EE211A90ED4F1A01EE801AD0ED101A14
:10BC500091ED002A61EE821A01EEC01AD1ED021AAE
:10BC600061EE801A90ED482A01EEC21AD1ED001A59
:10BC700061EE801A90ED4A2A01EE821A80ED4F1A89
:10BC800090ED081AD1ED011A61EE211A90ED501ACB
:10BC900001EE801AD0ED111A91ED002A61EE821AA0
:10BCA00001EEC01AD1ED011A61EE801A90ED482A1A
:10BCB00001EE821AD1ED001A61EE801A90ED492A48
:10BCC00001EEC21A80ED501A90ED011AD1ED021A60
:10BCD00061EE211A90ED061A01EE801AD0ED021ADB
:10BCE00091ED012A61EE821A01EEC01A80ED061A6A
:10BCF00090ED001AD1ED021A61EE211A90ED071AAB
:10BD000001EEC01AD0ED021A91ED002A61EE821AFE
:10BD100001EE801A80ED071A90ED001AD1ED011A9C
:10BD200061EE211A90ED081A01EE801AD0ED011A89
:10BD300091ED002A61EE821A01EEC01A80ED081A18
:10BD400090ED0A1AD1ED021A61EE211A90ED0F1A48
:10BD500001EE801AD0ED0B1A91ED012A61EE821AE4
:10BD600001EEC01A80ED0F1A90ED091AD1ED021AFA
:10BD700061EE211A90ED101A01EEC01AD0ED0B1AE7
:10BD800091ED002A61EE821A01EE801A80ED101A00
:10BD900090ED091AD1ED011A61EE211A90ED111AF8
:10BDA00001EE801AD0ED0A1A91ED002A61EE821A96
:10BDB00001EEC01A80ED111A90ED131AD1ED021A9E
:10BDC00061EE211A90ED181A01EE801AD0ED141AC6
:10BDD00091ED012A61EE821A01EEC01A80ED181A67
:10BDE00090ED121AD1ED021A61EE211A90ED191A96
:10BDF00001EEC01AD0ED141A91ED002A61EE821AFC
:10BE000001EE801A80ED191A90ED121AD1ED011A87
:10BE100061EE211A90ED1A1A01EE801AD0ED131A74
:10BE200091ED002A61EE821A01EEC01A80ED1A1A15
:10BE30009FED191A20EE011A61EE000A002210E0AF
:10BE400002EBC203134400EB830393ED001A31EEBF
:10BE5000201A02EBC203134400EB830383ED001AA4
:10BE6000521C032AECDB062212E002EBC20313444D
:10BE700000EB830393ED001ADFED081A00EEA11A20
:10BE800002EBC203134400EB830383ED001A521C40
:10BE9000092AEADB7047000017B7D1380000C84212
:10BEA00001480249086070470090D003304B0020E1
:10BEB00010B514F0DDFA28B195480088C0F30420CD
:10BEC0009449086014F02CFB10B1934893494867DB
:10BED00014F062FB30B18E48E0380068C0F34230A5
:10BEE0008F49086014F084FB28B18E48006820F068
:10BEF00080708C49086014F099FB48B100208A4991
:10BF000008604FF08041C1F810018549091F0860A1
:10BF100014F0B8FB18B1032081496431086014F0B3
:10BF2000CFFB68B105208149086001207F49783145
:10BF3000086000207D49083108603F20091F086023
:10BF400014F0DCFB002855D07148E03000687849D7
:10BF500008606F48E4300068091D08606C48E830EC
:10BF60000068091D08606A48EC300068091D086017
:10BF70006748F0300068091D08606548F4300068C3
:10BF8000091D08606248F83000686949203108607E
:10BF90005F48FC300068091D086066480068091D9C
:10BFA00008606448001D0068091D08606148083089
:10BFB0000068091D08605F480C300068091D0860B2
:10BFC0005C48103000685A494031086059481430C4
:10BFD0000068091D0860574818300068091D08608E
:10BFE00054481C300068091D086052482030006821
:10BFF000091D086014F010FA30B14548CC380068CB
:10C0000000F04F004C49086014F05EFA40B14B4814
:10C01000006800F0010018B16FF0010047490860A6
:10C0200014F09CFA28B14648006840F48060444906
:10C0300008603C487438006840F47000394974392D
:10C04000086000BF00BF00BFBFF34F8F00BF00BF3D
:10C0500000BF00BF00BF00BFBFF36F8F00BF00BFB6
:10C0600000BF3848006800F00100F0B101203649F7
:10C07000086000BF354800680028FBD031480068E0
:10C0800020F001004FF01021C1F80C0200BF2F4832
:10C0900000680028FBD000202B49086000BF2B4817
:10C0A00000680028FBD001F03BF826480C380068F7
:10C0B00000F0004028B923480838006800F000402C
:10C0C00018B301202049086000BF204800680028FC
:10C0D000FBD015201B490C39086000BF1B480068C5
:10C0E0000028FBD0152117480838016000BF174809
:10C0F00000680028FBD000201349086000BF1348E7
:10C1000000680028FBD001F00BF8FFF7C9FE10BD56
:10C1100024030010403501400DF0ADBA00C00740C7
:10C120003C050040FCED00E00C01004010560040D2
:10C1300020C5004024040010E40E0040000400402C
:10C140003C1700400C12001004E5014000E40140DF
:10C150000148006870470000904000207CB5002531
:10C160001B4903C9CDE9000102208DF8020000201F
:10C17000ADF80000174A6946174816F079FC0446E6
:10C1800004B16D1E012321220021134816F0FCFB8F
:10C19000044664B10123212200210F4816F0F4FB6C
:10C1A000044624B10D4A0EA10020FEF747F80A48C4
:10C1B00016F042FC084816F04BFC0F4800F086FDD4
:10C1C000681C20B90D4A0EA10020FEF737F87CBD8F
:10C1D000B0A304006D6E0400A8A30400494003004E
:10C1E0006273705F7274635F636F6E6669675F70BE
:10C1F000726F636573730000695503007940030033
:10C200006273705F7274635F696E69745F70726F7E
:10C2100063657373000000000246002112E00C48C1
:10C2200050F82100904202D16FF001007047084899
:10C2300050F8210020B9064840F821200020F5E7F9
:10C24000481CC1B20A29EADB4FF0FF30EEE70000DC
:10C25000E47B00207047000030B589B0054600241B
:10C26000002009E0C0F1050219498B5C2146621CDF
:10C27000D4B201AA5354401C0628F3DB0022204606
:10C28000611CCCB201A90A5401222046611CCCB227
:10C2900001A90A542046611CCCB201A90A542046C7
:10C2A000611CCCB201A90A5400222046611CCCB208
:10C2B00001A90A542A222046611CCCB201A90A54C1
:10C2C000234601AA2946002000F0C6F909B030BD76
:10C2D0007D3F0020F0B504460D461646244825490A
:10C2E000086004202449C1F804032448046023485A
:10C2F00008300560224804602248056030460FF08F
:10C300006DF91E49183108601C480C38006840F06F
:10C3100004001A490C3908604FF0FF301649886054
:10C32000086002200321002804DB4A07130E164A86
:10C33000135406E04A07170E144A00F00F031B1FA0
:10C34000D75400BF022000280DDB00BF00BF00F063
:10C350001F02012191404209920002F1E022C2F83D
:10C36000001100BF00BF00BF002009490860F0BDF8
:10C370000302020008230040002000400C2500407A
:10C38000104000201440002000E400E018ED00E020
:10C390001C21004070B504460D461646324629461B
:10C3A0002046FFF797FF054A05A10020FDF746FF4D
:10C3B000064A07A10020FDF741FF70BDDDC3020062
:10C3C00055415254305F527800000000F9C5020018
:10C3D00055415254305F54780000000070B565E05C
:10C3E0003348007810B101285BD12BE0FBF752FBFA
:10C3F000032800D270BD0020FBF71CFBAA2803D045
:10C400000120FBF79FFB1CE00220FBF713FB044617
:10C41000E043C4B20120FBF70DFB26490870084633
:10C420000078844209D108460078052805DB2048B9
:10C430000078401C1E49087002E00120FBF782FBD7
:10C4400000BF32E0FBF726FB1A490978884200D288
:10C45000D0E70025002406E02046FBF7EBFA28444D
:10C46000C5B2601CC4B213480078401EA042F3DC81
:10C4700010490978491E88B2FBF7DCFAA84208D1B6
:10C480000C480078FDF7FAFF0A480078FBF75AFBE2
:10C4900002E00120FBF756FB00200549087000BFB1
:10C4A00003E000200249087000BF00BF98E70000C9
:10C4B000284000202940002010B50246104800689E
:10C4C000092802D34FF0FF3010BD0E480C4B1B68FB
:10C4D00000EB0310C1600B48094B1B6800EB031015
:10C4E00002700948074B064C246803EB041358609C
:10C4F00003480068401C024B18600020E4E700007D
:10C500002040002060620020F06200202DE9F0430E
:10C51000C0B007468846164600240023701D00F070
:10C52000FF09AA200DF8030019465B1C1DF8010045
:10C530002044C4B20DF8039019465B1C1DF801009D
:10C540002044C4B26FEA0900C0B20DF803001946D6
:10C550005B1C1DF801002044C4B20DF8037019469D
:10C560005B1C1DF801002044C4B200250CE018F843
:10C5700005000DF803001846591CCBB21DF8000049
:10C580002044C4B2681CC5B2B542F0DB1846591C41
:10C59000CBB20DF80040002505E01DF8050000F0C5
:10C5A00007F8681CC5B29D42F7DB40B0BDE8F083D8
:10C5B0000549086000BF054909680029FBD0002132
:10C5C000024A1160704700001C2500401C210040F9
:10C5D00008490AE00A68824204D100234376136ABC
:10C5E0000B6001E002F1200100BF0A68002AF1D1CE
:10C5F000704700002440002070B5002515480468ED
:10C600001FE0E068D0B1E068401EE060E068A8B9D3
:10C61000207A00280ADD207A401E20726068E060DF
:10C62000227E207C6169FFF771FF07E02046FFF75B
:10C63000CFFFE06910B12046E1698847607E05437D
:10C64000246A002CDDD12946AFF25300FDF7D2FD5C
:10C6500070BD0000244000202DE9F04104468846CA
:10C6600015461E4613480768ECB184F810806561D2
:10C6700026766068E0602078002803DD2078401E80
:10C68000207201E0002020720120607604E0A742C1
:10C6900001D1BDE8F0813F6A002FF8D1054800685C
:10C6A000206204480460324629464046FFF72EFFC8
:10C6B00000BFEEE72440002070B505460C46002080
:10C6C0001F4908601F48204908600220002817DB26
:10C6D00000F01F02012191401C4A430942F8231037
:10C6E00000BF00BF00BFBFF34F8F00BF00BF00BF40
:10C6F00000BF00BF00BFBFF36F8F00BF00BF00BF10
:10C7000000BF0220002807DB00F01F02012191403A
:10C710000F4A430942F8231000BF284615F008F8D5
:10C72000204615F005F816200A4908600A490860F5
:10C730000A48FDF7D5FD0A48FDF7D2FD70BD00009F
:10C7400000250040840202000823004080E100E050
:10C7500080E200E01040002014400020DDC3020011
:10C76000F9C502002049086820490968B9B10022CA
:10C770001E4B1A601E4A1268D1B21B4A1268501C26
:10C780001C4A904201D3A2F580601B4A1268904275
:10C7900004D0154A12681170134A106000BF134983
:10C7A0003C31096819B10021104A3C3211600F492F
:10C7B0000839096819B100210C4A083A11600B497F
:10C7C000091F096819B10021084A121F11600749A1
:10C7D000143109680949D1F8241119B10021034A1B
:10C7E0001C321160704700001840002008210040F2
:10C7F00018250040606200201C40002000200040FE
:10C8000010B5FFF7ABFC07F025F8FAF72FFB0FF098
:10C8100035FAFAF73BFCFAF7F7FD0FF0CFFA0FF015
:10C820004BFA03F0C9F804F0F9F904F0F1FD02F055
:10C830000DFE05F037F903F0EFFE04F0D1FA04F035
:10C84000D1FB03F0C3FD05F0BBFA03F00BFE05F0CE
:10C8500033F804F0F1F904F0FBFDFFF7FBFC10BD29
:10C8600010B5FDF775FC78B9FEF7E8FC0FF02CFD6C
:10C8700004461AF047FA0749086008460068064966
:10C88000086000F009FA02E0002003490860FBF7A5
:10C89000E5FB10BDD03D0020D83D002010B588B08C
:10C8A00000200490059006900790304800790028F9
:10C8B0002BD02E4890F82800432855D12B4890F8CB
:10C8C000371090F8362090F83500284BDB79CDE909
:10C8D0000030CDE9022125488379427924A104A8BA
:10C8E00000F0D2FB04A8F9F7EFFD044604AB2246A2
:10C8F00026A10020FEF7E0F904A8F9F7E5FD0446BB
:10C90000214604A80FF062FD2EE0184890F8280098
:10C91000432829D1154890F8371090F8362090F820
:10C920003500124BDB79CDE90030CDE902210F480B
:10C93000837942790EA104A800F0A6FB04A8F9F7B8
:10C94000C3FD044604AB224615A10020FEF7B4F94E
:10C9500004A8F9F7B9FD0446214604A81BF04CFFD2
:10C960000C2113A00FF032FD08B010BD945100202F
:10C97000253032582530325825303258253032583B
:10C980002530325825303258000000007363616E44
:10C990004E616D65282564293A25730A0000000060
:10C9A0006164764E616D65282564293A25730A0015
:10C9B000313233323133323133313200B0EE401A5A
:10C9C00081EE200ADFED021A20EE210A70470000F6
:10C9D0000000C84210B52DED048BB0EE408A9FEDEB
:10C9E000260AB0EE409A9FED240AF0EE408A2348D2
:10C9F000006890F8230060B1B2EE040AC8EE000AA5
:10CA00001E480068C0ED000A00201C49096881F832
:10CA10002300B2EE040AC8EE000AF0EE609A17484E
:10CA20000068DFED170AB0EE690A0CF04CFEF0EE7C
:10CA3000408A9FED140AF4EEC08AF1EE10FA04D297
:10CA40009FED0D0AB0EE409A11E09FED0F0AF4EE53
:10CA5000C08AF1EE10FA04DD9FED0C0AB0EE409AA8
:10CA600005E0B0EE680A10F0F9FBB0EE409AB0EEC7
:10CA7000490ABDEC048B10BD0000000044400020BA
:10CA80000AD7233C0000A0430000D2430000C84264
:10CA900008B500BF4FF480700B49405808B1012021
:10CAA00000E0002078B109480068804700BF0020FE
:10CAB0004FF48071044A885008461146405800904F
:10CAC00000BF00BF00BF08BD00000140AC4A00200D
:10CAD0002DE9F0410246C2F30744C2F30726D5B25E
:10CAE000802300200021CCE0880006EA0307D7B1AC
:10CAF000664F3F88DFF898C12CF81070634FB7F885
:10CB000002C0DFF88C81471C28F817C05F4FB7F8C8
:10CB100004C0871C28F817C05C4FB7F806C0C71CB4
:10CB200028F817C019E05B4F3F88DFF864C12CF884
:10CB30001070584FB7F802C0DFF85481471C28F82E
:10CB400017C0544FB7F804C0871C28F817C0514FBE
:10CB5000B7F806C0C71C28F817C0880004EA030706
:10CB600017B34A4FB7F800C0494F403727F810C0F5
:10CB7000464FB7F80280464F403700F1010C27F8C6
:10CB80001C80424FB7F80480414F403700F1020C3F
:10CB900027F81C803D4FB7F806803D4F403700F125
:10CBA000030C27F81C8021E03A4FB7F800C0384F3B
:10CBB000403727F810C0374FB7F80280344F40375E
:10CBC00000F1010C27F81C80324FB7F80480304F79
:10CBD000403700F1020C27F81C802E4FB7F8068072
:10CBE0002B4F403700F1030C27F81C80880005EA22
:10CBF000030717B3254FB7F800C0254F803727F834
:10CC000010C0224FB7F80280214F803700F1010C8D
:10CC100027F81C801D4FB7F804801D4F803700F1A6
:10CC2000020C27F81C80194FB7F80680184F803780
:10CC300000F1030C27F81C8021E0164FB7F800C064
:10CC4000134F803727F810C0124FB7F80280104FEB
:10CC5000803700F1010C27F81C800E4FB7F80480D4
:10CC60000B4F803700F1020C27F81C80094FB7F8F2
:10CC70000680074F803700F1030C27F81C805B0803
:10CC8000491C0829FFF630AFBDE8F08198A30400E5
:10CC90004C740020A0A3040010B500240BE0084849
:10CCA00050F8240028B1064850F8241005480068C0
:10CCB0008847601CC4B2044800788442EFDB10BD92
:10CCC000604B0020D03D0020D53D002002460021D1
:10CCD00017E00E4850F82100904202D14FF0FF308B
:10CCE00070470A4850F8210048B909480078401CAC
:10CCF000074B1870054840F821200020F0E7481C39
:10CD0000C1B20629E5DB6FF00100E9E7604B0020C6
:10CD1000D53D002010B50CF0AFFC10BD10B5124C85
:10CD200002202061606111A0A0611349E1614FF40C
:10CD3000007121620021A1626162E1620BA0A06426
:10CD40000E49E164102121650021A1656165E1655D
:10CD50000BA1E01DF9F7DAFB0AA12046F9F7D6FB93
:10CD60002020A07110BD0000E09C00205465726D71
:10CD7000696E616C00000000589D0020589F0020E3
:10CD800052545400534547474552000010B50146E0
:10CD90000A69CB689A4204D88C68641EE41AA01809
:10CDA00001E0D41A601E10BD2DE9FC5F06460F4657
:10CDB00092469846DDE90C45002F01DA784200E002
:10CDC000384683464FF0010903E09BFBFAFB09F16B
:10CDD0000109D345F9DAC84500D9C14634B1002F5D
:10CDE00003DB05F00400042800D1641E05F00200F6
:10CDF00010B1B8F1000F11D005F0010070B96CB19D
:10CE000008E0641E2021304600F0BAF8F0680028DF
:10CE100000DA02E00CB1A145F3D300BFF0680028AE
:10CE200036DB002F05DA7F422D21304600F0A8F8CE
:10CE300007E005F00400042803D12B21304600F060
:10CE40009FF8F068002823DB05F00200022814D1C7
:10CE500005F0010088B9B8F1000F0ED16CB108E0FF
:10CE6000641E3021304600F08BF8F068002800DAAC
:10CE700002E00CB1A145F3D300BFF068002807DB46
:10CE80004346524639463046CDE9004500F002F8A7
:10CE9000BDE8FC9F2DE9FC5F8046894615461E468D
:10CEA0000C9CCDF804900127BB4605E00198B0FB2F
:10CEB000F5F001900BF1010B0198A842F6D25E4506
:10CEC00000D9B3460D9800F00100D0B9CCB10D984F
:10CED00000F00200022803D116B93020009001E0D2
:10CEE0002020009009E0641E4046009900F048F8B8
:10CEF000D8F80C00002800DA02E00CB1A345F2D308
:10CF000000BFD8F80C00002835DB09E0012E01D95C
:10CF1000761E04E0B9FBF7FAAA4500D201E06F43A0
:10CF2000F4E700BF00BFB9FBF7FA0AFB17991348F3
:10CF300010F80A10404600F023F8D8F80C0000283A
:10CF400000DA03E0B7FBF5F7002FECD100BF0D9836
:10CF500000F0010078B174B109E0641E2021404660
:10CF600000F00EF8D8F80C00002800DA02E00CB14E
:10CF7000A345F2D300BFBDE8FC9F000050A8040009
:10CF800070B504460E46A568681C6168814206D3E8
:10CF900020684655681CA060E068401CE060D4E949
:10CFA000011088420DD1A26821682069FDF724FE96
:10CFB000A168884203D04FF0FF30E06001E000201C
:10CFC000A06070BD2DE9F0470446894617464FF032
:10CFD000000AE56800BFD4F81080A84503D9A8EB83
:10CFE0000500461E04E0A5EB0800401CA1680E1ACF
:10CFF00006B90126A068401BB04201D9304601E0C5
:10D00000A068401B0646BE4201D2304600E03846CA
:10D0100006466168481932464946F9F731FAB24482
:10D02000B144BF1B3544A068A84200D10025E5608B
:10D03000002FD0D15046BDE8F0872DE9F0470446D7
:10D0400089461546E668A068871BAF4208D9616823
:10D0500088192A464946F9F713FA7019E06010E07A
:10D06000B8466168881942464946F9F709FAA5EBBE
:10D07000070809EB070142466068F9F701FAC4F8AE
:10D080000C80BDE8F08700000FB4084B10B504A970
:10D0900002AA039801F0A2FA044602A9002001F0B6
:10D0A00034FE204610BC5DF814FB00000BED0200BE
:10D0B00003B401984100009850EAC12018BF042031
:10D0C0004A0D18BF40F0010040F2FF72B2EB515F11
:10D0D00008BF40F00200012808BF052002B07047D9
:10D0E00000BF00BF00BFBFF34F8F00BF00BF00BF36
:10D0F0000948006800F4E06008490843001D06493B
:10D10000086000BF00BF00BFBFF34F8F00BF00BF6C
:10D1100000BF00BF00BFFDE70CED00E00000FA0516
:10D1200000BF00BF00BFBFF34F8F00BF00BF00BFF5
:10D130000948006800F4E06008490843001D0649FA
:10D14000086000BF00BF00BFBFF34F8F00BF00BF2C
:10D1500000BF00BF00BFFDE70CED00E00000FA05D6
:10D1600070B5C1482DED020B2DED0E8B82B0119DD7
:10D1700025F000449FEDBEDB9FEDBFEB84423EDB1C
:10D18000A4F140511098A1F17F6108430FD0BC4831
:10D19000844202DC28D1109830B39DED100B02B010
:10D1A000BDEC0E8B02B0BDE8704001F0E9B89DED1A
:10D1B000100B53EC1D2B51EC100BF9F757FA9DEDAA
:10D1C000100B41EC180B53EC1E2B51EC100BF9F724
:10D1D0004DFA53EC182BF9F7A2F941EC100B02B001
:10D1E000BDEC0E8B02B070BD012001F02FF902B032
:10D1F000BDEC0E8B02B0BDE8704001F0D5B8A1487F
:10D200009FEDA18B844256DA9DED100BB4F1795F4E
:10D210000ADA51EC100BFFF74BFF042808BF01F0AE
:10D22000D3F89DED100BDAE753EC102B51EC100BFB
:10D23000F9F71CFA41EC190B95480621B0EE490AA2
:10D24000F0EE690A784400F087FF53EC192B51EC9B
:10D25000100BF9F70BFA41EC1A0B8E48B0EE490AA5
:10D26000F0EE690A0421784400F076FF53EC192BA4
:10D2700051EC100BF9F7FAF953EC182BF9F74FF9B9
:10D2800041EC100B51EC1A0B53EC102BF9F760FA30
:10D29000CDE900019DED000B53EC102B9DED100B23
:10D2A00051EC100BF9F7E2F99DED101B53EC112B2B
:10D2B000F9F735F9D2E09DED100B51EC100B0CF0A5
:10D2C0000BF953EC182BF9F7CEF99FED730BCDE961
:10D2D000000153EC102B9DED000B51EC100BF9F7F6
:10D2E000C5F941EC190B6E480621B0EE490AF0EE83
:10D2F000690A784400F030FF53EC192B51EC100B05
:10D30000F9F7B4F941EC1B0B6648B0EE490AF0EEB0
:10D31000690A0421784400F01FFF53EC192B51ECEB
:10D32000100BF9F7A3F953EC182BF9F7F8F841ECC7
:10D330001C0B51EC190B1CF005F841EC180B5A486A
:10D340009FED5BABA04222DC53EC1C2B51EC1B0B82
:10D35000F9F7FEF9CDE900019DED000B51EC180B3A
:10D3600053EC102BF9F782F953EC182BF9F7D7F897
:10D3700053EC1A2BF9F77AF953EC1D2BF9F770F9E6
:10D3800053EC1E2BF9F76FF941EC100B5FE08DEDBC
:10D39000008B002000909DED000B51EC180B53EC1E
:10D3A000102BF9F7BCF89DED000B41EC1E0B53EC74
:10D3B000102B51EC100BF9F759F953EC192BF9F725
:10D3C00052F953EC1E2BF9F7C3F941EC190B53EC4E
:10D3D0001C2B51EC1B0BF9F7BBF941EC1B0B53EC6D
:10D3E0001A2B51EC190BF9F741F953EC1D2BF9F7F6
:10D3F0003AF941EC190B53EC1A2B51EC180BF9F7D5
:10D4000035F953EC1B2BF9F731F953EC192BF9F7DC
:10D4100027F99DED000B41EC180B53EC1A2B51EC46
:10D42000100BF9F723F99FED249B53EC192BF9F717
:10D430001AF941EC100B51EC180B53EC102BF9F7C7
:10D440000FF953EC192BF9F70EF941EC100B002DE5
:10D450003FF7C5AE51EC100B81F0004141EC100BD1
:10D46000BDE60000000000000000F03F00000000EA
:10D47000075C143326A6913C182D4454FB21F93F38
:10D480000000F07F0000E03F000000000000F03FDF
:10D49000D8D60100E6D60100000000000000E03F01
:10D4A0002AD6010038D601003333EF3F00000000D8
:10D4B0000000000000000040182D4454FB21E93F0B
:10D4C00070B59B482DED020B2DED068B079D25F0C9
:10D4D0000044A04218DC9748844202DC0AD1069836
:10D4E00040B19DED060BBDEC068B02B0BDE870406F
:10D4F00000F046BF002DCCBF9FED8F0B9FED900B32
:10D50000BDEC068B02B070BD8F48A04215DD8F4880
:10D51000A042D8BF4FF0FF3458DD9DED060B51EC13
:10D52000100BFFF7C5FD042808BF00F04DFF9DED6F
:10D53000060BBDEC068B02B070BD9DED060B51ECE9
:10D54000100B0BF0C9FFCDE9060181489FED828BDE
:10D55000A0423CDD8248A0421FDD00249FED82AB4B
:10D560009DED060B53EC1A2B51EC100BF8F7D7FF7F
:10D570009DED060B41EC190B53EC1A2B51EC100BE3
:10D58000F9F774F853EC182BF9F76AF853EC192BE8
:10D59000F9F7DEF8CDE9060149E09DED060B01241F
:10D5A00053EC182B51EC100BF8F7B9FF9DED060B5F
:10D5B00041EC190B53EC182B51EC100BF9F750F808
:10D5C00053EC192BF9F7C4F8CDE906012FE06848B0
:10D5D000A0421FDD02249FED689B9DED060B53ECDE
:10D5E000192B51EC100BF9F741F853EC182BF8F705
:10D5F00096FF9DED060B41EC180B53EC192B51ECEB
:10D60000100BF9F72DF853EC182BF9F7A1F8CDE929
:10D6100006010CE09DED060B032453EC102B9FED4F
:10D62000580B51EC100BF9F793F8CDE906019DED7D
:10D63000060B53EC102B51EC100BF9F717F841ECDB
:10D64000180B53EC182BF9F711F841EC190B4E4855
:10D650000621B0EE490AF0EE690A784400F07CFD3C
:10D6600053EC182B51EC100BF9F700F841EC180BA8
:10D670004648B0EE490AF0EE690A0521784400F008
:10D680006BFD53EC192B51EC100BF8F7EFFF41EC4D
:10D69000100B51EC180B53EC102B002C0EDAF8F792
:10D6A0003EFF9DED061B53EC112BF8F7DFFF9DEDC0
:10D6B000061B53EC112BF8F7D6FF35E0F8F72FFFD8
:10D6C0009DED061B53EC112BF8F7D0FF41EC100B2E
:10D6D0002F48784400EBC40090ED001B51EC100B78
:10D6E00053EC112BF8F7BCFF9DED061B53EC112BEF
:10D6F000F8F7B6FF41EC100B2648784400EBC40065
:10D7000090ED001B51EC100B53EC112BF8F7ABFF15
:10D7100041EC100B002DA2BFBDEC068B02B070BD1A
:10D7200051EC100B81F0004141EC100B01E70000BF
:10D73000000010440000F07F182D4454FB21F93FF5
:10D74000182D4454FB21F9BF0000DC3F0000203EAF
:10D750000000F33F00000000000000000000F03F68
:10D760000000E63F00000000000000000000004054
:10D770000080034000000000000000000000F83FAF
:10D78000000000000000F0BF7AD3010030D3010098
:10D79000BAD2010072D2010070B56B4E2DED040BB0
:10D7A0002DED028B82B0DDF81CC0DDE905235C4263
:10D7B0002CF000411C4341EAD474049D22F0004047
:10D7C000B44205D86C422C4340EAD474B4420BD91D
:10D7D0009DED061B9DED040B02B0BDEC028B04B069
:10D7E000BDE8704000F0D6BDACF14054A4F17F64B8
:10D7F0001C430BD0022404EAAC7444EAD2740543FF
:10D800009FED538B9FED542B07D015E09DED040B3E
:10D8100051EC100B04F0AAFB42E0002C11BF012CCC
:10D820009DED040B02B0BDEC028B04BF04B070BDD3
:10D83000022C38D0032C3BD00B439FED491B9FEDAE
:10D840004A0B0AD0B14218D1B04209D121F080412F
:10D8500020F08040079105900FE0002A15DA10E0D3
:10D86000434B7B44002C08BF93ED000B0DD0012CE3
:10D8700010D0022C17D0032C1AD0B0421DD1002A90
:10D8800003DAB0EE410AF0EE610A02B0BDEC028BA1
:10D8900004B070BD93ED000B51EC100B81F0004112
:10D8A00041EC100BF1E7B0EE480AF0EE680AECE745
:10D8B000B0EE420AF0EE620AE7E7401A00153C2893
:10D8C000C8BF8DED000B19DCBCF1000FBEBF10F11D
:10D8D0003C0F9FED290B8DED000B0FDB9DED060B33
:10D8E00053EC102B9DED040B51EC100BF8F730FFAF
:10D8F0000BF0F2FD04F03AFBCDE90001002C08BF6B
:10D900009DED000BC1D0012C10D0022C9FED1C0B03
:10D9100053EC102B9DED000B51EC100B0DD0F8F7D4
:10D920009FFE53EC182BF8F79BFEB9E7019880F0A7
:10D93000004001909DED000BA7E7F8F791FE53EC36
:10D94000182BF8F790FEABE70000F07F0000000016
:10D95000182D4454FB210940182D4454FB2109C0C3
:10D96000182D4454FB21F9BF182D4454FB21F93FD5
:10D97000D2D1010000000000000000000000000003
:10D98000075C143326A6A13C10B52F499FED2C1B34
:10D990002DED020B84B0059820F000408842D8BFDE
:10D9A0009DED040B2DDD2949884209D1049840B929
:10D9B0004FF0010000F04AFD00F0F6FC06B010BD8B
:10D9C00005DB9DED040B00F0DBFC06B010BD6846E6
:10D9D0009DED040B00F0ECF810F0030004BF9DED8A
:10D9E000021B9DED000B0CD001280ED09DED021BFB
:10D9F0009DED000B022817D0012000F029FC06B095
:10DA000010BD00F0F1FA06B010BD9DED021B9DEDBA
:10DA1000000B012000F01CFC51EC100B81F00041C8
:10DA200006B041EC100B10BD00F0DEFA51EC100B0B
:10DA300081F0004106B041EC100B10BD0000000069
:10DA40000000000000000000FB21E93F0000F07F23
:10DA50002DED020B019820F0004001909DED000B90
:10DA600002B070470000000010B52F499FED2C1B3D
:10DA70002DED020B84B0059820F000408842DCBFF9
:10DA800000209DED040B32DD2849884209D104981D
:10DA900040B94FF0010000F0D9FC00F085FC06B061
:10DAA00010BD05DB9DED040B00F06AFC06B010BD57
:10DAB00068469DED040B00F07BF810F0030011D0D8
:10DAC000012818D09DED021B9DED000B02281AD0F5
:10DAD00000F08AFA51EC100B81F0004106B041ECE5
:10DAE000100B10BD9DED021B9DED000B012000F001
:10DAF000AFFB06B010BD9DED021B9DED000B00F0CD
:10DB000073FA06B010BD012000F0A2FB51EC100B1F
:10DB100081F0004106B041EC100B10BD0000000088
:10DB20000000000000000000FB21E93F0000F07F42
:10DB300000B52DED048BB0EE409AF0EE609A83B004
:10DB400051EC190BF8F7F2FF41EC180B18EE100A24
:10DB500018EE901A8DED008B002818BF01200843A5
:10DB600020F00040C0F17F6000F1E040C00F14D011
:10DB700019EE101A19EE900A8DED009B002918BFBE
:10DB80000121084320F00040C0F17F6000F1E04037
:10DB9000C00F04BF012000F059FCB0EE480A03B0EA
:10DBA000F0EE680ABDEC048B00BD00000000000030
:10DBB0002DE9F14F04462DED020B2DED088B8AB0B7
:10DBC0009FEDE70B80ED020B139EE74826F0004522
:10DBD00085420ADC9DED120B002084ED000B0AB09B
:10DBE000BDEC088B03B0BDE8F08FE0489FEDE0ABE3
:10DBF0009FEDE1BBA84247DDE14F9FEDE39B9FED29
:10DC0000E48B9DED120B53EC1A2B51EC100B002EF4
:10DC10001CDDF8F725FD41EC100BBD4208D053EC9C
:10DC20001B2B51EC100BF8F71BFDC4E900010BE0B6
:10DC300053EC192B51EC100BF8F712FD53EC182B89
:10DC4000F8F70EFDC4E900010120C8E7F8F767FC0A
:10DC500041EC100BBD4208D053EC1B2B51EC100BC8
:10DC6000F8F75DFCC4E900010BE053EC192B51EC13
:10DC7000100BF8F754FC53EC182BF8F750FCC4E9E0
:10DC800000014FF0FF30AAE7C348A84279DB9DEDC1
:10DC9000120B51EC100B0BF01FFC41EC180B9FED1D
:10DCA000C00B53EC102BF8F7E1FC9FEDBF1B53ECBE
:10DCB000112BF8F734FCF8F7EEFD0746F8F7CDFD29
:10DCC00041EC190B53EC1A2BF8F7D0FC53EC182B42
:10DCD000F8F7C9FC41EC180B53EC1B2B51EC190B5A
:10DCE000F8F7C4FCDFF8C8A241EC100B4FEA155856
:10DCF0000125FA4453EC102B51EC180BF8F7B0FC4B
:10DD0000032DC4E900013DD0C1F30A5005EB4511D4
:10DD1000A8EB00001139814234DA0AEB051BB0EEA2
:10DD200048AA9BED000BF0EE68AA53EC102B51ECC7
:10DD3000190BF8F79BFC41EC1B0B51EC1A0B53EC45
:10DD40001B2BF8F78DFC41EC180B51EC1A0B53EC24
:10DD5000182BF8F785FC53EC1B2BF8F781FC9BED97
:10DD6000020B41EC1A0B53EC102B51EC190BF8F78A
:10DD70007DFC53EC1A2BF8F773FC41EC100B6D1C77
:10DD8000B8E70EE0002EA8BF3846BFF628AF94EDE6
:10DD9000000B51EC100B81F00041C4E90001784206
:10DDA0001DE7C6F3130040F4801EC6F30A50A0F22C
:10DDB000F530471100F01F05C5F12000DDF848B02F
:10DDC00008900020069007900520EC467949002D28
:10DDD00007EB0002794408BF51F8221009D051F82E
:10DDE000223001EB8201AB404A68089922FA01F126
:10DDF0001943A1FB0E26A1FB0B131A449A4234BF10
:10DE00000123002303EB06080CEB8003D3E901A6F2
:10DE10000E448E4234BF0121002192448A4411B144
:10DE2000924502D903E0924501D2012100E0002190
:10DE3000C3E901A641444CF82010011EA0F10100E5
:10DE4000C4DC029800F10050850F0298DDE90367F9
:10DE50008000DDF81480F8F700FD41EC1A0B304625
:10DE6000F8F70CFD9FED541B53EC112BF8F7FEFB5C
:10DE700041EC1B0B3846F8F701FD9FED511B53ECAD
:10DE8000112BF8F7F3FB41EC180B4046F8F7F6FCC2
:10DE90009FED4D1B53EC112BF8F7E8FB41EC190BF0
:10DEA00051EC180B53EC192BF8F739FB53EC1B2BE7
:10DEB000F8F735FB53EC1A2BF8F731FBCDE90801E5
:10DEC000002008909DED080B53EC1A2B51EC100B21
:10DED000F8F7C6FB53EC1B2BF8F7C2FB53EC182BDF
:10DEE000F8F7BEFB53EC192BF8F7BDFB9FED381B81
:10DEF00053EC112BF8F7BAFB9FED370B41EC180BE5
:10DF000053EC102B9DED080B51EC100BF8F7AEFB0A
:10DF100053EC182BF8F703FB9FED310B41EC180B7A
:10DF200053EC102B9DED080B51EC100BF8F79EFBFA
:10DF300053EC182BF8F7F3FA41EC100B139810F090
:10DF4000004F06D06D4251EC100B81F0004141ECC6
:10DF5000100B284684ED000B41E600000000000095
:10DF60000000000000000000FB21E93F7CD90240D6
:10DF700000004054FB21F93F3163621A61B4D03D87
:10DF8000FB21F93F000000000000601A61B4D03DA1
:10DF90007370032E8A19A33BFB2139410000000056
:10DFA00083C8C96D305FE43F000000000000E03F1F
:10DFB0004ACD010098CC0100000000000000103E96
:10DFC000000000000000103C000000000000103ABB
:10DFD000182D4454FB21F93D3326A611460B113C64
:10DFE00000000054FB21F93D10B52DED040B2DED83
:10DFF000088B82B0B0EE419AF0EE619A0B9820F057
:10E0000000449FED4BABB4F1795F11DA9DED0A0B43
:10E0100051EC100BF8F73FFC002801BFB0EE4A0AA4
:10E02000F0EE6A0A02B0BDEC088B04BF04B010BD6C
:10E030009DED0A0B53EC102B51EC100BF8F716FB6F
:10E0400041EC180B3C480621B0EE480AF0EE680A95
:10E05000784400F081F853EC182B51EC100BF8F7D2
:10E0600005FB9DED0A0B41EC1B0B53EC192B51ECFE
:10E07000100BF8F7FBFA41EC190B53EC1B2B51EC8E
:10E08000180BF8F7F3FA53EC192BF8F7E9FA9FEDB0
:10E090002C0B41EC190B53EC102B51EC180BF8F72F
:10E0A000E5FA41EC100B2848844210DA53EC192BA6
:10E0B00051EC100BF8F7D4FA53EC1A2BF8F7D3FA0B
:10E0C00041EC100B02B0BDEC088B04B010BD1F4832
:10E0D000A042BCBF9FED1E1B8DED001B06DBA4F50F
:10E0E00000100190002000909DED001B51EC100BE2
:10E0F00053EC112BF8F7B4FA9DED000B41EC180B23
:10E1000053EC102B51EC1A0BF8F7AAFA41EC1A0B4E
:10E1100053EC192B51EC180BF8F7A2FA53EC1A2B0D
:10E12000F8F7A1FA41EC100BCCE70000000000006A
:10E13000000000000000F03FB4C901000000000032
:10E14000000000000000E03F3333D33F0000E93F10
:10E15000000000000000D23F70B504462DED028B98
:10E160004D1E00EBC500B0EE408AF0EE608A90EDE7
:10E17000000B35F0060017D053EC182B51EC100BA8
:10E18000F8F774FA41EC100B6D1E04EBC50090ED2E
:10E19000001B51EC100B53EC112BF8F7C0F941ECBC
:10E1A000100B35F00600E7D1022D36D0042D1CD01F
:10E1B000062D1CBFBDEC028B70BD53EC182B51EC2F
:10E1C000100BF8F753FA94ED0A1B53EC112BF8F7E8
:10E1D000A6F953EC182BF8F749FA94ED081B53EC09
:10E1E000112BF8F79CF941EC100B53EC182B51EC68
:10E1F000100BF8F73BFA94ED061B53EC112BF8F7D4
:10E200008EF953EC182BF8F731FA94ED040B53EC1C
:10E21000102BF8F784F941EC100B53EC182B51EC50
:10E22000100BF8F723FA94ED021B53EC112BF8F7BF
:10E2300076F953EC182BF8F719FA94ED001B53EC10
:10E24000112BF8F76CF9BDEC028B41EC100B70BD93
:10E2500031B504462DED040B2DED0A8BB0EE41BA1D
:10E26000F0EE61BA0B989DED0A0B20F00040B0F182
:10E27000795F0DDA51EC100BFEF71AFF042808BF86
:10E2800000F0A2F89DED0A0BBDEC0A8B05B030BD85
:10E2900053EC102B51EC100BF8F7E8F941EC180B8C
:10E2A0009DED0A0B53EC182B51EC100BF8F7DEF92F
:10E2B00041EC190B2C48B0EE480AF0EE680A052133
:10E2C0007844FFF749FF9FED2ACBB0EE40AAF0EE6D
:10E2D00060AA9CB353EC1C2B51EC190BF8F7C6F950
:10E2E00041EC1C0B53EC1A2B51EC190BF8F7BEF94F
:10E2F0009FED210B41EC190B53EC102B51EC1B0B38
:10E30000F8F7B4F953EC192BF8F7AAF953EC182BDA
:10E31000F8F7ACF953EC1B2BF8F7A2F953EC1C2BD4
:10E32000F8F79EF99DED0A1B53EC112BF8F79BF9BA
:10E33000BDEC0A8B05B041EC100B30BDFFE753EC90
:10E340001A2B51EC180BF8F791F953EC1C2BF8F73A
:10E35000E6F853EC192BF8F789F99DED0A1B53ECFD
:10E36000112BF8F7DCF8E3E744C8010000000000D7
:10E37000495555555555C5BF000000000000E03F08
:10E3800010B553EC102B51EC100BF8F7C8F841EC1A
:10E39000100B10BD10B553EC112B51EC100BF8F70E
:10E3A000BEF841EC100B10BD9FED050B10B553EC02
:10E3B000102B51EC100BF8F7CBF941EC100B10BD02
:10E3C00000000000000000009FED050B10B553ECAD
:10E3D000102B51EC100BF8F749F941EC100B10BD64
:10E3E000000000000000001002E008C8121F08C171
:10E3F000002AFAD170477047002001E001C1121FC6
:10E40000002AFBD1704700000146202908DA0120CC
:10E4100088400A4A104008B1012070470020FCE7FC
:10E42000402909DAA1F12000012202FA00F008B126
:10E430000120F2E70020F0E70120EEE7FC06FFBD37
:10E4400000BFEFF31081084672B6704701490860BB
:10E4500070470000344B00202DE9FF5F82B000219F
:10E46000DDE90430020DDDF840B0034318D044F676
:10E470001050A2F2FF3242431514119801281FD008
:10E48000A5EB0B00401C5FEA000A4FF000064E4F60
:10E49000DFF83891B046504615D5CAF1000413E0B4
:10E4A000119801244AA3012801D16FEA0B010298B7
:10E4B000119AC0E90031C0E9024206B0BDE8F09F00
:10E4C000CBF10000DFE704460021404A491842EB47
:10E4D0000450CDE9001012E0E00707D032463B4679
:10E4E00040464946F8F7C2F88046894632463B46E0
:10E4F00010461946F8F7BAF806460F466410002C85
:10E50000EAD1DDE90401DDE90023BAF1000F06DA02
:10E51000F8F7ACF842464B46F8F7A8F805E0F8F7EC
:10E5200017F942464B46F8F713F904460E46002207
:10E53000284BF8F7FBF903D84FF0FF30014607E00E
:10E540000022254B20463146F7F7E9FFF8F73FFB5D
:10E55000102409E0002C0ADB0A220023F7F750FF01
:10E56000039B30321A55641E50EA0102F2D1641C3A
:10E57000039AC4F111031444119A012A03D0012211
:10E5800008430DD10AE0084304D000204FF0110BDE
:10E59000119072E7A3EB0B056D1E0DE05B4504DDEA
:10E5A0004FF0000205F1010504E003DA4FF000022C
:10E5B000A5F10105002AECD002981199C0E90231B9
:10E5C000C0E9004579E70000000014400000F03F7A
:10E5D000300000000000F0430000E03F2DE9FF4F55
:10E5E00095B09B468946064600250FE2252877D13F
:10E5F00000242746F84A0121059400E0044316F858
:10E60000013F203B01FA03F01042F7D130782A286D
:10E6100011D06FF02F033078A0F13002092A16D8FC
:10E62000059A44F0020402EB820203EB420210441A
:10E63000761C0590EFE759F8042B0592002A03DABF
:10E64000504244F40054059044F00204761C3078A3
:10E650002E2816D116F8010F44F004042A280DD0F4
:10E660006FF02F023078A0F13003092B09D807EBA7
:10E67000870302EB4303C718761CF3E759F8047BC2
:10E68000761C30786C280FD006DC4C2817D0682810
:10E690000DD06A2814D104E0742810D07A280FD144
:10E6A0000DE044F400140AE044F4801401E044F462
:10E6B00040147278824202D104F58014761C761CD4
:10E6C000307866280BD013DC582877D009DC002876
:10E6D00075D04528F6D04628F4D047281AD19DE1B8
:10E6E00018E0632835D0642879D0652812D195E1E7
:10E6F000702873D008DC6728F1D069286FD06E28A5
:10E700000DD06F2806D1B5E073282CD0752875D0B0
:10E71000782874D05A46179990476D1C75E1C4F358
:10E720000250022809D003280DD0D9F8001004287F
:10E730000DD00D6009F1040967E1D9F80010EA175E
:10E74000C1E90052F6E7D9F800100D80F2E70D702C
:10E75000F0E719F8041B8DF8001000208DF8010077
:10E76000EA46012003E059F804AB4FF0FF3061079F
:10E770004FF0000102D40DE008F101018846B942D2
:10E780000FDA8045F8DB1AF808100029F4D108E008
:10E7900008F1010188468142FADB1AF808100029C5
:10E7A000F6D105985B46A0EB080721463846179A34
:10E7B00000F094FA284400EB080507E04DE029E159
:10E7C0000DE01AF8010B5A4617999047B8F1010865
:10E7D000F7D25B4621463846179A13E142E00A22F7
:10E7E0000092C4F302524FF0000A022A08D059F8EE
:10E7F00004CB032A4FEAEC710AD00DE029E02AE0AD
:10E8000009F1070121F00702F2E802C1914609E08F
:10E810000FFA8CFC4FEAEC71042A03D14FFA8CFCFE
:10E820004FEAEC71002907DA0A460021DCF1000CFE
:10E8300061EB02012D2202E0220504D52B228DF886
:10E840000420012203E0E20701D02022F7E79046EE
:10E8500059E00A2102E010220DE010214FF0000AD9
:10E8600000910BE010224FF0000A44F00404082746
:10E87000009203E008224FF0000A0092C4F3025213
:10E88000022A05D059F804CB0021032A08D009E058
:10E8900009F1070121F00702F2E802C1914605E003
:10E8A0001FFA8CFC042A01D10CF0FF0C4FF0000879
:10E8B000220728D5702806D0009B83F0100353EA66
:10E8C0000A0305D00EE040228DF80420012208E062
:10E8D0005CEA010206D030228DF804208DF8050094
:10E8E00002229046009B83F0080353EA0A030AD1F0
:10E8F0005CEA010201D1620705D530228DF80420BF
:10E900004FF001087F1E582804D034A003900EA8B1
:10E9100002900DE036A0F9E753466046009AF7F7FB
:10E920006FFD84460398825C0298401E029002703C
:10E930005CEA0100F0D1029806A9081A00F1200A49
:10E94000600702D524F4803400E00127574502DD3A
:10E95000A7EB0A0000E0002000EB0A0100900598F8
:10E960004144401A0590E00306D45B462146179ABD
:10E97000059800F0B3F90544002706E001A85A46BF
:10E98000C05D179990476D1C7F1C4745F6DBE0037F
:10E990000CD55B462146179A059800F09FF905446F
:10E9A00004E030205A46179990476D1C0099481E84
:10E9B00000900029F5DC08E0029802995A46007898
:10E9C000491C0291179990476D1CBAF10001AAF1F8
:10E9D000010AF1DC65E10000092801003031323321
:10E9E000343536373839616263646566000000008B
:10E9F0003031323334353637383941424344454675
:10EA00000000000000F058F90544761C307800281A
:10EA10007FF4ECAD19B02846BDE8F08F620700D452
:10EA2000062709F1070222F0070CFCE80223E14661
:10EA300003F000485FEA080C02D00FF2702C0DE0E2
:10EA40005FEA045C02D50FF2682C07E05FEAC47C41
:10EA500002D00FF2602C01E0AFF2700C4FF0FF38E3
:10EA600023F00043CDF850C065280CD006DC4528C3
:10EA700009D046281DD047283DD13DE0662818D052
:10EA800067287ED138E00021112F01DB112000E042
:10EA9000781CCDE9000106A90EA8FFF7DDFCDDE931
:10EAA0000F010E9A03910021009207F1010A0491CF
:10EAB0004DE04FF000400097CDE9011006A90EA8E7
:10EAC000FFF7CAFCDDE90F0203920E9B11990022A9
:10EAD000DDF80CA00093049211B9791C00EB010A37
:10EAE000B7EB0A0004D4C0F1FF3007F1010A04902B
:10EAF000AAEB0700019044E0012F00DA0127002172
:10EB0000112F01DD112000E03846CDE9000106A9F2
:10EB10000EA8FFF7A1FCDDE90F010E9A0391002179
:10EB200004910092BA4621070CD40399514500DAAA
:10EB30008A46BAF1010F05DD009AAAF10101515C84
:10EB4000302908D0B84202DA10F1040F06DA0121A8
:10EB5000CDE9011015E0AAF10101E9E7002805DC83
:10EB6000049901440491AAEB000102E0411C5145C3
:10EB700000DD8A460499401A401C01904FF0004085
:10EB80000290200704D40198504501DBCDF80480A1
:10EB900000208DF84F0002980DF14F07B0F1004FA3
:10EBA00025D02B200E9002984FF0020800280CDA96
:10EBB000404202902D200E9007E00A210298F7F7BC
:10EBC000E9FE3031029007F8011DB8F10001A8F10B
:10EBD0000108F2DC02980028EFD1791E0E98087027
:10EBE000307800F0200040F0450007F8020D12A830
:10EBF000C01B00F107081498007800B1012000EB59
:10EC00000A01019801EBE07105984144401A401E49
:10EC10000590E00306D45B462146179A059800F05C
:10EC20005DF805441498007818B15A461799904732
:10EC30006D1CE00324D55B462146179A059800F029
:10EC40004DF805441CE00498002807DBDDE90301CA
:10EC5000884203DD0098405C179901E01799302045
:10EC60005A469047049805F10105401C049001980C
:10EC7000401E019004D12E205A46179990476D1CD2
:10EC8000BAF10001AAF1010ADDDC05E017F8010B79
:10EC90005A46179990476D1CB8F10001A8F1010878
:10ECA000F4DC5B462146179A0598ABE62D00000080
:10ECB0002B000000200000002DE9F0410446002553
:10ECC0001E461746880404D405E039462020B04784
:10ECD0006D1C641EF9D52846BDE8F0812DE9F04190
:10ECE000044600251E469046C80301D5302700E0A3
:10ECF0002027880404D505E041463846B0476D1CFE
:10ED0000641EF9D52846BDE8F0810A68531C0B60E3
:10ED10001070704770B50446207850B9054A1288C3
:10ED200091B2606813F00CFF054615B90120024945
:10ED3000087070BDF4400020F040002070B505461A
:10ED40000C4605B10CB9002070BD28784008217828
:10ED5000B0EB510F01D00020F6E70622611C681CC1
:10ED6000F7F7C7FB08B90120EEE70020ECE7014602
:10ED700001F0030008B9012070470020FCE70246BB
:10ED800050680068401E084008B901207047002004
:10ED9000FCE70246002104E0505C08B10120704706
:10EDA000491C0629F8D30020F9E710B50346D868B6
:10EDB000884206D88818401E1C69A04201D801204C
:10EDC00010BD0020FCE7000010B504466CB10848F7
:10EDD000C068A04209D806480069A04205D3204671
:10EDE0000FF067F808B1012010BD0020FCE700001B
:10EDF000384B002070B504460D4604F22740FFF75B
:10EE0000C8FF0646012D06D0022D0DD0032D11D0CE
:10EE1000042D19D113E0A07928B194F8240010B979
:10EE20000EB1012070BD00BFE07910B10EB102201B
:10EE3000F8E700BF207A08B10320F3E700BF607A4B
:10EE400008B10420EEE700BF0020EBE70146481CB4
:10EE5000052290FBF2F302FB1300C0B270472DE9CC
:10EE6000F04704460D462F4695F82080B4F81C90D4
:10EE700000260BE007EB46124946A06903F0AAFB07
:10EE800010B10120BDE8F087701CC6B24645F1DB29
:10EE90000020F7E7014691F82420012A01D1EE2055
:10EEA00000E01F20704770B504460D4616463246F6
:10EEB0002946204603F08EFB70BD000008B10149D1
:10EEC00008607047C847002030B5ADB004200190FD
:10EED000AC2102A8F7F7EDFA02208DF80800002017
:10EEE0008DF80A0005208DF80B0001A80390012180
:10EEF000ADF854101149169101218DF884104FF48A
:10EF0000A071249144F2506125910D482B9002A9E3
:10EF10000C4803F0CBFB044600BF254635B100BFCB
:10EF200009A27B212846F7F775F900BF00BF012130
:10EF3000044803F0B8FB2DB030BD0000484100206C
:10EF4000C9340400C47D00202E2E5C2E2E5C2E2E93
:10EF50005C626C655F6366675C736C6176652E638B
:10EF60000000000070B50321074803F041FC04468F
:10EF700000BF254635B100BF04A29A212846F7F705
:10EF800049F900BF00BF70BDC47D00202E2E5C2E4D
:10EF90002E5C2E2E5C626C655F6366675C736C61D1
:10EFA00076652E630000000070B5084991F85400A2
:10EFB00074DF044600BF254635B100BF04A2A0217E
:10EFC0002846F7F727F900BF00BF70BDC47D0020B9
:10EFD0002E2E5C2E2E5C2E2E5C626C655F63666747
:10EFE0005C736C6176652E630000000070B58CB0B8
:10EFF00004460D461646002005E0C0F10F01615C95
:10F000000DF80010401C1028F7D30D2104A8F7F7C5
:10F0100050FA002005E02A5CC0F10F0304A9CA548D
:10F02000401C0328F7D3684646DF002005E0C0F106
:10F030000F0208A9895C3154401C0328F7D30CB097
:10F0400070BD000010B5044602480178204603F068
:10F0500051FD10BD584A002070B51649002004F03B
:10F0600005FE05461349012004F000FE044612483F
:10F070000079E8B101F0CAFAD0B11048027910A1C4
:10F080000020FBF719FE0D4801790079401C0B4A5E
:10F09000107105290CDB00201146C870054804F0EA
:10F0A0001DFC0123054AD21CA2210020F8F758FBC1
:10F0B00070BD0000D0A1040094510020C03E00208B
:10F0C00067616D655F6D616E616765722E47616D29
:10F0D000654D6F64654865617274436E743A25646A
:10F0E0000D0A000030B587B0182101A8F7F7E1F943
:10F0F0000DF0EAF808B907B030BD0024002004F094
:10F1000039FC04B2002C7DDD611E01AA002004F050
:10F1100027FCBDF90420604803886049604819F065
:10F120000BFE5D480088052826DDBDF904005B491B
:10F13000B1F90010401AFF281BDC5948B0F9000053
:10F14000BDF90410401AFF2813DC5548B0F900003F
:10F150005249B1F90010401AFF280ADCBDF9040039
:10F1600010F5AF6F05DA4F480088401C4D49088004
:10F1700002E000204B49088047480088401C46496F
:10F180000880BDF8040010FB00F0BDF8061011FB6C
:10F190000100BDF8081011FB0105A5F5800000284D
:10F1A00001DB014600E041423F4A91420ADABDF9E3
:10F1B0000810B1F5C06F05DD3C480088401C3B4994
:10F1C000088002E000203949088038480088052876
:10F1D00003DA34480088042802DD06203449087028
:10F1E00033480078002804DD31480078401E30495B
:10F1F00008702F48007800282FDD2E480078B8B915
:10F20000642000E045E02B490870F9F703FD14285D
:10F2100004DD29490220FAF729FA03E027490220F0
:10F22000FAF724FA0121AFF24310FAF7E3FF0AE0FC
:10F2300020480078022806D1FAF74CFA0021AFF2F4
:10F240005B10FAF7D7FF1B480078012820DD19482A
:10F250000078401E174908701AE01648007850B12F
:10F260000020144908700220FAF734FA0021AFF2A6
:10F270008B10FAF7BFFF1248007848B901201049F7
:10F2800008700220FAF726FA00210E48FAF7B2FFBA
:10F2900000BF00BF2FE70000E03D0020003E00203F
:10F2A000E83D0020E23D0020A0860500E43D00206E
:10F2B000E63D0020E73D0020007F00FF00106FFFCB
:10F2C000DC3D0020C9F2020030B587B0182101A84A
:10F2D000F7F7EFF80CF0F8FF08B107B030BD0024E5
:10F2E000002004F047FB04B2002C70DD611E01AA6F
:10F2F000002004F035FBBDF8040010FB00F0BDF861
:10F30000061011FB0100BDF8081011FB0105A5F561
:10F310008000002801DB014600E041423C4A914266
:10F3200008DABDF90810B1F5C06F03DD03203949D3
:10F33000087008E037480078002804DD3548007878
:10F34000401E34490870A5F58000002801DB014605
:10F3500000E041422E4A914207DABDF9081011F54A
:10F36000806F02DA00202B4908702A4800780028B4
:10F370002EDD29480078A8B90A2027490870F9F736
:10F3800049FC142804DD25490220FAF76FF903E04F
:10F3900023490220FAF76AF90121AFF2D300FAF704
:10F3A00029FF0AE01C480078022806D1FAF792F9F2
:10F3B0000021AFF2EB00FAF71DFF17480078012893
:10F3C00023DD15480078401E134908701DE01DE03C
:10F3D0001148007850B100200F4908700220FAF758
:10F3E00079F90021AFF21F10FAF704FF0D480078F9
:10F3F00001280AD100200B4908700220FAF76AF9A7
:10F400000021AFF23B10FAF7F5FE00BF00BF64E742
:10F41000A0860500DD3D0020DE3D0020007F00FFCE
:10F4200000106FFFDC3D0020044803E0012142682A
:10F430001170406841680029F8D17047883F00206A
:10F440000148007870470000C43F00202DE9F041DA
:10F4500019210020002213461446154600BF4FF024
:10F46000A0473E4642EA430747EA800747EA0427A7
:10F4700047EA054C06F5E06747F821C000BF00BF2A
:10F480000F49A820F7F7BAFE0E49A820F8F78AF826
:10F490000D49A720F7F7B2FE0C49A720F8F782F82C
:10F4A0000B4A0CA14FF47A70FAF7C8FE00F032F85C
:10F4B0000B4A0CA10A20FAF7C1FEBDE8F08100005A
:10F4C00055510300B14F0300E54B0300694F0300A2
:10F4D00015F502006170705F636861726765000016
:10F4E000D1F602006170705F6368617267655F6D7D
:10F4F0006F6E69746F725F626174746572795F6355
:10F5000068617267655F646174615F70726F636583
:10F510007373000038B519F069F960B14348007899
:10F5200048B902F063FA0020009001236A46A7213F
:10F53000F8F716F90DE019F059F950B93B48007881
:10F5400038B13B48007920B900203A4908703A495F
:10F55000087019F04BF935490978884203D019F041
:10F5600045F932490870192012F0CDF90446CCB99A
:10F5700032480078012814D031A10020FBF79CFB11
:10F5800001202E49087000213148FAF733FE05208A
:10F59000FAF7A0F802F02AFA002026490870264956
:10F5A000087038BD2248007908B100F069F8224897
:10F5B0000078022803D02048007803281FD1F9F7EB
:10F5C00029FB64281BDB1B480078642817DB1B48D9
:10F5D0000078032828D0174802781EA10020FBF7E6
:10F5E0006BFB03201549087001211948FAF702FE48
:10F5F0001D490520FAF73AF802F0F8F914E00F482F
:10F600000078022810D019A10020FBF755FB02203A
:10F610000A49087001210E48FAF7ECFD1749052048
:10F62000FAF724F802F0E2F900BFBAE7C73F00207A
:10F6300094510020C53F0020C63F0020C43F002059
:10F64000636861726765206F75742E2E2E0A000044
:10F6500015F5020063686172676520646F6E653A34
:10F6600025642E2E2E0A0000007F00FF6368617261
:10F67000676520696E2E2E2E0A00000000106FFFB5
:10F680003EB500200090019002900024F9F7C2FAE4
:10F690002246641C0DF802000B4802782146641CC7
:10F6A0000DF801200948007930B123466A46A821A7
:10F6B0000020F8F755F805E023466A46A821002007
:10F6C000F7F772FE3EBD0000C43F002094510020B9
:10F6D0002DE9F041002600BF0027192012F013F990
:10F6E0008046B8F1000F21D10420F7F7D5FA4FF486
:10F6F000167110FB01F5E81705EB1050001300EB35
:10F700004000400004B23748B0F90000A04201DDDB
:10F71000204602E03348B0F900003249088000205A
:10F720003149088032203149086059E02F4800688B
:10F7300008B30420F7F7B0FA4FF4167110FB01F587
:10F74000E81705EB1050001300EB4000400004B236
:10F750002548B0F90000A04201DA204602E0224824
:10F76000B0F900002049088020480068401E1F4969
:10F770000860BDE8F0810420F7F78EFA4FF41671A7
:10F7800010FB01F5E81705EB1050001300EB4000EB
:10F79000400004B21448B0F90000A04201DA20464B
:10F7A00002E01148B0F900000F4908800720F7F780
:10F7B00073FA4FF4167110FB01F5E81705EB1050C2
:10F7C000001300EB4000400000EB8000032190FBA1
:10F7D000F1F006B20448008802490988401A07B2CD
:10F7E00000BFC6E7CC3F0020CE3F0020C83F00202E
:10F7F00030B589B0002468464CDF00988010009036
:10F8000001222146641C01A84254F9F703FA01467B
:10F810002246641C01A881540098C2B22146641C8F
:10F8200001A8425400222146641C42542146641C13
:10F8300042542146641C42542146641C42544D48A3
:10F840004069020E2046611CCCB201A90A54494805
:10F850004069C0F307422046611CCCB201A90A549A
:10F860004448808AC0F307222046611CCCB201A91B
:10F870000A544048027D2046611CCCB201A90A54BA
:10F8800001F0C6F92146621CD4B201AA505401F01D
:10F89000B3F92146621CD4B201AA505401F0A6F972
:10F8A000020E2046611CCCB201A90A5401F09EF957
:10F8B000C0F307422046611CCCB201A90A5401F0F2
:10F8C00095F9C0F307222046611CCCB201A90A5465
:10F8D00001F08CF9C2B22046611CCCB201A90A54D5
:10F8E00024488069020E2046611CCCB201A90A544A
:10F8F00020488069C0F307422046611CCCB201A9B0
:10F900000A541C48008BC0F307222046611CCCB26D
:10F9100001A90A541748027E2046611CCCB201A9F5
:10F920000A540CF03DF80546C5F307222046611C39
:10F93000CCB201A90A542046611CCCB201A90D54D5
:10F9400001F060F9C0F307222046611CCCB201A986
:10F950000A5401F057F9C2B22046611CCCB201A989
:10F960000A54234601AAA1210020F7F71DFD09B082
:10F9700030BD00009451002070B50546002400BF42
:10F9800006E0601C6968095C0A480155601CC4B245
:10F99000082CF6DB6968487A01F048FA05480C380B
:10F9A000406A28B1002103480C38416209F056FF33
:10F9B00070BD0000A051002010B50849A120F7F744
:10F9C0001DFC00F00FFA0648007928B9054A06A187
:10F9D0004FF4FA60FAF732FC10BD0000AD4E0300A0
:10F9E00094510020F5F902006170705F636C6965E5
:10F9F0006E74000010B518F0F9FE90B100F006FE2C
:10FA000068B1084801780078401C064A1070042943
:10FA100007DB002011460870FFF7EAFE01E0FFF760
:10FA2000E7FE10BD123F002070B504466068807884
:10FA30006168497840EA01251648406AA0B1154836
:10FA4000406A401E2821B0FBF1F0401C124908809A
:10FA50001048406A401E2821B0FBF1F201FB120061
:10FA6000401C0E49088004E000200B4908800B4927
:10FA7000088055B901200A4908700020094908800A
:10FA80000846008800F010F802E0284600F090F8E0
:10FA900070BD0000945100201C3E00201E3E00203E
:10FAA000193E00201A3E00202DE9F04105460024B1
:10FAB00009F0D1FE691EA02202FB010702222146A5
:10FAC000641C36484254002007E035490B5C21464F
:10FAD000621CD4B2314A5354401C0828F5DB31482B
:10FAE000008802122046611CCCB22C490A542D48D1
:10FAF00002782046611CCCB228490A542A122146B9
:10FB0000601CC4B2254842542146601CC4B223483C
:10FB1000455405BB01F0BAFF804601F0BDFF08EB7C
:10FB20000006320E2046611CCCB21C490A54C6F3B2
:10FB300007422046611CCCB218490A54C6F307227A
:10FB40002046611CCCB215490A542046611CCCB237
:10FB500012490E541AE01348008885420DD112480C
:10FB6000008882000D480119384609F05FFE0E48F2
:10FB7000007804EB8000C4B208E008480119A02214
:10FB8000384609F053FE04F1A000C4B22346034AEC
:10FB9000A1210648F7F708FCBDE8F081804F00205E
:10FBA000A05100201C3E00201E3E0020203E0020D0
:10FBB00070B5C0B00546002409F04DFE691EA022B4
:10FBC00002FB010602222146641C01A842540020C7
:10FBD00007E023490B5C2146621CD4B201AA5354AE
:10FBE000401C0828F5DB1F48008802122046611CD3
:10FBF000CCB201A90A541B4802782046611CCCB241
:10FC000001A90A542A122046611CCCB201A90A5447
:10FC10002046611CCCB201A90D54124800888542CF
:10FC20000DD111480088820001A80119304609F061
:10FC3000FDFD0D48007804EB8000C4B208E001A887
:10FC40000119A022304609F0F1FD04F1A000C4B270
:10FC5000234601AAA1210020F7F7A6FB40B070BD02
:10FC6000A05100201C3E00201E3E002070B5A2B016
:10FC7000412480216846F6F71CFC00208DF8000026
:10FC800000BF05E049A10A5C411C0DF80120401CA1
:10FC90000B28F7D320A86DDF054600BF2E4636B1EE
:10FCA00000BF45A27C213046F6F7B4FA00BF00BF82
:10FCB00000200AE0C0F105020DF181018B5C2146B4
:10FCC000621CD4B20DF80130401C0628F2DB002281
:10FCD0002046611CCCB20DF8002001222046611C98
:10FCE000CCB20DF800202046611CCCB20DF80020EB
:10FCF0002046611CCCB20DF8002000222046611C79
:10FD0000CCB20DF800202A222046611CCCB20DF89E
:10FD10000020002007E02F490B5C2146621CD4B272
:10FD20000DF80130401C0628F5DB2A483238C06A3D
:10FD3000020E2046611CCCB20DF800202548323856
:10FD4000C06AC0F307422046611CCCB20DF8002007
:10FD500020483238808DC0F307222046611CCCB287
:10FD60000DF800201B48323890F82C202046611CEA
:10FD7000CCB20DF8002017483238008E021220460F
:10FD8000611CCCB20DF800201248323890F83020B7
:10FD90002046611CCCB20DF8002023466A46A12102
:10FDA0000020F7F701FB22B070BD0000534D415217
:10FDB000542053484F4500002E2E5C2E2E5C2E2ED4
:10FDC0005C6170705C6170705F636C69656E742EED
:10FDD00063000000C6510020014800787047000011
:10FDE000183E002010B50E4A0EA14FF47A70FAF7B3
:10FDF00025FA10484169C069814202D20D48416923
:10FE0000C1610C480CA1426A0020FAF755FF09486D
:10FE1000836910A142690020FAF74EFF10BD00006F
:10FE20008DFE02006170705F636C69656E745F7354
:10FE300074657000945100206D466C6173682E6D7E
:10FE4000537465702E737465705F6E756D3D2564B7
:10FE50000A0000006D466C6173682E6D5374657006
:10FE60002E737465704375725B305D3D25642C6D37
:10FE7000466C6173682E6D537465702E7374657073
:10FE80004375725B315D3D25640A000010B5214861
:10FE9000007820B101280DD0022833D11BE01E4884
:10FEA0000078012805D11B490870FCF751F91B495E
:10FEB00008602DE0FCF74CF918490968401A42F235
:10FEC0001071884203D302201249087002E0012019
:10FED00000F066FE1CE0F8F75DFD18B110A10B20E4
:10FEE000F7F734FF00200C4908700A490870FCF746
:10FEF0002FF904460E4822460EA183690020FAF726
:10FF0000DBFE05E00020034908700349087000BFCC
:10FF100000BF10BD443E0020183E0020483E002097
:10FF2000736176652073746570206661696C00008A
:10FF300094510020466C6173685F53617665496E29
:10FF4000666F6D6174696F6E3A25642C6D466C61E5
:10FF500073682E6D537465702E737465704375727B
:10FF60005B315D3A25640D0A000000000120014963
:10FF700008707047183E002010B53648007810B160
:10FF800001285BD109E018F031FC28B1012031498A
:10FF9000087000203049087059E00CF011FAC0B127
:10FFA0002D480078F8B901202B49087000F048FA74
:10FFB0002A49087001230A46A3212948F7F7F4F9D2
:10FFC000FCF7C6F80446224626A10020FAF774FE84
:10FFD00009E021480078002805DD00201E4908704E
:10FFE0001F48F7F789F92B48008898B1FCF7B0F85B
:10FFF00029490968401A2749098888420AD30020FC
:020000040003F7
:10000000244908800220F9F765FB0021AFF2970030
:10001000FAF7F0F818F0EAFB78B900200D490870FB
:100020001C4908800021AFF2AF00FAF7E3F8022084
:10003000F9F750FB0A48F7F75FF908E00020054997
:100040000870144908800220F9F744FB00BF00BF84
:1000500010BD0000413F0020403F0020423F0020F3
:10006000143F00203D3D3D3D3D3D3D3D3D3D3D3D41
:100070003D3D3D3D3D3D3D3D3E424C455F486F73FE
:10008000745F545F434F4E4E45545F4C45443A2590
:10009000640A0000383F00203C3F002070B58048D3
:1000A000007820B1012834D002287CD189E0FFF704
:1000B00093FE30B918F09AFB18B9FFF7C1F901287F
:1000C0001BD001F09FF9C0B918F090FB0446FFF770
:1000D00083FE054623462A4672A10020FAF7ECFD6E
:1000E0000121AFF24700FAF785F816F0F5FF00207E
:1000F0007349086001206A4908707248007938B174
:1001000018F074FB20B90CF05BF908B10CF010F991
:10011000C4E0FFF761FEC8B918F068FBB0B9FFF79B
:100120008FF9012812D168A10E20F7F70FFE6DA1FB
:100130000020FAF7C1FD11F072F80021AFF2A30020
:10014000FAF758F800205649087016E00CF038F914
:1001500098B16BA10020FAF7AFFD0021AFF2C30008
:10016000FAF748F85748007920B100206A4908801A
:100170006A49087002204A49087051480068401CCA
:100180004F49086064281BD3FFF726FE40B94D484D
:1001900090F82800432803D161A10F20F7F7D6FD7E
:1001A00066A1002000E075E0FAF786FD11F037F84F
:1001B0000021AFF21710FAF71DF800203849087037
:1001C0006CE000F023FA18B354480078022842D0BB
:1001D000514800883C283EDCF1EE0E0AB1EE0E0AD2
:1001E000F7F75EFB30B902204C49087000204A49FD
:1001F000088030E0484800883C2803D159A10F20EE
:10020000F7F7A4FD44480088401C4349088022E0D9
:100210004248007801281ED03F4800883C281ADC5C
:10022000DFED590A9FED580AF7F73AFB30B9012084
:100230003A4908700020384908800CE036480088A8
:100240003C2803D151A10F20F7F780FD32480088E8
:10025000401C31490880FFF7BFFD58B918F0C6FAB5
:1002600040B9FFF7EDF8012804D10CF0A9F808B166
:100270000CF05EF80CF0A4F858B94DA10020FAF784
:100280001BFD0021AFF2EB10F9F7B4FF0020044989
:10029000087003E000200249087000BF00BF70BD75
:1002A000433F00203D3D3D3D3D3D3D3E7363616E1E
:1002B0005F73746172743A25642C25640A0000002F
:1002C000443F002094510020616476206469736388
:1002D0006F6E6E746564206F7665722074696D65EB
:1002E000000000003D3D3D3D3D3D3D3E6E72665F80
:1002F000626C655F7363616E5F73746F700A000098
:100300003D3D3D3D3D3D3D3E686F73745F697363A8
:100310006F6E6E6563740A00483F00204A3F0020FC
:100320007363616E2072696768742073686F6573A8
:10033000206F7665722074696D6500003D3D3D3D1E
:100340003D3D3D3E6170705F6572725F5365742024
:100350006E72665F626C655F7363616E5F73746F0C
:10036000700A000075706461746520426C652063DA
:100370006F6E6E20696E74657276616C20372E35F3
:100380006D73206661696C000000C842757064611D
:10039000746520426C6520636F6E6E20696E7465B3
:1003A0007276616C203130306D73206661696C004B
:1003B0003D3D3D3D3D3D3D3E686F73745F646973F7
:1003C000636F6E6E6563740A0000000010B50E481E
:1003D000007920B10D4A0EA16420F9F72FFF0F48D4
:1003E000F7F726FA0E48F7F7EBF90E4A0EA164204C
:1003F000F9F724FF1049A320F6F700FF0F49AC20BE
:10040000F6F7FCFE10BD0000945100209D00030093
:100410006170705F636F6E6E65637400E551030019
:10042000A151030079FF02006170705F636F6E6E0F
:100430006563745F6C656400E14A0300FD4A030074
:1004400010B50024064890F82800432801D0022463
:1004500003E00BF0B5FF00B10124204610BD000001
:100460009451002010B5054A05A10020F9F7E6FED9
:100470000A48F7F7C1F8002010BD0000A1040300EE
:100480006170705F646174615F7472616E736665E0
:10049000725F50726F636573730000004105030063
:1004A00010B500F0B3F818B901F080FC002832D084
:1004B0001E48007830B901201C49087001211C48F1
:1004C000F9F798FEFBF744FE1A490968401AB0F59F
:1004D000FA7F12D3FBF73CFE1649086018F086F944
:1004E00018B9FEF761FDFEF73DFD1348007920B114
:1004F0000BF066FF08B916F0EFFDFBF729FE0F4978
:100500000968401A032810D3FBF722FE0B49086044
:10051000F8F744FD09E00548007830B100200349B0
:10052000087000210248F9F765FE10BDC03F0020A9
:10053000A1040300B83F002094510020BC3F0020DC
:1005400070B504460D46E078042803D129462046BC
:10055000F8F7EEFD00F0DCF970BD00002DE9F04782
:1005600004460D461646324629462046F8F776F9E7
:100570001CA10020FAF7A0FB142001210A46002349
:100580001F469C4600BF4FF0A049C84641EA4209B9
:1005900049EA830949EA072949EA0C4908F5E06A6A
:1005A0004AF8209000BF00BF002159B900BF00BF2A
:1005B00082061346012707FA00F2C3F80C2500BF94
:1005C00000BF0CE000BF00BF4FF0A0421346012760
:1005D00007FA00F2C3F8082500BF00BF00BF00BF44
:1005E000BDE8F0876170705F6572726F725F6661FF
:1005F000756C745F68616E646C65722C537973748A
:10060000656D2072657365740A00000001484079C9
:1006100070470000C03E002010B50A4A0AA14FF4FE
:100620007A70F9F70BFE0B49A220F6F7E7FD0A4AAC
:100630000AA14EF66020F9F701FE0C49012003F0F3
:1006400017FC10BD710603006170705F67616D6516
:1006500000000000D54C030059F002006170705F8B
:100660004175746F4F757467616D650011AD03005E
:1006700070B5002400256D480078002804DD6B4823
:100680000078401E694908706948007810B1012857
:1006900076D148E06548C078002839D06549002007
:1006A00003F0E4FA04466349012003F0DFFA05464B
:1006B0002B46224660A10020FAF7FEFA802C07D1D3
:1006C000802D05D101205A4908705849487119E018
:1006D000402C01D1402D15D0564803F0D7F85D4885
:1006E0000078401CC0B25B49087014280ADB002067
:1006F00008704E49C8704F4803F0F0F856A1092021
:10070000F7F724FB4948007910B1002047490871E8
:1007100046480078002805DD5648007910B10020D1
:1007200000F038F97FE05348007900282ED00BF014
:1007300047FE30B33D480078A0B9012000F02AF907
:1007400044480078401CC0B2424908700A2810DBB7
:100750000020087048A1FAF7AFFA4FA10920F7F777
:10076000F5FA06E03B480078002802DD0020394910
:1007700008702E48407848B100202C49487005E0A8
:100780004AE02A484078401C2849487018F02EF862
:1007900028B926488078401C2449887005E0234801
:1007A000807810B10020214988702048C07838B185
:1007B0001E488078052803DC1C4840780A282ADD7A
:1007C0001A4840780A2803DD39A10920F7F7BEFA54
:1007D00016488078052803DD41A10920F7F7B6FA0D
:1007E00000201C490870124908701049C8708870B0
:1007F000487048710F4803F071F81E48007910B135
:10080000002000F0C7F800204049087017F0ECFE07
:10081000002000F087F806E0002005490870034931
:10082000C870887000BF00BF70BD0000C03E0020CF
:10083000DB3E0020D0A1040066726F6E745F4353EC
:100840003A2564206261636B5F43533A25640D0A65
:1008500000000000DA3E002073686F657320696E47
:10086000746F2067616D65206D6F646520666169D6
:100870006C000000945100204552525F4E554D5F70
:1008800047414D45206170705F67616D655F5072D3
:100890006F636573730D0A006E6F20676574207255
:1008A000696768742073686F6573206461746100A0
:1008B000496E2067616D65206D6F64652C72696794
:1008C00068742073686F657320646973636F6E6EFC
:1008D000746564206C6F6E672074696D650000003C
:1008E000496E2067616D65206D6F64652C636C696E
:1008F000656E7420646973636F6E6E746564206CDA
:100900006F6E672074696D6500000000CD3E0020A9
:1009100003480078032802D003200149087070477B
:10092000C03E002010B504462CB317480078401C88
:100930001549087008460078642811D113480078DA
:1009400038B100201149087011490120F8F78EFED6
:1009500006E001200D4908704FF07F41F8F786FE50
:100960000948007866280DDD00200749087001203D
:10097000F8F7B0FE06E005480078022802D1012011
:10098000F8F7A8FE10BD0000D93E0020D83E002098
:10099000007F00FF38B50446009401236A46A22177
:1009A0000020F6F7DDFE38BD70B586B01821684628
:1009B000F5F77FFD002400255B48007830B1012861
:1009C0002BD0022868D003287ED191E0FFF71EFECD
:1009D000002821D15548007801281DD10121544813
:1009E000F9F708FC534802F051FF01204E49087006
:1009F00000204E49087050490870FBF7A9FB4F4989
:100A00000860FBF7A5FB4FF47A71B0FBF1F63246B4
:100A10004BA10020FAF750F982E04649002003F08C
:100A200025F904464349012003F020F90546802CAE
:100A300010D1802D0ED102203B4908700A213C487C
:100A4000F9F76EFC00204C490880FBF781FB3B491D
:100A500008601AE0402C01D1402D16D0354802F034
:100A600015FF35480078401CC0B23349087014287F
:100A70000BDB002008702F4802F030FF03202A49CA
:100A800008703EA10920F7F761F9FFF7BFFD10B12B
:100A900003202549087043E0002002F06BFF012885
:100AA00011DB6A460021084602F05AFF3248B0F9CD
:100AB00000100DF1060008F093FB2F480088401C41
:100AC00000B22D49088000E024E0FBF741FB1B4900
:100AD0000968401A42F21071884202D30320124979
:100AE0000870FFF793FD10B103200F49087017E05D
:100AF0004FF47A710E48F9F713FC0E4802F0EEFE3F
:100B000000210B48F9F776FB0020074908700A49D5
:100B1000087005E00020044908700749087000BF0C
:100B200000BF06B070BD0000703F0020543F0020A1
:100B3000A9090300F0A10400783F0020743F0020C1
:100B40003D3D3D3D3E3E3E3E48414C5F5345525F3C
:100B5000494D555F4D4F44455F4D414E4147455FBF
:100B600043414C4942524154494F4E2C74696D3AAD
:100B7000256420730D0A0000723F002073686F65C2
:100B80007320696E746F2043414C4942524154496D
:100B90004F4E206D6F6465206661696C0000000037
:100BA00010B504460123094AA1210020F6F7D8FD1B
:100BB0000748007840B9022C06DB05480470012381
:100BC000024AA121F6F7CCFD10BD0000A13E002095
:100BD0007C3E002010B50123024AA1210248F6F70D
:100BE000BFFD10BDA03E0020583E00200148006817
:100BF00070470000503E0020014800787047000018
:100C00004D3E00200148B0F900007047543E0020DE
:100C100001480078704700004C3E002010B50448A1
:100C20000079012803D10349A120F6F7BBFC10BDD0
:100C3000945100205150030010B50548007928B1A7
:100C4000044A05A14FF47A70F9F7F8FA10BD0000D4
:100C500094510020F59902004C6F73735061636BDF
:100C60005F70726F636573730000000030B58BB006
:100C70000025182101A8F5F71CFC0BF025FB002826
:100C80003DD020480078012839D0002002F072FEC3
:100C900005B2002430E001AA2146002002F060FEE7
:100CA000BDF81000ADF81C00BDF81200ADF81E0034
:100CB000BDF81400ADF82000BDF80400ADF8240024
:100CC000BDF80600ADF82600BDF80800ADF8280014
:100CD000BDF9281007A805F0A1FC01280BD10A488E
:100CE0004069401C08494861084608A14269002043
:100CF000F9F7E2FF02E0641CAC42CCDB00BF0BB0B2
:100D000030BD0000A43E0020945100204461696C75
:100D100079537465702063757272656E7420737494
:100D200065703A25640D0A0070B5002521480468F5
:100D300021480068844201D204F180741E48006892
:100D4000201A1E49096808441C49086008460068C2
:100D50001B49B1F900100844C50BB4F1807F04D9D8
:100D6000A4F180701449086001E013480460B5F5EF
:100D7000E16F08D313480078012804D001201149FD
:100D8000087011490870B5F5616F11D300200B4947
:100D90000860FFF7EBF801200B49087000200949B3
:100DA00008702B46054809A102680020F9F784FF66
:100DB00070BD000004B500406C3F0020503F002093
:100DC000563F0020683F0020543F002074696D6545
:100DD000434E5428256429282564290A0000000070
:100DE00010B5064A06A14FF4FA70F9F727FA0A4A35
:100DF0000AA14FF47A70F9F721FA10BDA90903008E
:100E00006170705F6779726F5F4669785F70726F4B
:100E10006365737300000000290D03006170705F4B
:100E20006D6174685F486F75720000002DE9F047CE
:100E30002DED048B8AB0064600BF00BF4848007BFA
:100E4000020600214648407B094342EA0040444AEA
:100E5000927B4FEA022C0A4640EA0C014048C07BD4
:100E600001433F48037C0020000640EA132042EA89
:100E7000036201433A48437C0020000440EA134CDB
:100E800042EA034041EA0C01354A937C00221202F7
:100E900042EA136C40EA032241EA0C053049C97C5E
:100EA00042EA01042F4807682F490968781AF5F7C4
:100EB000E5FC9FED2E0B53EC102BF5F749FCF5F7F5
:100EC00009FD00902B480068231A32462AA14FF0F2
:100ED0000000F9F7F1FE00BF4EF660220023204625
:100EE0002946F5F78DFA02F0FF091E480068C00B8D
:100EF0003C21B0FBF1F201FB12081A480068C00B5C
:100F0000B0FBF1FA4B46324626A10020CDE900A8FD
:100F1000F9F7D2FE202102A8F5F7CBFA202102A88A
:100F2000F5F7C7FA0F480068C00B3C21B0FBF1F899
:100F30004346324624A102A8FCF7A6F802A90B20DA
:100F4000F6F704FFC6EB0610400406490860094A9C
:100F500030C2054807600AB0BDEC048BBDE8F087DD
:100F600094510020503F0020643F0020FCA9F1D2A2
:100F70004D624040583F00206170705F6D61746841
:100F80005F63616C69745F74696D653A7265616C09
:100F90006D696E7574653A25642C256C752C256C0D
:100FA000750A000061707074696D65203A202575BE
:100FB0003A25752C73686F65732074696D653A20E6
:100FC0002025753A25750A006170706D696E75741B
:100FD000653A25642C6D6375206D697574653A25D5
:100FE0006400000070B511486DDF044600BF25465F
:100FF00035B100BF0EA2CC212846F5F70BF900BF92
:1010000000BF114A11A10020F9F718F91349A620D1
:10101000F6F7F4F81249A620F6F7C4FA114A12A11D
:101020004FF4FA70F9F70AF970BD0000DC3E0020B9
:101030002E2E5C2E2E5C2E2E5C6170705C617070AA
:101040005F6F74612E6300007D1003006170705F3C
:101050006F74615F50726F6365737300254C03009A
:10106000CD4F0300311303006170705F6F74615FD7
:10107000636C6561725F666C6173680010B58AB0FD
:10108000002005907048007820B101286BD002281C
:1010900076D18BE06D48007900281ADD6C48007825
:1010A00001285FD16BA10020F9F706FE01206649F7
:1010B00008700BF03DF910F0B2F842F210716A4876
:1010C000F9F72EF9012305AAA6210020F6F76CF9FD
:1010D00048E066480068012844D165480078012846
:1010E00040D10020614908606149087017F07EFB1B
:1010F00010B117F043FB01E0FDF756FF002006900A
:101100000790089009905B4840785A498978594A75
:10111000D278584B1B79CDE90032CDE90210554801
:101120004379827954A106A8FBF7AEFF06A8F5F72C
:10113000CBF9044606AB224656A10020F9F7BCFDC8
:1011400006A8F5F7C1F90446214606A817F054FB96
:1011500017F00CFB01203C4908704FF4FA6142483B
:10116000F9F7DEF86DE039480079002809DD002044
:1011700037490870344908704BA1F9F79DFD14E018
:1011800057E017F033FB70B94DA10020F9F794FD3B
:10119000FDF7E8FE42F210713348F9F7C1F802207A
:1011A0002949087001E017F0E9FA4AE017F01EFB40
:1011B00010B100202449087000212B48F9F7B0F83D
:1011C000FDF7F2FE002006900790089009901F4856
:1011D00090F8371090F8362090F835001B4BDB79EB
:1011E000CDE90030CDE902211848837942793DA14B
:1011F00006A8FBF749FF06A8F5F766F9044606AB13
:1012000022463FA10020F9F757FD06A8F5F75CF943
:101210000446214606A817F0EFFA3EA10E20F6F785
:1012200095FD17F0A3FAFDF79DFE00200649087012
:1012300007E000200449087000210B48F9F770F816
:1012400000BF00BF0AB010BD103F00209451002025
:10125000E83E00202D2D2D2D2D2D3E6973486F73F6
:10126000744F54410A0000007D100300E43E00204A
:10127000EA3E0020DC3E002053485F2530325825EE
:1012800030325825303258253032582530325825E2
:10129000303258004F5441206E616D652825642915
:1012A0003A25730A000000002D2D2D2D2D2D3E6CAA
:1012B000656674206F757420746F206466750A000B
:1012C0006170705F6F74615F50726F6365737320DC
:1012D0006164766572746973696E675F7374617255
:1012E000740D0A00253032582530325825303258D6
:1012F0002530325825303258253032580000000051
:10130000414456206E616D65282564293A25730A8B
:101310000000000061647620646973636F6E6E7410
:101320006564206F7665722074696D650000000049
:1013300010B51B48007801282AD1F8F7F1F8F7F723
:1013400029FB18B117A10E20F6F700FD2422194938
:101350001948F5F795F81849164814F035FB0020A0
:1013600016494876F7F728FA18B115A10E20F6F7B6
:10137000EDFCF7F7F9F918B118A10E20F6F7E6FC25
:101380001BA10020F9F798FC02200549087006E02F
:1013900003480078022802D1042010F0DFFC10BDC1
:1013A000E93E002073617665207374657020666184
:1013B000696C00005C4F0020005200202452002085
:1013C0006F7461207361766520696E666F726D61FE
:1013D00074696F6E206661696C0000006F74612033
:1013E00073617665206261636B206661696C0000E1
:1013F0002D2D2D2D2D2D3E7361766520666C61732C
:10140000680A00000148007870470000E83E0020AC
:1014100010B5064A06A16420F8F710FF074A08A194
:101420004FF47A70F8F70AFF10BD0000E5F00200F3
:1014300042617444697370616C790000C9F2020002
:1014400042617444697370616C795F4E0000000002
:1014500070B50E486DDF044600BF25463DB100BFA4
:101460000BA240F22D112846F4F7D4FE00BF00BFB6
:101470000D4A0EA16420F8F7E1FE11490120FBF7A7
:101480001BF810490220FBF717F870BD7C3F0020C5
:101490002E2E5C2E2E5C2E2E5C6170705C61707046
:1014A0005F706169722E6300C91403006170705F20
:1014B000706169725F50726F636573730000000042
:1014C000415303002552030030B589B0FDF7B8FF42
:1014D00001282FD0A7480078012811D00120A54964
:1014E0000870A548007928B1A44A13210846FAF7E4
:1014F00051FF32E0A14A13211620FAF74BFF2CE0EE
:101500009F480088322828DA9D480088401C9C4962
:1015100008809948007900B3984A13210846FAF7E1
:1015200039FF0120FAF798FE944A13211620FAF7A2
:1015300031FF12E08F480078022807D002208D4941
:10154000087013210846FBF7B7F806E08C480088BE
:10155000002802DD00208A4908800024894800789C
:1015600010B101287AD168E087480078002863D05C
:101570000020854908704FF4FA70F8F7ABFAF6F7D7
:1015800084FD20B181A10B20F6F7E0FBEEE01C21E9
:1015900079480C30F4F78DFF4320774981F8280013
:1015A000F7F7F8F938B17DA10B20F6F7CFFB7FA153
:1015B0000020F9F781FB704890F8371090F836203A
:1015C00090F8353090F83400CDE901320391009065
:1015D000694890F8333090F832207DA10020F9F767
:1015E0006BFB00240CE06448401D015D86480155FA
:1015F00061483230015D8448801D0155601CC4B2D1
:10160000062CF0DB5C48C06A7F49091F08615A4814
:10161000008E8882584890F828008875F7F7A4F85B
:1016200018B17AA10C20F6F791FB012055490870FA
:10163000FAF78EFD7B49086098E0FAF789FD794951
:101640000968401A42F2107188420BD3FAF780FD04
:101650007449086000204B49087000E082E072A1E4
:10166000F9F72AFB4448007900283CD00AF0A8FE8C
:1016700010B10AF05DFE74E070A10020F9F71CFBC8
:10168000002005900690079008903B4890F837207E
:1016900090F8361090F83500374BDB79CDE9003003
:1016A000CDE902123448837942796BA105A8FBF792
:1016B000EBFC05A8F4F708FF054605AB2A466DA12B
:1016C0000020F9F7F9FA05A8F4F7FEFE05462946C9
:1016D00005A80AF07BFEF9F779FDF9F753FD002024
:1016E000284908703DE017F081F810B117F046F86E
:1016F00037E0002005900690079008901E4890F86B
:10170000372090F8361090F835001B4BDB79CDE987
:101710000030CDE902121848837942794EA105A81C
:10172000FBF7B2FC05A8F4F7CFFE054605AB2A4649
:1017300055A10020F9F7C0FA05A8F4F7C5FE054643
:10174000294605A817F058F8FDF72EFC17F00EF8FB
:1017500051A10020F9F7B0FAFDF704FC0020094977
:10176000087003E000200749087000BF00BF09B0FF
:1017700030BD0000903F00209451002090D0030025
:10178000843F0020913F0020863F0020636C65610C
:10179000722073746570206661696C007361766590
:1017A0002073746570206661696C0000455843457C
:1017B00050545F444154455374657020736176659D
:1017C0002073746570206661696C0D0A000000006A
:1017D0006D466C6173682E6D436C69656E742E6D19
:1017E0006163416464723A253032582025303258A2
:1017F00020253032582025303258202530325820CC
:10180000253032580A0000002852002070616972A9
:101810002073617665206261636B75702066616913
:101820006C000000943F0020506169725F73746126
:101830007465203D30200D0A000000003E3E3E3E13
:101840003E53545F7363616E5F7374617274203DC5
:1018500030200D0A00000000253032582530325863
:1018600025303258253032582530325825303258FC
:10187000000000007363616E4E616D652825642968
:101880003A25730A000000006164764E616D652898
:101890002564293A25730A003E3E3E3E3E3E3E3ECA
:1018A0006164766572746973696E675F737461727F
:1018B00074203D30200D0A0010B50648407E401CC3
:1018C00004494876044A05A142F21070F8F7B6FCC4
:1018D00010BD000024520020F11803006170705FF9
:1018E000736166655F50726F63657373000000001B
:1018F00000B58BB02048007E002816DD1F48007818
:10190000401C1E4908700846007806280DDB0020A0
:1019100019490876F6F728FF18B119A10D20F6F736
:1019200015FA1DA10020F9F7C7F91348407E0128D8
:1019300020DD282101A8F4F7BCFD282101A8F4F737
:10194000B8FD1D48007930B10B48427E1BA101A8AB
:10195000FBF79AFB05E00848427E1EA101A8FBF7B1
:1019600093FB01A90D20F6F7F1F910B90020024907
:10197000487600BF0BB000BD24520020C13F0020BC
:1019800073617665204572725374617274436E742C
:10199000206661696C000000636C656172206D42B5
:1019A00061636B75702E4572726F725374617274DD
:1019B000466C61670A000000945100206C656674F3
:1019C0002073686F657320726573746172743A2551
:1019D0006400000072696768742073686F65732023
:1019E000726573746172743A2564000038B5002022
:1019F000009000240E48007930B100222046611C7E
:101A0000CCB20DF8002005E001222046611CCCB2CA
:101A10000DF80020074802782046611CCCB20DF872
:101A2000002023466A46A7210020F5F7BDFC38BDFB
:101A300094510020C43F002010B50446022C0FD161
:101A40000C48007810B1012807D104E001200949B1
:101A50000870002010BD0020FCE700BF00BF01E0BF
:101A60000120F7E700BF04A10020F9F725F90120C4
:101A7000F0E70000E93E0020496E746F20626F6F4E
:101A8000746C6F616465720A00000000014840696F
:101A900070470000945100200148806970470000A1
:101AA0009451002010B50F48007920B90E4A0FA1BB
:101AB0006420F8F7C3FB1149A520F5F79FFB104AF6
:101AC00010A16420F8F7BAFB1349A520F5F76AFDC9
:101AD0001249012002F0CCF9114A12A10020F8F7B6
:101AE000ADFB10BD94510020DD1C030073746570C4
:101AF0005F5265616C53656E64000000614D0300C8
:101B0000411B0300737465705F5265616C436F6EB7
:101B10006E65637400000000015003000565040059
:101B20006D0C03006170705F6D6174685F44616982
:101B30006C79537465705F50726F636573730000E6
:101B400038B500200090002400255348007820B1CB
:101B500001281CD0022872D156E050480078012894
:101B600008D14D49087000204D4908704D4801F0DA
:101B70008DFE0BE04C480078002807DD00204A4924
:101B800008700123454AA521F5F7EAFD81E04549A2
:101B9000002002F06BF804464249012002F066F88A
:101BA0000546802C15D1802D13D140A10020F9F7D6
:101BB00083F8022038490870434840694349086067
:101BC00000204349086043490880012042490870C9
:101BD00019E0402C01D1402D15D0324801F056FEBD
:101BE0002F480078401C2E490870084600781428B9
:101BF00009DB2C4801F072FE0020274908702749B4
:101C000008703549087044E032480088401C31496A
:101C1000088008460088B0F5167F11DB0020088098
:101C2000009001236A46A521F5F79AFD1D4801F0B1
:101C300055FE0020284908701749087014E020E07C
:101C400019480078002804DD17480078401E16491E
:101C500008701548007838B90120009001236A46C1
:101C6000A5210020F5F77CFD0C48007840B9002044
:101C7000194908700B4801F031FE00200649087030
:101C800007E00020054908701349087002490870F0
:101C900000BF00BF38BD0000BC3E0020B43E0020A5
:101CA000BD3E0020B0A10400B03E00203E3E3E3EBE
:101CB0003E3E696E746F207265616C20737465704E
:101CC000206D6F64650A000094510020A83E00203A
:101CD000AC3E0020B23E0020A43E00201CB52F48A0
:101CE0000078012858D100200090019000240122A2
:101CF0002146641C0DF801202948406929490968DA
:101D0000401A020E2146641C0DF801202448406947
:101D100024490968401AC0F307422146641C0DF8A3
:101D200001201F48808A1F490988401AC0F30722F2
:101D30002146641C0DF801201948007D19490978D5
:101D4000401AC2B22146641C0DF8012016480068F2
:101D5000020E2146641C0DF8012013480068C0F3F0
:101D600007422146641C0DF801200F480088C0F38B
:101D700007222046611CCCB20DF800200A480278E8
:101D80002046611CCCB20DF8002023466A46A521EE
:101D90000020F5F709FB00BF1CBD0000A43E002099
:101DA00094510020A83E0020AC3E0020034800785B
:101DB000012800D170470020FCE70000A43E00206D
:101DC00010B50249AB20F5F719FA10BD254E0300F6
:101DD00010B5024806F0D2FE10BD0000C04A002037
:101DE00010B503460C460AB9072010BD19684A61B0
:101DF000012C01D1012000E0002008610020F4E75F
:101E000038B5134800680090082358221149124839
:101E100000680EF0AAFC04460CB1204638BD0F4AFB
:101E200069460F4806F0B0FE04460CB12046F5E7BF
:101E300001210B4806F01AFF01230A4A19460848F7
:101E400006F06EFE0120084908702046E6E7000013
:101E5000F8A70400D89A0020E8A70400496C040001
:101E6000C04A0020FFFF7F00CC4A00202DE9F0414E
:101E700006460D4617463446207F10B10020BDE8C7
:101E8000F081A76109F05EFC401941F10001C4E94D
:101E90000201206900B125612146002017F086FB70
:101EA000EDE770B504462546002028772946012035
:101EB00017F07CFB70BD10B50446204615F0C2F942
:101EC00010BD000070B5044625460E488068B0B1CC
:101ED000ADB9FCF7B5FA06460A4800680A49086039
:101EE000084840684FF0E021C1F80401002005498E
:101EF00088601EB900BF62B600BF00BF00BF00BF50
:101F000070BD0000C09A002000E100E0F8B5054671
:101F10000C4617462088001DB84201D90C20F8BD98
:101F2000684679DF064600BF304600B1F7E700BFDC
:101F30000320218868542088401C20801920218893
:101F400068542088401C208020884119BDF800007A
:101F500017F06DFB2188084420800020DFE770B572
:101F600004460D4620460CF02BF970BD10B541EC2F
:101F7000100BFBF7A5FA51EC100B10BD2DE9F04149
:101F80002DED028B04460E4617461D46B0EE408AE4
:101F9000B0EE000A86ED000A95ED020A20EE080A6E
:101FA00086ED010A95ED010AF1EE480A20EE200ABD
:101FB00086ED020A95ED020AF1EE480A20EE200AAB
:101FC00086ED030AB0EE000A86ED040A95ED000ADC
:101FD00020EE080A86ED050A95ED010A20EE080AB2
:101FE00086ED060A95ED000AF1EE480A20EE200A79
:101FF00086ED070AB0EE000A86ED080A394630463B
:102000000BF002FC24213046F4F753FA94ED010A58
:1020100020EE080AD5ED020A20EE200AD4ED000ACF
:10202000B0EE001A01EE200AD4ED020A60EE880A32
:1020300095ED011A00EEC10A86ED000A94ED010A41
:10204000F0EE000A20EE200AD4ED000A60EE880AC5
:1020500095ED021A00EEC10AD4ED020A60EE880A7C
:1020600095ED001A00EE810A86ED010A94ED000A52
:1020700020EE080AD5ED010A20EE200AD4ED020A6E
:10208000B0EE001A01EE200AD4ED010A60EE880AD3
:1020900095ED001A00EEC10A86ED020A94ED040ADD
:1020A00020EE080AD5ED020A20EE200AD4ED030A3C
:1020B000B0EE001A01EE200AD4ED050A60EE880A9F
:1020C00095ED011A00EEC10A86ED030A94ED040AAB
:1020D000F0EE000A20EE200AD4ED030A60EE880A32
:1020E00095ED021A00EEC10AD4ED050A60EE880AE9
:1020F00095ED001A00EE810A86ED040A94ED030ABC
:1021000020EE080AD5ED010A20EE200AD4ED050ADA
:10211000B0EE001A01EE200AD4ED040A60EE880A3F
:1021200095ED001A00EEC10A86ED050A94ED070A46
:1021300020EE080AD5ED020A20EE200AD4ED060AA8
:10214000B0EE001A01EE200AD4ED080A60EE880A0B
:1021500095ED011A00EEC10A86ED060A94ED070A14
:10216000F0EE000A20EE200AD4ED060A60EE880A9E
:1021700095ED021A00EEC10AD4ED080A60EE880A55
:1021800095ED001A00EE810A86ED070A94ED060A25
:1021900020EE080AD5ED010A20EE200AD4ED080A47
:1021A000B0EE001A01EE200AD4ED070A60EE880AAC
:1021B00095ED001A00EEC10A86ED080A224639465E
:1021C00030460DF070FFBDEC028BBDE8F08110B51C
:1021D0000446637903F00302217920880BF0ADFFF8
:1021E00010BD10B50446207918B9204600F008F853
:1021F00003E02046FFF7EBFF00BF00BF10BD00006B
:102200002DE9FC41064637884FF00008002244487B
:102210000178384600F084FC7079C0F3800028B95A
:102220000021304612F0CCF9BDE8FC8107F5807141
:1022300088B26B460122072112F070FA054645B1BB
:102240002946384615F00AFF0021304612F0B8F949
:10225000EAE738460AF0ACFA04464FF6FF718C42C2
:102260001BD101980AF0F4F904464FF6FF7084423E
:1022700013D0214638460AF079FA3846FCF7E2FED8
:1022800058B9384615F084FE3846FCF7DBFE20B915
:102290000021304612F094F9C6E74FF6FF708442F1
:1022A00015D112F0D3FB04464FF6FF70844208D1DB
:1022B0000421384615F0D2FE0021304612F080F994
:1022C000B2E7214638460AF051FA4FF0010807F507
:1022D000807188B22246072112F096FA054625B988
:1022E0000121304612F06CF917E0862D07D13846EF
:1022F00015F08EFE0121304612F062F90DE02946FC
:10230000384615F0ABFE0021304612F059F9B8F10D
:10231000000F02D020460AF033FA00BF84E7000025
:10232000554A002010B5034693ED002AB0EE420A4C
:1023300093ED002AF0EE420A91ED002AB0EE421A27
:1023400091ED002AF0EE421A01203CE003EB8004FC
:1023500094ED002AB4EEC02AF1EE10FA05DD03EB8D
:10236000800494ED002AB0EE420A03EB800494ED61
:10237000002AB4EEE02AF1EE10FA05D203EB800455
:1023800094ED002AF0EE420A01EB800494ED002A5D
:10239000B4EEC12AF1EE10FA05DD01EB800494EDF4
:1023A000002AB0EE421A01EB800494ED002AB4EE4C
:1023B000E12AF1EE10FA05D201EB800494ED002A37
:1023C000F0EE421A401C9042C0DB9FED0B2A30EE2B
:1023D000822AB4EEC02AF1EE10FA08D39FED062A45
:1023E00031EE822AB4EEC12AF1EE10FA01D20120B8
:1023F00010BD0020FCE700009A99993E2DE9F041BC
:1024000004460F46154615B90E20BDE8F0810020A0
:10241000286000BF0CB90E20F7E700BF00BF20689E
:1024200008B90E20F1E700BF00BFE088C11700EB3C
:1024300091718910A0EB810109B10720E5E700BF88
:10244000384600F0DDFAC6B2142E01D10520DCE7D3
:102450002079B04201DC0420D7E7E188206806FB40
:10246000010028600020D0E72DE9FC4105468846A0
:102470001646002437880020308095F82D0058B18A
:102480003A463146404600F00FFC044600BF204665
:1024900008B1BDE8FC8100BFA87850B13A4631468A
:1024A0004046FFF733FD044600BF204600B1F0E789
:1024B00000BFE87860B1E97848B23B463246414611
:1024C00007F05DF9044600BF204600B1E1E700BF18
:1024D000686868B1696891F900003B463246414638
:1024E00017F084F8044600BF204600B1D1E700BFD2
:1024F000288900280EDD43460622022105F1080046
:10250000CDE9006717F03EF9044600BF204600B150
:10251000BFE700BF288A00280EDD434607220321BB
:1025200005F11000CDE9006717F02CF9044600BF53
:10253000204600B1ADE700BF288B00280EDD4346E2
:102540001522142105F11800CDE9006717F01AF9DA
:10255000044600BF204600B19BE700BF286A58B17F
:102560003B4632464146286A03F053FB044600BF0F
:10257000204600B18DE700BF686A58B13B4632463D
:102580004146686A0CF07AFD044600BF204600B15F
:102590007FE700BF95F82C0000280BDD3B46324654
:1025A0004146284615F096FE044600BF204600B17D
:1025B0006FE700BF287858B13B463246414628466F
:1025C0000DF059FE044600BF204600B161E700BF90
:1025D00020465EE72DE9F84306468846154600206A
:1025E00000900DB9BDE8F88309236A46414630469C
:1025F00000F02BF80446BDF800003718BDF80000C5
:1026000068B164B12846F3F75FFFA04207D12246C4
:1026100039462846F3F76DFF08B90120E2E70020AC
:10262000E0E7F8B504460E461546002000902B461C
:102630006A463146204600F008F807460FB90020E8
:10264000F8BDBDF800002044FAE7F0B504460D4699
:102650001E4604B10AB90020F0BD002103E0605C11
:10266000401C084481B2481CA84206DA10888842FF
:10267000F5DC481C205CB042F1D1A94201DB00200E
:10268000EAE7881C87B2605C10B1605C401E00E025
:10269000002083B213B1F818A84201DD0020DBE767
:1026A00017801846D8E780F83010704770B5044698
:1026B0000D4605B10CB90E2070BD05F1780003F090
:1026C000C0F908B90720F7E70020A0702C2205F117
:1026D0007801201DF3F7D4FE002084F83000D5F8EF
:1026E000A4006063D5F8A800A0634FF6FF70A4F8BB
:1026F000240404F58260C4F82004002140F22C4038
:10270000C4F82614A4F82A140155207810B9FF2023
:1027100084F8540004F15500C4F810042046FCF776
:10272000B9FB40F21441085304F2144204F155017C
:102730002846FFF799FE064600BF304600B1BBE7CA
:1027400000BF04F231204FF4836108512046FCF7AA
:10275000A1FBA4F81C044FF48360015904F21C424D
:1027600005F13C00FFF780FE064600BF304600B191
:10277000A2E700BF012151200155208B81B24820E2
:102780000153012084F83C000021216450200155B0
:102790006169616404F13C02002104F1540072DFBC
:1027A000064600BF304600B186E700BF012020701A
:1027B000304681E770B504460D462E462088102825
:1027C00004D0112807D026280FD109E02146304631
:1027D00011F00CFA0AE02146304611F082FB05E0C8
:1027E0002146304611F0A2FD00E000BF00BF70BDE1
:1027F00070B504460E46207808B9082070BDA67052
:10280000002140F22C40C4F82614A4F82A140155E3
:10281000A07910B1A078012809D0E07910B1A07892
:10282000012804D0E07970B1A07802280BD1606B48
:1028300030B1012084F82D040820616B884702E044
:10284000002084F82D0431462046FCF7D3FAA0700E
:10285000606BA0B1A078032802D0A07804280ED124
:10286000607960B194F82E0448B9002084F83004EF
:10287000012084F82F040720616B884702E00020C4
:1028800084F82F04182104F13C00F3F712FE012014
:1028900084F83C0004F12C0012F018FA20B194F8EE
:1028A0002C105120015502E001215120015594F8CE
:1028B000240060B104F1280012F008FA20B194F865
:1028C00028105220015502E001215220015500211B
:1028D00050200155A078052824D2DFE800F01F031E
:1028E0000A11180004F13C01204615F0F1FD0546DF
:1028F00019E004F13C01204615F0D2FD054612E036
:1029000004F13C01204615F0F5FD05460BE004F10D
:102910003C01204615F01CFE054604E0002084F82A
:10292000310000E000BF00BFA07898B104F13C0284
:1029300004F15400D4F8201472DF05460DB1284686
:102940005CE794F8301094F8540073DF05460DB13D
:10295000284653E7606B18B194F83100616B8847E3
:1029600000204BE72DE9F041044600BF14B90E20CA
:10297000BDE8F08100BF1C2221461C48F3F780FD12
:102980001B481A490860206860B120687ADF054654
:102990000DB12846ECE7164821680A6802604968CC
:1029A000416005E012487BDF05460DB12846DFE7B0
:1029B000002617E006EB86000E4901EB800700BFFA
:1029C0004FF6FF70388000BF0B4800EB4610786070
:1029D0000A4A0021381DFFF703FA05460DB103200E
:1029E000C6E7761C002EE5D00020C1E79C960020AB
:1029F000224A0020889600206896002095960400C0
:102A000010B50446204600F0A1F808B1204610BDDC
:102A10001420FCE710B50446204600F097F820B1DA
:102A2000214603480DF043FF10BD0020FCE70000E5
:102A3000F895002070B504460D461646204616F05F
:102A400073FE08B9002070BD034951F824003246D6
:102A5000294608F03DF9F6E70496002010B5044633
:102A6000204600F073F820B1214603480DF01FFF07
:102A700010BD0020FCE700000096002010B50446C1
:102A8000204600F063F820B1214603480DF00FFF07
:102A900010BD0020FCE70000FC95002070B5044646
:102AA0000025204600F052F850B1214605480DF0AF
:102AB000FEFE06460EB1022000E00120054600BFE2
:102AC000284670BDF495002070B5044600252046C8
:102AD00000F03CF850B1214605480DF0E8FE0646EE
:102AE0000EB1022000E00120054600BF284670BD5F
:102AF000F095002070B505460C46204616F014FEF1
:102B000050B1284600F022F830B1044901EB8400AE
:102B100029460DF0CCFE70BD0020FCE70496002095
:102B200070B505460C461646204616F0FDFD50B120
:102B3000284600F00BF830B1034901EB840032461F
:102B4000294606F00DFE70BD0496002010B504461F
:102B5000142C01DB002010BD214602480DF0A7FE19
:102B6000F9E70000EC95002010B5044600BF0CB951
:102B70000E2010BD00BF00BF06480078012801D01C
:102B80000820F6E700BF04480168204613F068FFFC
:102B9000EFE70000204A0020144A002001460022EE
:102BA00000BF09B90E20704700BF00BF086808B910
:102BB0000E20F8E700BF00BF486808B90E20F2E712
:102BC00000BF0020064B18600120064B1870064B12
:102BD00008681860054B486818601046E3E7000075
:102BE0001C4A0020204A0020144A0020184A0020D5
:102BF00070B504460D4600BF04B970BD00BF00BFEC
:102C000005B9FAE700BF00BF14480078012800D0DA
:102C1000F3E700BF2E462088112815D0302804D0B5
:102C2000322807D0332814D109E0211D304611F095
:102C300089FA0FE0211D304610F07CFE0AE0211DCC
:102C4000304611F08DF805E0211D304611F03CF9B9
:102C500000E000BF00BF00BFCFE70000204A002017
:102C600070B504460D4600BF0CB90E2070BD00BF04
:102C700000BF0B480078012801D00820F6E700BF0C
:102C80000848006808B90820F0E794F8C80208B1BD
:102C90001120EBE72946204604F020F9E6E7000082
:102CA000204A00201C4A00202DE9FC4105460C4624
:102CB000174620880930B84202D90C20BDE8FC81B3
:102CC00068466DDF064600BF304600B1F6E700BF3C
:102CD0000820218868542088401C20801B202188DF
:102CE00068542088401C208020882844DDF801108A
:102CF0000160BDF8051081802088801D20809DF82E
:102D00000000400818B900202188685402E0012022
:102D1000218868542088401C20800020CEE70000D5
:102D200070B50EF0EBFA044600BF204600B170BD4E
:102D300000BF00BF084D28464FF0030C00DF00BF66
:102D4000044600BF204600B1F1E700BF0EF0F0FAE4
:102D500004462046EBE70000849F0020014600BFA8
:102D600009B90E20704700BF014801600020F9E753
:102D70002C4B002010B54FF0FF3100203DDF044602
:102D800000BF204600B110BD00BFB12100203CDFD4
:102D9000044600BF204600B1F5E700BF0448416982
:102DA0000120884702200EF0D9FF0020EBE7000049
:102DB000689F002010B505480068416900208847D9
:102DC000FFF7D8FF0446204610BD00002C4B002022
:102DD00010B588B0044620216846F3F76AFB03204B
:102DE000ADF8000020788DF802009DF80D0020F06D
:102DF000200020308DF80D009DF80D0020F0080017
:102E000008308DF80D0001208DF810008DF80C00B1
:102E10001720ADF8040001208DF813008DF8120082
:102E20008DF811006088A21D694602F0F3FB08B01E
:102E300010BD000030B585B00546244B0FCB8DE8A2
:102E40000F0000BF15B90E2005B030BD00BF4FF612
:102E5000FF701F498880286848610020087608466E
:102E6000406908B91B4848611948FFF777FF0446D5
:102E700000BF204600B1E7E700BF00BF01208DF88A
:102E800012004FF65960ADF8100000BF104A921CB6
:102E900004A90120A8DF044600BF204600B1D3E703
:102EA00000BF0B49684662DF044600BF204600B100
:102EB000CAE700BF0648FFF78BFF044600BF204665
:102EC00000B1C1E700BF0020BEE700000CA904006C
:102ED000689F0020B18F030070B504460D4600BF07
:102EE00004B970BD00BF2088102806D0112808D072
:102EF00051280AD0532810D10BE0204610F06CFE68
:102F00000CE0204610F0D2FF08E0204611F05CF9FA
:102F100004E0204611F070F800E000BF00BF00BFE1
:102F2000DFE7000070B504460426207B012802D0AC
:102F3000022822D109E006F047F805460DB901261E
:102F400002E0112D00D1062619E0607B142801DC77
:102F5000607B08B905260FE0627B04F10E01124880
:102F6000F3F78EFA607B1049091F8861084615F057
:102F70001DFB054605B9012601E0022600BF00BF82
:102F8000012E0FD0207B314600F058F8054625B1C0
:102F90000648006841690320884704480068416981
:102FA0000220884770BD0000949F00202C4B002019
:102FB00070B505460E4600BF1E48006820B11D488A
:102FC000406808B1012000E0002000B970BD00BFDA
:102FD000184800F10801426828469047044600BF9F
:102FE000082C24D07CB900201349096848760121B7
:102FF000022000F023F80446CCB10F480068416974
:103000000320884713E000200B4909684876062111
:10301000022000F013F8044624B107480068416913
:10302000032088470448006841690220884700BFA0
:10303000CCE70000849F00202C4B0020F0B587B027
:1030400004460D460327002001900290039004904F
:103050000320069020208DF814008DF815408DF87F
:1030600016500E48C088ADF8040002208DF8060006
:103070000020ADF8080006A8039005A804900749B1
:10308000888801A9AEDF064626B9BDF818000328D6
:1030900000D00C26304607B0F0BD0000689F00202D
:1030A00030B1012805D0022804D0032807D102E05E
:1030B00006E005E004E000BF002100BF00E000BF23
:1030C00000BF70472DE9F04104460F46A688304600
:1030D000FFF7E4FC0546012D03D0204600F0C2F8BE
:1030E00018B1204610F0FEFA08E0022D02D0208828
:1030F0001D2803D10021204610F010FABDE8F08110
:103100002DE9F04104460F46A6882088102806D0F5
:10311000112819D019283FD01A284AD118E013F0E5
:1031200039FC304613F0BAFA30B900BF22A2F021C0
:103130000420F3F76FF806E0E07B022803D1314664
:103140002C480DF0C3FB34E0304613F047FC30E070
:10315000207A0509042D01DB012000E00020024651
:10316000314624480C3006F0FBFA032D01DB012028
:1031700000E00020024631461E48083006F0F0FA12
:10318000022D01DB012000E00020024631461948F3
:10319000001D06F0E5FA0CE0207A48B9607AC0F329
:1031A000C0052A46314613480C3006F0D9FA00BF54
:1031B00000BF00BFBDE8F0812E2E5C2E2E5C2E2EAF
:1031C0005C2E2E5C2E2E5C2E2E5C636F6D706F6EEF
:1031D000656E74735C626C655C636F6D6D6F6E5C65
:1031E000626C655F636F6E6E5F73746174652E638E
:1031F00000000000F495002070B504460D462088BC
:10320000102806D0112808D012280ED0502810D12E
:1032100007E0204610F06EFC0CE0204610F02DFE7A
:1032200008E0204611F0B4F804E0204610F04AFC13
:1032300000E000BF00BF70BD70B504460D4600BF82
:103240000748007800B970BD00BF204609F06AF950
:10325000204615F075FB204608F0AEF800BFF2E7F7
:10326000804A002001460888262801D101207047A5
:103270000020FCE710B5002408E0074850F82400BF
:1032800018B1054951F824008047641C03480078B0
:103290008442F2DB10BD0000A8840020C447002057
:1032A00010B5002408E0074850F8240018B105497B
:1032B00051F824008047641C034800788442F2DB04
:1032C00010BD0000B4840020C54700202DE9F04166
:1032D00007460C46207820B1012824D0022829D1A5
:1032E00027E0618804F10E02384600F035F8054603
:1032F00000BF2E4636B100BF10A275213046F2F74E
:1033000089FF00BF00BF384600F02EF9054600BF18
:103310002E4636B100BF09A278213046F2F77AFF77
:1033200000BF00BF06E0A1890A4AA0681268904762
:1033300000E000BF00BFBDE8F08100002E2E5C2E33
:103340002E5C2E2E5C626C655F6366675C686F73D3
:10335000742E6300B841002070B504460E46154631
:1033600000BF0CB90E2070BD00BF26812DB1698849
:10337000A18128886081A988E1813146A0690DF08A
:103380000FFCF0E770B586B004460D461A4B0FCB24
:1033900001AE0FC600BF14B90E2006B070BD00BF4D
:1033A00000BF0DB90E20F8E700BF00BFA86808B93C
:1033B0000E20F2E700BFE11D01A862DF064600BF54
:1033C000304600B1E9E700BFE0798DF81600012032
:1033D000ADF814004FF6FF702081286820616868FE
:1033E0006061002060810021E181A868A06105A8DA
:1033F000FFF7BAFBD1E7000070A6040070B586B0F5
:1034000005460E46344604B10DB906B070BD20899C
:103410004FF6FF71884203D02089A988884200D0E6
:10342000F3E72888112806D0392816D129462046E6
:1034300010F0F8FD12E0A888218988420CD120699B
:1034400050B102208DF804004FF6FF70208101A9D1
:1034500020462269904700BF00E000BF00BF00BFC8
:10346000D3E770B586B005460C46142101A8F3F7E2
:1034700020F804F10E06207800283AD1A08801280F
:1034800037D1A079E979884233D1002022E000EBDE
:10349000C00136F81110022902D0032917D107E024
:1034A00000EBC00106EB41010A89ADF816200FE0E0
:1034B00000EBC00106EB41010989ADF8121000EBE9
:1034C000C00106EB41014A89ADF8142000E000BFBD
:1034D00000BF401C217A8142D9D8286948B1608850
:1034E000ADF8060000208DF8040001A928462A69DD
:1034F000904706B070BD000070B588B004460E4617
:10350000154600BF14B90E2008B070BD00BF2021C1
:103510006846F2F7CEFFF42D01DD0720F4E720899D
:103520004FF6FF71884201D10820EDE701208DF8A8
:1035300000000C4802900394E189ADF81210ADF838
:1035400016500021ADF81410069602208DF81000D8
:1035500001218DF8111022896946A0690DF04AFBFE
:10356000D2E7000061AF030010B5044600BF0CB9FC
:103570000E2010BD00BF20894FF6FF71884201D098
:10358000A08908B90820F4E70121204601F0F4FFE2
:10359000EFE72DE9F04186B00446884617461D4600
:1035A00000BF1CB90E2006B0BDE8F08100BF01AA23
:1035B00029466069FEF722FF064600BF304600B18B
:1035C000F1E700BF4FF6FF70854201D0019808B9BE
:1035D0000520E8E70198007808B90820E3E7388873
:1035E000F42801DD0720DEE700200290039004901C
:1035F0000590A088ADF80800CDF81480049701204C
:103600008DF80A0002A92846AEDFCCE770B58EB06F
:1036100004460E463E4B0FCB09AD0FC500BF14B993
:103620000E200EB070BD00BF00BF0EB90E20F8E72F
:1036300000BF3068A061214609A862DF054600BFCF
:10364000284600B1EDE700BF20788DF83600012054
:10365000ADF83400A21C0DA9A8DF054600BF28461E
:1036600000B1DEE700BF202101A8F2F722FF02200F
:10367000ADF8040020788DF80600F420ADF80800BD
:103680000120ADF80A008DF810009DF8110020F01F
:10369000080008308DF811009DF8110020F004009A
:1036A000001D8DF8110001208DF815008DF8160011
:1036B000608804F10C0201A901F0ACFF05460DB1D0
:1036C0002846AEE7202101A8F2F7F3FE0320ADF86B
:1036D000040020788DF80600F420ADF808000120E1
:1036E000ADF80A008DF810009DF8110020F01000D0
:1036F00010308DF8110001208DF815008DF816009E
:103700008DF817006088221D01A901F083FF88E76A
:1037100080A6040070B504460D4605B104B970BD1D
:103720002E462088102804D0502807D057280FD1C3
:1037300009E02146304610F015FA0AE021463046ED
:1037400010F052FE05E02146304610F087FC00E004
:1037500000BF00BF00BFE2E710B5002408E0074843
:1037600050F8240018B1054951F824008047641C22
:10377000034800788442F2DB10BD00001082002074
:103780008A41002010B5002408E0074850F82400C2
:1037900018B1054951F824008047641C034800789B
:1037A0008442F2DB10BD0000508200208B410020DB
:1037B00070B50446204615F034FF0546C5F34000B9
:1037C00070BD70B50446204615F02BFF054605F088
:1037D000010070BD38B50EF07DFD044600BF2546E2
:1037E0003DB100BF15A240F2A1112846F2F712FD2B
:1037F00000BF00BF00200090694601200EF06AFC67
:10380000044600BF25463DB100BF0CA240F2A711FF
:103810002846F2F7FFFC00BF00BF68460EF0B8FC78
:10382000044600BF25463DB100BF04A240F2AB11E3
:103830002846F2F7EFFC00BF00BF38BD2E2E5C2EED
:103840002E5C2E2E5C626C655F6366675C686F73CE
:10385000742E630010B5002406F022F8401C00B955
:10386000641E70210848F2F724FE074890F86E00A5
:1038700040F08000044981F86E00601C10B94FF0E0
:10388000FF3010BD0020FCE74C75002070B50446E9
:103890000CB9002070BD002509E00F4850F8250044
:1038A000A04203D100F034FB2046F3E76D1C0C2D41
:1038B000F3DB00250BE0084850F8250030B9064836
:1038C00040F8254000F024FB2046E3E76D1C0C2D5A
:1038D000F1DB0020DEE700004C75002070B50546E6
:1038E00015B94FF0FF3070BD00240DE0094850F8C5
:1038F0002400A84207D10020064941F8240000F026
:1039000007FB0020EFE7641C0C2CEFDB6FF00100DD
:10391000E9E700004C75002010B5002006F0A0F883
:103920000446601C10B94FF0FF3010BD012006F0B6
:1039300097F80446601C10B94FF0FF30F5E770218E
:103940000648F2F7B6FD054890F86E0040F080009A
:10395000024981F86E000020E7E700004C75002066
:1039600070B504460D46164632462946204606F0F6
:10397000CBF870BD10B50446204606F0E3F810BD44
:1039800010B5024602B111B94FF0FF3010BD002052
:1039900067E100EB400303EBC00313441B7A00EB29
:1039A000400404EBC0040C44247AA34206DD00EB7F
:1039B000400303EBC00313441B7A05E000EB400314
:1039C00003EBC0030B441B7A00EB400404EBC00480
:1039D0001444237200EB400303EBC00313445B79F0
:1039E00000EB400404EBC0040C446479A34206DD00
:1039F00000EB400303EBC00313445B7905E000EBED
:103A0000400303EBC0030B445B7900EB400404EB81
:103A1000C0041444637100EB400303EBC003D35CA8
:103A200000EB400404EBC0040C5DA34205DD00EB99
:103A3000400303EBC003D35C04E000EB400303EB63
:103A4000C003CB5C00EB400404EBC004135500EB57
:103A5000400303EBC00313449B7800EB400404EBEA
:103A6000C0040C44A478A34206DD00EB400303EB42
:103A7000C00313449B7805E000EB400303EBC00355
:103A80000B449B7800EB400404EBC0041444A37087
:103A900000EB400303EBC00313445B7A00EB4004EC
:103AA00004EBC0040C44647AA34206DD00EB40033F
:103AB00003EBC00313445B7A05E000EB400303EB28
:103AC000C0030B445B7A00EB400404EBC0041444D5
:103AD000637200EB400303EBC00313449B7900EBDC
:103AE000400404EBC0040C44A479A34206DD00EBBF
:103AF000400303EBC00313449B7905E000EB400354
:103B000003EBC0030B449B7900EB400404EBC004BF
:103B10001444A37100EB400303EBC00313445B7830
:103B200000EB400404EBC0040C446478A34206DDBF
:103B300000EB400303EBC00313445B7805E000EBAC
:103B4000400303EBC0030B445B7800EB400404EB41
:103B5000C0041444637000EB400303EBC003134440
:103B60009B7A00EB400404EBC0040C44A47AA3420B
:103B700006DD00EB400303EBC00313449B7A05E032
:103B800000EB400303EBC0030B449B7A00EB4004C3
:103B900004EBC0041444A37200EB400303EBC00326
:103BA0001344DB7900EB400404EBC0040C44E479DB
:103BB000A34206DD00EB400303EBC0031344DB79B3
:103BC00005E000EB400303EBC0030B44DB7900EBA3
:103BD000400404EBC0041444E37100EB400303EB26
:103BE000C0031344DB7800EB400404EBC0040C4436
:103BF000E478A34206DD00EB400303EBC00313446B
:103C0000DB7805E000EB400303EBC0030B44DB78FB
:103C100000EB400404EBC0041444E37000EB4003E9
:103C200003EBC00313441B7900EB400404EBC00416
:103C30000C442479A34206DD00EB400303EBC003F0
:103C400013441B7905E000EB400303EBC0030B4476
:103C50001B7900EB400404EBC00414442371431CA3
:103C6000D8B20228FFF695AE00208FE6F0B50746E1
:103C70000E4600210EB1022F03DB41F0C0010846C1
:103C8000F0BD326873686C4C04F10B0517B1012F5D
:103C900076D163E0107A94F808C0604503DD41F006
:103CA000C0000146ECE7507994F805C0604503DD9B
:103CB00041F0C0000146E3E7107894F800C0604589
:103CC00003DD41F0C0000146DAE7907894F802C0C5
:103CD000604503DD41F0C0000146D1E7507A94F819
:103CE00009C0604503DD41F0C0000146C8E7907996
:103CF00094F806C0604503DD41F0C0000146BFE70F
:103D0000507894F801C0604503DD41F0C0000146E1
:103D1000B6E7907A94F80AC0604503DD41F0C00030
:103D20000146ADE7D07994F807C0604503DD41F066
:103D3000C0000146A4E7D07894F803C0604503DDD5
:103D400041F0C00001469BE7107994F804C060453B
:103D500003DD41F0C000014692E765E0187A95F86E
:103D600008C0604503DD41F0C000014688E758798E
:103D700095F805C0604504DD41F0C00001467FE7CD
:103D800051E0187895F800C0604503DD41F0C000AF
:103D9000014675E7987895F802C0604503DD41F06B
:103DA000C00001466CE7587A95F809C0604503DD0C
:103DB00041F0C000014663E7987995F806C0604578
:103DC00003DD41F0C00001465AE7587895F801C07C
:103DD000604503DD41F0C000014651E7987A95F84F
:103DE0000AC0604503DD41F0C000014648E7D879CC
:103DF00095F807C0604503DD41F0C00001463FE78C
:103E0000D87895F803C0604503DD41F0C000014655
:103E100036E7187995F804C0604503DD41F0C0002D
:103E200001462DE700E000BF00BF0348583890F876
:103E30006E10084624E70000A475002000210B4AFC
:103E400082F86E10411C39B9114691F86E1041F09C
:103E5000800182F86E1007E0044A82F86E00114675
:103E600091F86E1082F86E10704700004C750020BB
:103E700002460B460BB1022A02DB4FF0FF307047BF
:103E800000210BE0114800EBC1004068984204D1CA
:103E90000E4800F831200020F1E7491C0529F1DB2C
:103EA00000210EE0094800EBC100406840B9074816
:103EB00000EBC1004360054800F831200020DEE738
:103EC000491C0529EEDB4FF0FF30D8E77C75002058
:103ED00070B50646012515E0002410E00B4810F8E7
:103EE0003400A8420AD1094800EBC400406828B158
:103EF000064800EBC400416830468847641C052C26
:103F0000ECDB6D1E002DE7DA70BD00007C75002033
:103F100070B5FF25002400BF0CE004EB440000EB6B
:103F2000C4012E4808440021016041600181817272
:103F3000601CC4B2022CF0DB002414E0274858387F
:103F400050F8240068B12548583850F8240001681A
:103F50002248FFF715FD0546681C10B94FF0FF30E9
:103F600070BD601CC4B20C2CE8DB1C49002005F0BD
:103F7000B1FD0546681C10B94FF0FF30F0E7174956
:103F80000B31012005F0A6FD0546681C10B94FF065
:103F9000FF30E5E7124806F0C5FA0546681C10B97F
:103FA0004FF0FF30DCE70F4806F0C8FA0546681C02
:103FB00010B94FF0FF30D3E706F0CCFA05465DB9F3
:103FC00000200649583981F86E00084690F86E00C6
:103FD00040F0400081F86E000020C1E7A475002089
:103FE0003D3E0300D13E030010B504A11220F3F7BB
:103FF000ADFE10B90748F6F773F910BD6273705F34
:104000006164635F696E69745F6572726F720D0AD5
:1040100000000000E93F030010B504A11720F3F7EA
:1040200095FE10B90748F6F75BF910BD6273705F33
:1040300070776D5F696E69745F6572726F720D0A79
:10404000000000001940030010B504A11920F3F787
:104050007DFE10B90748F6F743F910BD6273705F33
:104060007274635F636F6E6669675F6572726F72A9
:104070000D0A00004940030010B504A11920F3F710
:1040800065FE10B90748F6F72BF910BD6273705F33
:104090007274635F696E69745F6572726F720D0A24
:1040A000000000007940030010B504A11320F3F7CD
:1040B0004DFE10B90748F6F713F910BD6273705F33
:1040C000737069305F696E69745F6572726F720DCB
:1040D0000A000000A940030010B504A11820F3F75E
:1040E00035FE10B90748F6F7FBF810BD6273705F34
:1040F0007764745F696E69745F6572726F720D0ABE
:1041000000000000D940030030B503460C460020F3
:104110001FE09FED110A02EB800181ED000A0021F2
:1041200014E002EB800595ED000A01EB800503EB3E
:104130008505D5ED000A04EB810595ED001A00EE2A
:10414000810A02EB800585ED000A491C0429E8DBA1
:10415000401C0928DDDB30BD0000000030B5A1B0F7
:1041600005460C4694ED140A8DED010A94ED180AEB
:104170008DED020A94ED190A8DED030A94ED1A0AE9
:104180008DED040A94ED380A8DED050A94ED3C0A94
:104190008DED060A94ED3D0A8DED070A94ED3E0A79
:1041A0008DED080A94ED410A8DED090A94ED450A5A
:1041B0008DED0A0A94ED460A8DED0B0A94ED470A3F
:1041C0008DED0C0A94ED4A0A8DED0D0A94ED4E0A20
:1041D0008DED0E0A94ED4F0A8DED0F0A94ED500A05
:1041E0008DED100A002012E001A901EB001101EB96
:1041F000800191ED000ADFEDFE0A30EE200A01A9F0
:1042000001EB001101EB800181ED000A401C042844
:10421000EADB11A901A80AF06DFF94ED020ADDEDB9
:10422000110A20EE200AD4ED060A9DED151A00EEC3
:10423000810AD4ED070A9DED191A00EE810AD4ED2A
:10424000080A9DED1D1A00EE810A85ED000A94ED25
:10425000020ADDED120A20EE200AD4ED060A9DEDD9
:10426000161A00EE810AD4ED070A9DED1A1A00EE27
:10427000810AD4ED080A9DED1E1A00EE810A85ED33
:10428000010A94ED020ADDED130A20EE200AD4EDB6
:10429000060A9DED171A00EE810AD4ED070A9DED7E
:1042A0001B1A00EE810AD4ED080A9DED1F1A00EEDC
:1042B000810A85ED020A94ED020ADDED140A20EE72
:1042C000200AD4ED060A9DED181A00EE810AD4EDFD
:1042D000070A9DED1C1A00EE810AD4ED080A9DED37
:1042E000201A00EE810A85ED030A94ED0B0ADDED3C
:1042F000110A20EE200AD4ED0F0A9DED151A00EEEA
:10430000810AD4ED100A9DED191A00EE810AD4ED50
:10431000110A9DED1D1A00EE810A85ED040A94ED47
:104320000B0ADDED120A20EE200AD4ED0F0A9DEDF6
:10433000161A00EE810AD4ED100A9DED1A1A00EE4D
:10434000810AD4ED110A9DED1E1A00EE810A85ED59
:10435000050A94ED0B0ADDED130A20EE200AD4EDD8
:104360000F0A9DED171A00EE810AD4ED100A9DED9B
:104370001B1A00EE810AD4ED110A9DED1F1A00EE02
:10438000810A85ED060A94ED0B0ADDED140A20EE94
:10439000200AD4ED0F0A9DED181A00EE810AD4ED23
:1043A000100A9DED1C1A00EE810AD4ED110A9DED54
:1043B000201A00EE810A85ED070A94ED140ADDED5E
:1043C000110A20EE200AD4ED180A9DED151A00EE10
:1043D000810AD4ED190A9DED191A00EE810AD4ED77
:1043E0001A0A9DED1D1A00EE810A85ED080A94ED6A
:1043F000140ADDED120A20EE200AD4ED180A9DED14
:10440000161A00EE810AD4ED190A9DED1A1A00EE73
:10441000810AD4ED1A0A9DED1E1A00EE810A85ED7F
:10442000090A94ED140ADDED130A20EE200AD4EDFA
:10443000180A9DED171A00EE810AD4ED190A9DEDB8
:104440001B1A00EE810AD4ED1A0A9DED1F1A00EE28
:10445000810A85ED0A0A94ED140ADDED140A20EEB6
:10446000200AD4ED180A9DED181A00EE810AD4ED49
:10447000190A9DED1C1A00EE810AD4ED1A0A9DED71
:10448000201A00EE810A85ED0B0A94ED1D0ADDED80
:10449000110A20EE200AD4ED210A9DED151A00EE36
:1044A000810AD4ED220A9DED191A00EE810AD4ED9D
:1044B000230A9DED1D1A00EE810A85ED0C0A94ED8C
:1044C0001D0ADDED120A20EE200AD4ED210A9DED31
:1044D000161A00EE810AD4ED220A9DED1A1A00EE9A
:1044E000810AD4ED230A9DED1E1A00EE810A85EDA6
:1044F0000D0A94ED1D0ADDED130A20EE200AD4ED1D
:10450000210A9DED171A00EE810AD4ED220A9DEDD5
:104510001B1A00EE810AD4ED230A9DED1F1A00EE4E
:10452000810A85ED0E0A94ED1D0ADDED140A20EED8
:10453000200AD4ED210A9DED181A00EE810AD4ED6F
:10454000220A9DED1C1A00EE810AD4ED230A9DED8E
:10455000201A00EE810A85ED0F0A94ED260ADDEDA2
:10456000110A20EE200AD4ED2A0A9DED151A00EE5C
:10457000810AD4ED2B0A9DED191A00EE810AD4EDC3
:104580002C0A9DED1D1A00EE810A85ED100A94EDAE
:10459000260ADDED120A20EE200AD4ED2A0A9DED4E
:1045A000161A00EE810AD4ED2B0A9DED1A1A00EEC0
:1045B000810AD4ED2C0A9DED1E1A00EE810A85EDCC
:1045C000110A94ED260ADDED130A20EE200AD4ED3F
:1045D0002A0A9DED171A00EE810AD4ED2B0A9DEDF3
:1045E0001B1A00EE810AD4ED2C0A9DED1F1A01E082
:1045F000BE37863500EE810A85ED120A94ED260A53
:10460000DDED140A20EE200AD4ED2A0A9DED181AD9
:1046100000EE810AD4ED2B0A9DED1C1A00EE810AF2
:10462000D4ED2C0A9DED201A00EE810A85ED130AC7
:1046300094ED2F0ADDED110A20EE200AD4ED330AA5
:104640009DED151A00EE810AD4ED340A9DED191A7C
:1046500000EE810AD4ED350A9DED1D1A00EE810AA7
:1046600085ED140A94ED2F0ADDED120A20EE200AE2
:10467000D4ED330A9DED161A00EE810AD4ED340A0A
:104680009DED1A1A00EE810AD4ED350A9DED1E1A31
:1046900000EE810A85ED150A94ED2F0ADDED130A6F
:1046A00020EE200AD4ED330A9DED171A00EE810AA0
:1046B000D4ED340A9DED1B1A00EE810AD4ED350AC3
:1046C0009DED1F1A00EE810A85ED160A94ED2F0A62
:1046D000DDED140A20EE200AD4ED330A9DED181A00
:1046E00000EE810AD4ED340A9DED1C1A00EE810A19
:1046F000D4ED350A9DED201A00EE810A85ED170AEA
:1047000094ED380ADDED110A20EE200AD4ED3C0AC2
:104710009DED151A00EE810AD4ED3D0A9DED191AA2
:1047200000EE810AD4ED3E0A9DED1D1A00EE810ACD
:1047300085ED180A94ED380ADDED120A20EE200A04
:10474000D4ED3C0A9DED161A00EE810AD4ED3D0A27
:104750009DED1A1A00EE810AD4ED3E0A9DED1E1A57
:1047600000EE810A85ED190A94ED380ADDED130A91
:1047700020EE200AD4ED3C0A9DED171A00EE810AC6
:10478000D4ED3D0A9DED1B1A00EE810AD4ED3E0AE0
:104790009DED1F1A00EE810A85ED1A0A94ED380A84
:1047A000DDED140A20EE200AD4ED3C0A9DED181A26
:1047B00000EE810AD4ED3D0A9DED1C1A00EE810A3F
:1047C000D4ED3E0A9DED201A00EE810A85ED1B0A0C
:1047D00094ED410ADDED110A20EE200AD4ED450AE0
:1047E0009DED151A00EE810AD4ED460A9DED191AC9
:1047F00000EE810AD4ED470A9DED1D1A00EE810AF4
:1048000085ED1C0A94ED410ADDED120A20EE200A26
:10481000D4ED450A9DED161A00EE810AD4ED460A44
:104820009DED1A1A00EE810AD4ED470A9DED1E1A7D
:1048300000EE810A85ED1D0A94ED410ADDED130AB3
:1048400020EE200AD4ED450A9DED171A00EE810AEC
:10485000D4ED460A9DED1B1A00EE810AD4ED470AFD
:104860009DED1F1A00EE810A85ED1E0A94ED410AA6
:10487000DDED140A20EE200AD4ED450A9DED181A4C
:1048800000EE810AD4ED460A9DED1C1A00EE810A65
:10489000D4ED470A9DED201A00EE810A85ED1F0A2E
:1048A00094ED4A0ADDED110A20EE200AD4ED4E0AFD
:1048B0009DED151A00EE810AD4ED4F0A9DED191AEF
:1048C00000EE810AD4ED500A9DED1D1A00EE810A1A
:1048D00085ED200A94ED4A0ADDED120A20EE200A49
:1048E000D4ED4E0A9DED161A00EE810AD4ED4F0A62
:1048F0009DED1A1A00EE810AD4ED500A9DED1E1AA4
:1049000000EE810A85ED210A94ED4A0ADDED130AD5
:1049100020EE200AD4ED4E0A9DED171A00EE810A12
:10492000D4ED4F0A9DED1B1A00EE810AD4ED500A1A
:104930009DED1F1A00EE810A85ED220A94ED4A0AC8
:10494000DDED140A20EE200AD4ED4E0A9DED181A72
:1049500000EE810AD4ED4F0A9DED1C1A00EE810A8B
:10496000D4ED500A9DED201A00EE810A85ED230A50
:1049700021B030BD30B502460B46002046E0002194
:1049800041E003EB001494ED000A01F1120402EB84
:104990008404D4ED000A20EE200A012404EB8004F4
:1049A00003EB8404D4ED000A01F1360402EB840425
:1049B00094ED001A00EE810A022404EB800403EB5C
:1049C0008404D4ED000A01F13F0402EB840494ED69
:1049D000001A00EE810A032404EB800403EB840434
:1049E000D4ED000A01F1480402EB840494ED001AAE
:1049F00000EE810A00EBC0040C44104D05EB84046A
:104A000084ED000A491C0929BBDB401C0928B6DBE0
:104A100000200FE002EB800191ED000A074901EB55
:104A20008001D1ED000A30EE600A02EB800181EDD9
:104A3000000A401C5128EDDB30BD0000049200202C
:104A400010B502460023002003E032F81040234452
:104A5000401C8842F9DBB3FBF1F080B210BD024686
:104A60008A4201DC881A70474FF6FF70801A401C9A
:104A70000844F8E77CB50446204607F099FE054651
:104A800000236A4609210FF03DFF052805D10122C8
:104A9000024801782046FEF743F87CBD3C4A0020DE
:104AA0007CB504460E460020019042F6A620ADF8E3
:104AB000040001208DF806000748006800906A464F
:104AC00001A92046A0DF05462DB90122034801783F
:104AD0002046FEF725F87CBD6CA504003D4A002069
:104AE00038B5044600200090FBF7AAFC0090012393
:104AF0006A46A3210020F2F757FC38BD38B50446BA
:104B0000254600200090686800788DF800006868ED
:104B100040788DF80100686840786968097800EB92
:104B20000120124908800846028811A10020F6F7EA
:104B3000C3F802236A46AC210020F2F711FE0121DE
:104B40001648F5F757FBF7F703FB15490860F4F72C
:104B500061F8142804DD13490220F4F787FD03E00F
:104B600011490220F4F782FD38BD0000383F0020D3
:104B70003D3D3D3D3D3D3D3E63625F424C455F42B4
:104B80004C494E4B5F4C45442C646973706C6179A1
:104B900074696D653A25640A0000000079FF02001F
:104BA0003C3F0020007F00FF00106FFF10B504465F
:104BB00001231A4603A10020F6F77EF801200849D8
:104BC000087010BD63625F424C455F436C69656E5F
:104BD000745F4552523A25642C25640A0000000097
:104BE0004040002070B50446254606A10020F6F797
:104BF00063F8FCF7FBFE2B7AA72100206A68F2F726
:104C0000AFFD70BD212121212121212163625F425D
:104C10004C455F436C69656E745F525F4348415217
:104C200047450A0070B5054616A10020F6F744F87E
:104C30002C461B480079002811DD6068007818B9FF
:104C400001201849087070BD60680078012817D1EC
:104C50000123A62100206268F2F782FD10E0012303
:104C6000114AA6211148F2F79FFB01201049086064
:104C700001211048F5F7BEFA0FA10020F6F71CF845
:104C800000BFE0E73E3E3E3E3E3E3E3E3E3E424CA4
:104C9000455F436C69656E745F525F4446550A0018
:104CA00094510020E83E0020113F0020EC3E0020FF
:104CB000E43E00207D1003003E3E3E3E3E3E3E3E32
:104CC0003E3E4446552073746172742E2E2E2E0A79
:104CD0000000000070B50446254668680078144955
:104CE000C8700846C07890B1002008711148FEF7DE
:104CF000CDFD0F48C078012802D1F4F765F909E02D
:104D00000B48C078022805D1F4F764F902E009489D
:104D1000FEF7E4FD0123064AD21CA2210020F2F78F
:104D20001FFD0348C27804A10020F5F7C5FF70BD40
:104D3000C03E0020D0A104003E3E3E3E3E3E3E3EF0
:104D40003E3E63625F424C455F436C69656E745FD3
:104D5000525F47414D454D4F44453A25640D0A0089
:104D600070B504462546686800780B490870084607
:104D70000078012806D10020084908800848FEF77D
:104D800085FD02E00648FEF7A9FD0123024AA521A0
:104D90000020F2F7E5FC70BDB43E0020B23E0020DA
:104DA000B0A1040070B505462C4660684078616883
:104DB000097840EA012617480079D8B16068807800
:104DC000012803D13046F4F785FE1DE06068807845
:104DD00048B93046F4F77EFE237AA42100206268A9
:104DE000F2F7BEFC10E0237AA42100206268F2F7FB
:104DF000B7FC09E060688078022802D0606880789B
:104E000010B93046F4F766FE324603A10020F5F7EC
:104E100053FF70BD945100204D542052554E3A25F9
:104E200064200A0008B50446A146D9F804000078B9
:104E3000009001236A46AB210020F2F791FC4FF469
:104E4000FA7505B90EE000BF4FF47A7606B905E0B1
:104E5000134F4FEA86184046B84700BF681E051E2C
:104E6000F2D100BF00BF00BF00BF00BF00BFBFF353
:104E70004F8F00BF00BF00BF0A48006800F4E06029
:104E800009490843001D0749086000BF00BF00BF73
:104E9000BFF34F8F00BF00BF00BF00BF00BFFDE7E3
:104EA00001A204000CED00E00000FA0570B5054613
:104EB0002C466068067836B1012E0ED0022E17D02F
:104EC000032E26D11BE014480079012802D1FBF7FC
:104ED00081FE01E0FAF7CAFE1CE00F4800790128C4
:104EE00003D11420FBF75CFE01E0FAF781FC11E02E
:104EF000FCF75CFF10B92046FAF796FD0AE0237A2A
:104F0000A12100206268F2F74FFA2046FAF734FD3B
:104F100000E000BF00BF70BD9451002010B50446F2
:104F20000E48007800B910BD0D4800880D49098869
:104F3000884210DA0A480088401C80B2084908807C
:104F400008490988884202DB0020044908700448A7
:104F50000088FAF7A9FD00BFE5E70000193E002030
:104F60001A3E00201C3E002038B5044625462B7A08
:104F7000A72100206A68F2F717FA287A009068687B
:104F80004378027802A10020F5F796FE38BD0000B4
:104F900063625F424C455F486F73745F525F434882
:104FA000415247453A25642C25642C25640A0000AB
:104FB00001464A681278034B1A704A685278024BCD
:104FC0001A707047C53F0020C63F002038B5044620
:104FD00000200090254668680078009001236A460A
:104FE000A6210020F2F7E0F938BD70B50446254649
:104FF0002B7AAD2100206A68F2F7D6F970BD000067
:1050000070B505462C4660680078012818D10D4817
:105010000078012811D160684078000661688978BD
:1050200040EA01406168C97840EA01206168097975
:10503000084305490860FCF751FE03200349087046
:1050400070BD0000A43E0020AC3E0020B03E002019
:105050002DE9F041064634466068077817B1012F04
:1050600067D12BE0002006E000F141016268525C4C
:1050700032490A54401C0628F6DB47256068405D2B
:105080000106681C6268105C41EA0041A81C105CC3
:1050900041EA0020E91C515C084328493239C862C2
:1050A000681D6168095C281D6268105C41EA002186
:1050B000224832380186FAF7D9FD3BE06068407833
:1050C0001F490870606880781E4908706068C07861
:1050D00000066168097940EA01406168497940EA5F
:1050E0000120616889790843174908606068C079C0
:1050F00000066168097A40EA01406168497A40EA3D
:1051000001216068807A01430C4832388161207A3D
:10511000192808DB6068807D6168497D00EB01200B
:1051200000B20A490880002009490870FAF760FBBC
:1051300000E000BF00BFBDE8F0810000C6510020C4
:105140004C3E00204D3E0020503E0020543E0020AA
:105150007C3E002070B50446254668680078064904
:10516000087068684078054908700548007908B9F2
:10517000FAF786FA70BD0000C53F0020C63F002048
:105180009451002010B5044600210348F5F732F889
:1051900001200249087010BD7D100300EA3E002086
:1051A00010B502A10020F5F787FD10BD3D3D3D3D46
:1051B0003D3D3D3E63625F486F73745F436F6E6E4B
:1051C0006563740A0000000010B5044600210E203B
:1051D0000CF0FBFBF5F7B2F910BD10B50446F5F77E
:1051E0008DF910BD10B507A10020F5F765FD0C483D
:1051F000007928B1F3EE0E0AB3EE0E0A13F016FB97
:1052000010BD00003D3D3D3D3D3D3D3E63625F5371
:105210006C6176655F436F6E6E6563740A000000B3
:10522000945100202DE9FF47804645464FF0000984
:105230000024FAF705F9012801D1BDE8FF873548B8
:10524000007900B9F9E7002405E06868005D02A96B
:105250000855601CC4B2062CF7DB6868807900062C
:105260006968C97940EA01406968097A40EA012021
:105270006968497A40EA01066868C07A6968897A8B
:1052800040EA012733202449088000240BE021480C
:105290003230005D02A9095D884202D04FF0010959
:1052A00003E0601CC4B2062CF1DB00BF1948C06AE1
:1052B000B04206D11748008EB84202D1B9F1000FB2
:1052C00023D0144890F82800CDE900091148038E36
:1052D00012A1C26A0020F5F7EFFC0E48C6620786ED
:1052E00000240DE002A8015D0A4832300155C4F1E6
:1052F00005011148415C0748401D0155601CC4B2BE
:10530000062CEFDB01200D490870FAF78DF800BF7D
:1053100093E7000094510020843F00206D466C61AB
:10532000736820636F6E6669673A25642025642080
:1053300025642025640A0A007D3F0020863F002066
:105340002DE9FF4781464D464FF000080024FAF74B
:1053500077F8012801D1BDE8FF874148007900B105
:10536000F9E7002405E06868005D02A90855601CA3
:10537000C4B2062CF7DB6868807900066968C979D1
:1053800040EA01406968097A40EA01206968497A7F
:1053900040EA01066868C07A6968897A40EA0127AC
:1053A000304A16211320F6F7F5FF002404E002200E
:1053B000F6F752FF601CC4B20A2CF8DB294A13210D
:1053C0001620F6F7E7FF00240BE02548401D005D9E
:1053D00002A9095D884202D04FF0010803E0601C79
:1053E000C4B2062CF1DB00BF1D48C06AB04206D132
:1053F0001B48008EB84202D1B8F1000F2BD03B46BB
:10540000324619A10020CDF80080F5F755FC14486C
:1054100090F82800CDE900081148038E19A1C26A4E
:105420000020F5F749FC0E48C662078600240DE00F
:10543000C4F105011B48415C09483230015502A8FE
:10544000015D0748401D0155601CC4B2062CEFDB0E
:10545000012015490870F9F7E7FF00BF7BE700005E
:105460009451002090D00300686F737420636F6EB6
:105470006669673A25642025642025642025640A2E
:10548000000000006D466C6173682E6D436C6965A9
:105490006E743A25642025642025642025640A0A58
:1054A000000000007D3F0020863F002010B504462C
:1054B000F1F7E4FB10BD10B50446F1F7E9FB10BDB0
:1054C00010B5F2F777FB254908600846006890F8A8
:1054D0002000032841D00320096881F820009FEDB7
:1054E000200A1E48006880ED050A9FED1E0A1B4831
:1054F000006880ED070A9FED1B0A1848006880EDE0
:10550000060AB7EE000A1548006880ED030A9FED11
:10551000150A1248006880ED040A9FED120A0F4830
:10552000006880ED010A9FED0F0A0C48006880EDCD
:10553000000A00200949096881F821009FED090A45
:105540000648006880ED020A01200449096881F8D4
:1055500023000249096881F8220010BD4440002060
:105560000000C84200000000024909680144014AE5
:10557000116070479040002070B58AB004460D4617
:105580002E46202102A8F0F794FFF0B28DF8040017
:10559000300A8DF8050001208DF808000D480490B0
:1055A0000594A189ADF81A100221ADF81E10002152
:1055B000ADF81C1001A9089101208DF818000121F7
:1055C0008DF81910228902A9A0690BF013FB0AB00B
:1055D00070BD000061AF030001468879012809D140
:1055E0000879012806D1488842F60212904201D17A
:1055F000012070470020FCE70146024850F82100D6
:1056000070470000B099002001460148405670479D
:10561000E099002070B590B006460C461546A0787B
:1056200018B901208DF80E0002E0A0788DF80E0068
:105630002088ADF80C0000200290607C02A912F0D6
:10564000D9FFA07C0DF1090112F0D4FFE07B08B175
:10565000012000E000209DF80A1060F3C3018DF8DE
:105660000A10207C08B1012000E000209DF80A10FB
:1056700060F304118DF80A10207B08B1012000E0CE
:1056800000209DF80A1060F300018DF80A10207DBB
:1056900008B1022000E001209DF80A1060F34201E9
:1056A0008DF80A101C2109A8F0F703FF607BC0F3F6
:1056B000001018B9607BC0F34010F8B100200090D2
:1056C000E07C0DF1010112F095FF00BF9DF8000094
:1056D00020F00F00401C8DF800009DF8000020F025
:1056E000F00010308DF8000000BF9DF8020020F09F
:1056F0000600801C8DF80200CDF838D0607B8DF854
:105700002400A07B8DF82500142104A8F0F7D1FE19
:1057100003A8049002A80590A088ADF81C00A0681A
:1057200020B1E088ADF81800A0680890A0690028B2
:1057300049D000200190A0690088ADF82C00A06934
:105740004088ADF82E00A06940680A9001A80D902D
:10575000A169087B01A912F04DFFA169487B0DF1F9
:10576000050112F047FFA069807A08B1012000E02E
:1057700000209DF8061060F3C3018DF80610A069A3
:10578000C07A08B1012000E000209DF8061060F307
:1057900004118DF80610A069007A08B1012000E01C
:1057A00000209DF8061060F300018DF80610A06936
:1057B000807B08B1022000E001209DF8061060F314
:1057C00042018DF80610E06908B1E0690C902B46A3
:1057D00004AA09A93046AADF10B070BD70B58AB01E
:1057E00004460E46202101A8F0F763FE0020099030
:1057F00094F8C60200EB8001C1EB801004EB400579
:1058000094F8C502B8B194F8C522521ED1B294F8EA
:10581000C62202EB8203C3EB821204EB420501EBCA
:10582000C10305F10A0202EB43000289521C92B245
:10583000ADF8242002E0E888ADF824002889ADF80E
:10584000260003208DF8040009980590049405486B
:105850000390324601A9044800680BF0CBF90AB066
:1058600070BD0000B56E0300184A002010B52DED84
:10587000048BB0EE408A9FED270AB0EE409A9FED70
:10588000250AF0EE408A2448006890F8220060B1B2
:10589000B2EE040AC8EE000A1F480068C0ED010A13
:1058A00000201D49096881F82200B2EE040AC8EE02
:1058B000000AF0EE609A18480068001DDFED170A34
:1058C000B0EE690A03F0FFFEF0EE408A9FED140A85
:1058D000F4EEC08AF1EE10FA04D29FED0E0AB0EE9B
:1058E000409A11E09FED0F0AF4EEC08AF1EE10FA33
:1058F00004DD9FED0D0AB0EE409A05E0B0EE680AB7
:1059000007F0F0FDB0EE409AB0EE490ABDEC048B12
:1059100010BD00000000000044400020CDCC4C3DF4
:105920000000AF430080CF430000C842192000BFF1
:105930004FF0A0431A4600BFD2F81035C34003F021
:105940000103194609B1012070470020FCE710B59A
:10595000014600220B46002004E00C1D245C144488
:10596000E2B2401CDC788442F7DC9878904201D1A6
:10597000012010BD0020FCE72DE9F04104460D4652
:105980004FF6FF76304684420AD14FF480712846A4
:105990000AF05DFF86B2B6F5807F10D126460EE094
:1059A000FF2C0CDC214628460AF03AFF80F0010764
:1059B0000FB1204601E04FF6FF70064600BF3046AB
:1059C000BDE8F08170B505460DB9094C01E0084C01
:1059D000083409E0204608F074FA064606B904E0E7
:1059E00028467168884700BFF4E700BF70BD00001B
:1059F000A499002010B504462CB90120064948702E
:105A00000020FFF7DFFF012C04D10120024988703C
:105A1000FFF7D8FF10BD00009C9900202DE9F0474A
:105A2000024613468C46D3E90245DCE90267B6EB31
:105A3000040877EB050002D30120BDE8F0870020C1
:105A4000FBE701468878012805D191F8200001285C
:105A500001D100207047886A042802D0486A0428CF
:105A600001D10020F6E70120F4E72DE9FF4F0346BE
:105A70000C46002047E0225CFF2A3ED0C2F3C0194A
:105A800022F080014DF82010B9F1000F0DD05DF823
:105A9000201000BF4FF0A0452E46012707FA01F560
:105AA000C6F8085500BF00BF0DE05DF8201000BF2C
:105AB0004FF0A0452E46012707FA01F5C6F80C5510
:105AC00000BF00BF00BF5DF8201001252E46002753
:105AD000BC46B84600BF4FF0A04BDA4645EA460B3D
:105AE0004BEA870B4BEA0C2B4BEA084E0AF5E06BAE
:105AF0004BF821E000BF00BF03E04FF0FF314DF84D
:105B00002010411CC8B20428B5DB6D461A6800217C
:105B100007E055F8217002F5AC6646F821704E1C7E
:105B2000F1B20429F5DB00BFBDE8FF8F024600207B
:105B300007E0536833F810308B4200D17047431CA4
:105B400098B213888342F4DC00BFF7E733B58BB01B
:105B50000546002000900C9878B100240BE0214607
:105B60000CA80AF0A4FE28B1009A501C009001A8CD
:105B700020F81240641C142CF1D32C2269462846CC
:105B8000F0F77EFC0DB030BD10B502460B4600218B
:105B90000DE0506830F811004FF6FF74A04204D1B8
:105BA000506820F81130002010BD481C81B21088C8
:105BB0008842EEDC0420F7E701460888062808DB67
:105BC0000888B0F5486F06DD08884FF6FF729042EE
:105BD00001D0072070474888062808DB4888B0F5C0
:105BE000486F06DD48884FF6FF72904201D00720CB
:105BF000F0E708884FF6FF72904208D0488890423C
:105C000005D008884A88904201DD0720E2E700209D
:105C1000E0E72DE9F04107460D46144698462088F6
:105C2000801D404502D90C20BDE8F0813846FFF7C1
:105C3000C3FF064600BF304600B1F5E700BF0520B0
:105C4000218868542088401C2080122021886854B4
:105C50002088401C208022885119388813F0E7FCE6
:105C600021880844208022885119788813F0DFFCAD
:105C70002188084420800020D6E7000010B50446A3
:105C800000BF03A281212046F0F7C4FA00BF10BD77
:105C90002E2E5C2E2E5C2E2E5C626C655F6366671A
:105CA0005C736C6176652E630000000030B587B0D0
:105CB0001C216846F0F7FDFB002000904FF4804067
:105CC00001904FF4A030029001208DF80C004FF6A7
:105CD000FF70ADF80E0001208DF810000020059037
:105CE000094806906846FCF73DFE044600BF25467D
:105CF00035B100BF05A294212846F0F78BFA00BF0A
:105D000000BF07B030BD00007D5C03002E2E5C2E6E
:105D10002E5C2E2E5C626C655F6366675C736C61E3
:105D200076652E6300000000F8B505460C46607AE3
:105D300088B9207A10B91048476801E00E48876892
:105D40002A4639466068FCF791F8064616B1304697
:105D500012F030F90EE0002020720748406948B187
:105D600001208DF80000ADF80250034841696846F3
:105D7000884700BFF8BD00009C960020F0B585B0B4
:105D800004460D4617461E4614220B496846F0F796
:105D900077FBADF802408DF80850ADF80A708DF829
:105DA0000C600022054801782046FCF7B9FE6846E1
:105DB00003F05AFB05B0F0BD04A60400554A0020CC
:105DC00010B586B0044620880EF0C6FB00BB2088C4
:105DD000FCF720FE30B92088012241F2060103F0D1
:105DE000E8F815E0208800220A490978FCF798FEB7
:105DF00002208DF804002088ADF8060000208DF800
:105E00000C0000218DF80D1001A803F02DFB00BF40
:105E100006B010BD554A00200246002003E0064BA4
:105E20001B5C1354401C054B1B789842F7DB03485E
:105E3000007808707047000030850020D2470020AD
:105E40000246002003E0064B1B5C1354401C054B2C
:105E50001B789842F7DB0348007808707047000011
:105E6000F4840020D1470020F0B504460D46002000
:105E7000002108E014F801C00646471CF8B20B4F99
:105E800007F806C0491CA942F4DB002108E012F81B
:105E900001C00646471CF8B2044F07F806C0491C6B
:105EA0009942F4DB02490870F0BD0000F484002040
:105EB000D14700202DE9F0410646DDE906450020E6
:105EC0000F88C7F307280746401CDFF83CC10CF8D1
:105ED000078091F800800746401C0CF807804F8827
:105EE000C7F307280746401C0CF8078091F802808A
:105EF0000746401C0CF807808F88C7F30728074621
:105F0000401C0CF8078091F804800746401C0CF8F0
:105F100007801788C7F307280746401C0CF807803E
:105F200092F800800746401C0CF807805788C7F39A
:105F300007280746401C0CF8078092F802800746A5
:105F4000401C0CF807809788C7F307280746401CB9
:105F50000CF8078092F804800746401C0CF8078074
:105F60001F88C7F307280746401C0CF8078093F8E2
:105F700000800746401C0CF807805F88C7F307289D
:105F80000746401C0CF8078093F802800746401C27
:105F90000CF807809F88C7F307280746401C0CF8B9
:105FA000078093F804800746401C0CF80780278878
:105FB000C7F307280746401C0CF8078094F80080B8
:105FC0000746401C0CF807806788C7F30728074678
:105FD000401C0CF8078094F802800746401C0CF81F
:105FE0000780A788C7F307280746401C0CF80780DE
:105FF00094F804800746401C0CF80780DFF80CC0BA
:106000008CF80000BDE8F08130850020D2470020E8
:106010007FB506460C46002002900390ADF808407C
:10602000ADF80A40009001906A4602A9304690DF20
:10603000054605B100BF284604B070BD10B5044642
:1060400021460248FDF70DFA10BD000090820020A5
:106050007CB500200090019009480090094801900B
:106060006846FCF79BFD044600BF254635B100BFDE
:1060700005A22D212846F0F7CDF800BF00BF7CBD5A
:106080003D600300A44700202E2E5C2E2E5C2E2E99
:106090005C626C655F6366675C686F73742E630037
:1060A0002DE9F04105460F460F4C012120460AF02C
:1060B0004FFC064600BF00BF00BF00BFBFF35F8FAD
:1060C00000BF00BF00BF0EB9012000E0002040B1BA
:1060D000284608F0C1F808B1BDE8F08102480BF08D
:1060E00099FD00BFF8E70000344A002070B52DED9F
:1060F0000A8B04460D4694ED060AB1EE400A10EEF6
:10610000101A0846F0F7FFFB41EC1B0BB0EE4B0AF0
:10611000F0EE6B0AF7F724F8B0EE40AAF0EE60AAB2
:1061200051EC1A0BF0F71AFC09EE100A94ED060A6E
:10613000DFED530AB4EEE00AF1EE10FA08DC94ED5C
:10614000060ADFED500AB4EEE00AF1EE10FA2AD2A8
:1061500094ED040A10EE101A0846F0F7D4FB41EC57
:106160001B0B94ED010AB1EE400A10EE101A08461E
:10617000F0F7C9FB41EC1C0BB0EE4B1AF0EE6B1ABA
:10618000B0EE4C0AF0EE6C0AF7F706FBB0EE40AA50
:10619000F0EE60AA51EC1A0BF0F7E0FB08EE100AE3
:1061A000DFED398A4BE094ED000A10EE101A084634
:1061B000F0F7A9FB41EC1B0B94ED030A10EE101A4B
:1061C0000846F0F7A0FB41EC1C0BB0EE4B1AF0EECA
:1061D0006B1AB0EE4C0AF0EE6C0AF7F7DDFAB0EE8F
:1061E00040AAF0EE60AA51EC1A0BF0F7B7FB08EEEC
:1061F000100A94ED080A10EE101A0846F0F783FB17
:1062000041EC1B0B94ED070A10EE101A0846F0F74C
:106210007AFB41EC1C0BB0EE4B1AF0EE6B1AB0EEB1
:106220004C0AF0EE6C0AF7F7B7FAB0EE40AAF0EEBF
:1062300060AA51EC1A0BF0F791FB08EE900A9FED63
:10624000130A28EE000ABDEEC00A10EE100A00B2D2
:1062500028809FED0E0A29EE000ABDEEC00A10EE5E
:10626000100A00B268809FED090A28EE800ABDEE90
:10627000C00A10EE100A00B2A880BDEC0A8B70BDF7
:10628000EFFF7F3FEFFF7FBF0000000000401C4694
:1062900002781206437842EA0342837842EA0322F4
:1062A000C3781A433C4B1A6002791206437942EADA
:1062B0000342837942EA0322C3791A43364B5A6078
:1062C000027A1206437A42EA0342837A42EA0322BE
:1062D000C37A1A43304B9A60427B037B42EA032223
:1062E00012B22E4B1A80C27B837B42EA032212B287
:1062F0002A4B5A80427C037C42EA032212B2274B8B
:106300009A80C27C837C42EA0322254B1A80427D1C
:10631000037D42EA0322234B1A80827D224B1A809E
:10632000C27D224B1A70427E037E42EA032212B2E1
:106330001F4B1A80C27E837E42EA032212B21D4B9B
:106340001A80427F037F42EA032212B2194B5A801D
:10635000C27F837F42EA032212B2164B9A8090F8E2
:10636000212090F8203042EA032212B2124B1A8008
:1063700090F8232090F8223042EA032212B20E4B0A
:106380005A8090F8252090F8243042EA032212B275
:10639000094B9A8070470000C48C00200C490020F3
:1063A0003E490020424900201E4900203A49002071
:1063B00008490020124900201849002002781206DE
:1063C000437842EA0342837842EA0322C3781A43BD
:1063D0003C4B1A6002791206437942EA0342837900
:1063E00042EA0322C3791A43364B5A60027A1206F4
:1063F000437A42EA0342837A42EA0322C37A1A4387
:10640000304B9A60427B037B42EA032212B22E4B4E
:106410001A80C27B837B42EA032212B22A4B5A8043
:10642000427C037C42EA032212B2274B9A80C27C50
:10643000837C42EA0322254B1A80427D037D42EA97
:106440000322234B1A80827D224B1A80C27D224B6D
:106450001A70427E037E42EA032212B21F4B1A8058
:10646000C27E837E42EA032212B21D4B1A80427F13
:10647000037F42EA032212B2194B5A80C27F837F04
:1064800042EA032212B2164B9A8090F8212090F82B
:10649000203042EA032212B2124B1A8090F82320D5
:1064A00090F8223042EA032212B20E4B5A8090F842
:1064B000252090F8243042EA032212B2094B9A8038
:1064C00070470000D08C0020244900203C49002067
:1064D0004049002036490020394900202049002049
:1064E0002A4900203049002070B506460D4616B1F5
:1064F0004FF4064070BD287920B1012809D0022848
:1065000015D111E002202871284610F025F9044623
:1065100010E0284603F0B8F8044648F209608442C7
:1065200001D141F61D5405E041F61D5402E048F248
:106530000E6400BF00BF2046DCE700002DE9F04FED
:1065400089B004460F4691464FF0000B2021684663
:10655000EFF7AFFF94F8C60200EB8001C1EB8010AB
:1065600004EB400594F8C50200EBC00105F10A00F8
:1065700000EB410A94F8C502401C2979884207D1F2
:1065800008AB00225146204607F047FC834627E02F
:1065900094F8C5621FE02879401EB04202D14FF046
:1065A000000806E0701C00EBC00105F10A0000EBDA
:1065B000410808AB42465146204607F02EFC10B178
:1065C0004FF0010B0AE0C24694F8C502401C84F863
:1065D000C502701CC6B22879B042DCDC00BF00BF27
:1065E000BBF1000F05D101203870002009B0BDE8D3
:1065F000F08F0020387004208DF800000898049077
:106600000394044802904A466946034800680AF029
:10661000F1FAEBE7B56E0300184A00202DE9F041CE
:106620002DED068B84B006460F464FF00008002083
:1066300005E036F9101001AA42F82010401C03288A
:10664000F7DB0398002801DB014600E041429B4A4A
:1066500011809B48007803280BDB9A4840689949D1
:1066600008600846806848600220954908704FF02D
:10667000010892480188924802780078401C904BAB
:106680001870904840F822108F480078032809DBE2
:106690008E4840888D4908800846808848800220BE
:1066A00089490870784202B2874801780078401C16
:1066B000854B1870854820F81120B8F1010F72D170
:1066C000804880687F494968401A15D4804800880E
:1066D00028B97C48008900B27E49088014E07948D6
:1066E00080687C49B1F9001088420DDD7548008949
:1066F00000B27849088007E07548008820B97148E1
:10670000008900B2744908806E4880687249B1F906
:106710000010401AB0F5487F15DD01206C49088053
:10672000684880686C49B1F90010401A6B49B1F9AA
:106730000010884207DD6348008967490988401ACC
:1067400000B2664908805F4880686349B1F900106B
:10675000401AB0F5487F2BDD6048B0F90000F0F733
:106760007CF841EC1A0B9FED5E0B53EC102BEFF70E
:106770007DFF41EC180B53498968564AB2F9002055
:10678000501AF0F76AF841EC190B53EC182BF0F79C
:10679000CDF814D24B4880684A494968451A002D03
:1067A00002DB284601E077E06842B0F5C87F06DAF0
:1067B0000020474908804FF44870484908804A48FB
:1067C000007830BB0020494908804948B0F90000F2
:1067D000B0F5967F05DA46480088401C00B244496F
:1067E00008803B48008801280ED14148B0F90000DC
:1067F000082809DB012401203B49087022463DA1FD
:106800000020F4F759FA52E00024002036490870BD
:106810004DE000240020364908803448B0F90000DB
:10682000B0F5967F05DA31480088401C00B22F4948
:106830000880274B1B8873BB244BB3F90030A3F5AA
:10684000FA62002A01DB134600E05342B3F5967F5B
:1068500019DC1E4BB3F90230A3F5FA61002901DB04
:106860000B4600E04B42B3F5967F0CDC174BB3F9B7
:106870000430A3F5FA60002801DB034600E0434240
:10688000B3F5967F13DD194BB3F90030062B0EDB01
:106890000020154908700AE000240A48008900B267
:1068A0000D4908800748008900B20A490880E0B213
:1068B00004B0BDEC068BBDE8F0810000C4490020A7
:1068C000054A0020C4950020044A0020FE4900200B
:1068D0000A4A0020084A0020064A00200C4A0020EC
:1068E0009A9999999999D93FFC4900200E4A00201C
:1068F000104A0020737465703D3D25640A00000055
:106900002DE9F04F8BB082468B4615461C46BAF9EE
:106910000400002801DB014600E0414209B20A916F
:10692000BBF90400002801DB014600E0414209B246
:1069300009917622FA49881EEFF7A2FD7622F949DD
:10694000881EEFF79DFD7622F749881EEFF798FD28
:106950007622F649881EEFF793FD7622F449881EC9
:10696000EFF78EFDEE49891E0A98A1F87600ED48F2
:10697000801E0999A0F876102888EB49891EA1F895
:1069800076006888E949891EA1F87600A888E84958
:10699000891EA1F8760007A808A904233C22CDE9A6
:1069A00000101421E048801E02F0A0FE05A806A9F0
:1069B00004233C22CDE900101421DC48801E02F0A3
:1069C00095FE03A804A904233C22CDE9001014215C
:1069D000D748801E02F08AFED64B4FF4FA623C2163
:1069E000D048801E07F0EDF88046B8F1010F02D1C3
:1069F0005020D1490880D14B4FF4FA623C21C9485C
:106A0000801E07F099F80290CB48B0F900000028EA
:106A100009DDCB4B4FF4FA623C21C148801E07F0E0
:106A2000D0F8064608E0C64B40F6B8323C21BC48D8
:106A3000801E07F0C6F80646C24B4FF4FA623C21AE
:106A4000B748801E07F078F88146B648801EB0F936
:106A50007600B849B1F90010401AB0F5FA6F0ADDB6
:106A6000B048801EB0F97600B449B1F90010081A98
:106A7000B0F57A7F15DBAA48801EB0F97600B049E0
:106A8000B1F90010401AB0F5FA6F0DDDA448801E70
:106A9000B0F97600AB49B1F90010081AB0F57A7F69
:106AA00002DA2820A84908809E48801EB0F97600A6
:106AB000A049B1F90010401AB0F5FA6F0BDD984803
:106AC000801EB0F976009E49B1F90010401AB0F569
:106AD000FA6F00DD01269D4A0FFA89F130B211F0FC
:106AE000D1FC9A48B0F90000002802DD50209849F6
:106AF0000880012228218E48801E12F0D5FE95487C
:106B000080ED000A8A48801E884B9B1E864A921E92
:106B1000214600908D4811F073FC8D48B0F90000BB
:106B2000002804DC8848B0F9000000281CDDBDF90D
:106B30002000BDF91C10401AC82815DABDF918004C
:106B4000BDF91410401AC8280EDABDF91000BDF9BD
:106B50000C10401AC82807DA012020807B480088E2
:106B600010B90220794908807748B0F90000002860
:106B700011DD784890ED000AF7EE000AB4EEE00A65
:106B8000F1EE10FA07DD012020807048008810B96E
:106B900002206E490880BDF92000BDF91C10401A82
:106BA000672816DABDF91800BDF91410401A6728D5
:106BB0000FDABDF91000BDF90C10401A672808DA89
:106BC00001211598018064480068401C62490860F2
:106BD00005E000211598018000205F4908605E48AB
:106BE0000068B0F5C87F03DD012020805749088088
:106BF00067275A48B0F90000002802DD40F2064736
:106C000003E0F2F71FFF00B1FA27554B1B88012B59
:106C100040D1454B9B1EB3F96E30DFF80CC1ACF18F
:106C2000020CBCF976C0A3EB0C02002A01DB134670
:106C300000E05342BB422DDA3C4B9B1EB3F96E3051
:106C4000DFF8E8C0ACF1020CBCF976C0A3EB0C0194
:106C5000002901DB0B4600E04B42BB421ADA344B01
:106C60009B1EB3F96E30DFF8C8C0ACF1020CBCF962
:106C700076C0A3EB0C00002801DB034600E0434292
:106C8000BB4207DA012020803048008810B902207A
:106C90002E4908802E48B0F90000002805DD2C4858
:106CA0000088401E00B22A4908802E48B0F9000032
:106CB000002805DD2B480088401E00B229490880C5
:106CC0002648B0F90000002805DD24480088401E51
:106CD00000B2224908801848B0F90000002805DDFC
:106CE00015480088401E00B2134908801648B0F9C4
:106CF0000000002805DD14480088401E00B212493B
:106D00000880208810B1502011490880208814493B
:106D1000088014980088144908800BB0BDE8F08FF3
:106D200056930020CE93002046940020BE9400206D
:106D300036950020BC490020B6490020C0490020FB
:106D4000BA490020BE490020B84900209C490020D3
:106D5000A8490020A0490020B0490020AE490020E9
:106D6000A4490020AC490020A649002070B5044683
:106D700020793D2802D141F23D0001E04FF48850D6
:106D8000054620880022294607F0D7F970BD00008B
:106D900030B59FB004460D467C216846EFF789FB6D
:106DA000ADF8025003208DF80000019404480068FB
:106DB00018B168460249096888471FB030BD000015
:106DC000144A00202DE9F04104460D46164694F879
:106DD000C60200EB8001C1EB801004EB4008404686
:106DE0000FF01EFE0746E7B3D4F8CC02062838D2CF
:106DF00004F53470D4F8CC1200EBC110468004F5D1
:106E00003471D4F8CC2201EBC211081D7622414620
:106E1000EFF736FB45B1002104F53470D4F8CC22ED
:106E200000EBC210017007E0022104F53470D4F8C1
:106E3000CC2200EBC210017004F53470D4F8CC12EF
:106E400000EBC110C767D4F8CC02401CC4F8CC02D8
:106E50000549D4F8CC020968884202D120460DF0D9
:106E60001DFFBDE8F08100001C4A00202DE9F04123
:106E7000A0B004460D46164694F8C60200EB800109
:106E8000C1EB801004EB400840460FF0C9FD0746F7
:106E900057B17C22064901A8EFF7F2FAADF8066077
:106EA000029501A8B84700BF20B0BDE8F0810000FE
:106EB0007CA404002DE9F04105460C461646274601
:106EC000002087F8C802324629463846FFF7CEFF31
:106ED00031463846FFF75CFFBDE8F081F0B589B078
:106EE00004460E464FF4BA612046EFF7E2FA20213D
:106EF00001A8EFF7DEFA31461E48006809F050FE9F
:106F0000054600BF284608B109B0F0BD00BFA4F88F
:106F1000CA620020C4F8CC0284F8C70284F8C60212
:106F200084F8C50294F8C60200EB8001C1EB801022
:106F300004EB400794F8C6020F4901EB800000689B
:106F4000386002208DF804000120ADF81400396883
:106F5000CDF81610049409480390324601A905485B
:106F6000006809F047FE054615B9012084F8C802FB
:106F70002846C9E7184A0020D0950020B56E0300C6
:106F80001CB518213348EFF794FA002131482C380A
:106F900080F84C1080F8491080F84D1080F84A10A5
:106FA00080F84E1080F84B1080F8461080F848109A
:106FB00080F84710002027492C3981F8440000212F
:106FC00024482C3880F84510234822492C39486041
:106FD0002248086000208862032103460122CDE98F
:106FE0000010114605200AF067FB06200AF00BFC92
:106FF00007200AF008FC08200AF005FC09200AF026
:1070000002FC002106200AF02FFD002107200AF0D3
:107010002BFD002108200AF027FD002109200AF09D
:1070200023FD002105200AF01FFD03200DF059FE6D
:10703000012105200AF018FD03200DF052FEF3F7A0
:107040009BFF074A07A14FF47A70F3F7F7F810F0A7
:107050007BFB1CBD347D0020014D0400694D040004
:10706000718703006472765F6C736D5F7370695F24
:107070006572726F725F7265706F72745F70726F3B
:10708000636573730000000038B50446134890F838
:107090004900E8B16946114807F057FE9DF8000025
:1070A00000F0010088B10E48002101608180014696
:1070B0000A4807F003F90A480088208008484088F9
:1070C000608007488088A08005E04FF0FF3038BD21
:1070D0004FF0FF30FBE70020F9E70000087D0020BB
:1070E000587D00200146054802680A6042684A60EF
:1070F00002890A81807A8872002070474C7D0020C6
:107100002DE9F041054600260024474890F84A0042
:1071100000B1B61D444890F8490000B1B61D424880
:1071200090F84B0000B1B61D3F4890F84800012888
:1071300000D1B61D18213D48EFF7BBF9F2B23B492B
:10714000394807F0E4FA0746781C18B94FF0FF30C9
:10715000BDE8F081002D64D0334890F84A0098B122
:1071600004EB4400314931F81000E88004EB44009E
:1071700001EB40004188298104EB44002B4901EBDD
:10718000400081886981641C274890F8490090B1CB
:1071900004EB4400254931F81000288004EB44003A
:1071A00001EB40004088688004EB440001EB4000A4
:1071B0008088A880641C1C4890F84B0098B104EBB0
:1071C00044001A4931F81000A88104EB440001EB97
:1071D00040004188E98104EB4400144901EB400080
:1071E00081882982641C104890F84800012818D131
:1071F00004EB44000D4901EB40004078000404EB2F
:1072000044010A4A12F8111040EA012004EB44013B
:1072100002EB4101C978084300EBC00101EB00100B
:107220006861002094E70000087D0020587D002060
:107230007CB5002000900025002401A9144807F027
:10724000B6FA9DF8040008B36946114807F096F8AD
:107250000F4890F8490008B1E01C84B20C4890F83F
:107260004A0008B1E01C84B2094890F84B0008B10C
:10727000E01C84B2064890F84800012801D1E01CC7
:1072800084B2BDF8000090FBF4F085B228467CBDC6
:10729000087D0020052070471CB5F3F74BFE002049
:1072A000032103460122CDE90010114605200AF012
:1072B00003FA06200AF0A7FA002106200AF0D4FB00
:1072C000002107200AF0D0FB002108200AF0CCFBA7
:1072D000002109200AF0C8FB002105200AF0C4FBA8
:1072E00000201CBD7CB5012105200AF0BDFB062550
:1072F00001240020009023460246014601902846C2
:107300000AF0DAF900BF18211548EFF7D2F800218A
:1073100013482C3880F84C1080F8491080F84D1034
:1073200080F84A1080F84E1080F84B1080F8461014
:1073300080F8481080F84710002009492C3981F85E
:107340004400002106482C3880F8451000200449EC
:107350002C398862F3F7EEFDF3F70EFE00207CBDBA
:10736000347D002010B51C491C4806F0FBFF1A486C
:1073700000786A2806D01AA10020F3F79DFC4FF090
:10738000FF3010BD0121154807F0D4FB4FF4FA601F
:107390001249886200BF1949104807F0BAFB0F482C
:1073A000806A401E0D4988621448007818B108466A
:1073B000806A0028EFD10948806A10B94FF0FF3089
:1073C000DFE70721054807F085FD0221034807F0A4
:1073D000D3FD0020D5E7000014410020087D0020E7
:1073E0004C534D2073656C665F636865636B206505
:1073F00072726F722121210D0A00000015410020D8
:1074000010B54FF4FA604B49886200BF4A494948B9
:1074100007F079FD4748806A401E46498862464821
:10742000007818B90846806A0028EFD14148806A80
:1074300010B94FF0FF3010BD40493E4806F03EFF06
:107440003F48002101604160816000203D49087093
:1074500047E04FF4FA603749886200BF3649354843
:1074600007F051FD3348806A401E32498862324835
:10747000007818B90846806A0028EFD12D48806A44
:1074800010B94FF0FF30D6E72C492A4806F016FF16
:1074900000202D4908701BE028492B4A127831F949
:1074A000120007F0EDF926482749097800EB810022
:1074B000D0ED000A30EE200A21482349097800EB7C
:1074C000810080ED000A20480078401C1E490870A9
:1074D0001D4800780328DFDB1A480078401C194952
:1074E0000870184800780528B3DB0020154908709B
:1074F00016E013481349097800EB810090ED000A6B
:10750000F1EE040A80EE201A0D480E49097800EBCE
:10751000810080ED001A0B480078401C0949087072
:10752000084800780328E4DB0221024807F074FDD4
:10753000002080E7087D00201D410020164100202A
:10754000707D00201E4100201F41002010B52DED50
:10755000048B4FF4FA608549886200BF84498348F0
:1075600007F0D1FC8148806A401E804988628048CB
:10757000007818B90846806A0028EFD17B48806AF5
:1075800020B94FF0FF30BDEC048B10BD794977482E
:1075900006F094FE7848002101604160816000207F
:1075A0007649087047E04FF4FA607049886200BF7E
:1075B0006F496E4807F0A7FC6C48806A401E6B4913
:1075C00088626B48007818B90846806A0028EFD1B5
:1075D0006648806A10B94FF0FF30D4E765496348C8
:1075E00006F06CFE0020664908701BE06149644AA1
:1075F000127831F9120007F043F95F4860490978C1
:1076000000EB8100D0ED000A30EE200A5A485C49B8
:10761000097800EB810080ED000A59480078401C91
:1076200057490870564800780328DFDB5348007834
:10763000401C52490870514800780528B3DB0020EF
:107640004E49087016E04C484C49097800EB81001F
:1076500090ED000AF1EE040A80EE201A46484749F0
:10766000097800EB810080ED001A44480078401C46
:1076700042490870414800780328E4DB00203F4974
:1076800008702EE03C483D4A127800EB820090EDF5
:10769000000A3C48394A127800EB8200D0ED000A1B
:1076A00030EE600A10EE101A0846EFF72CF941ECA4
:1076B000190BB0EE490AF0EE690AF6F7C9F9B0EE17
:1076C000408AF0EE608A51EC180BEFF747F92E492B
:1076D0002A4A127841F8220028480078401C27499D
:1076E0000870264800780328CCDB01202749087061
:1076F00000202249087023E023482049097800EB44
:10770000810090ED000ADFED220AB4EEE00AF1EE0E
:1077100010FA0DD31C481949097800EB810090ED4F
:10772000000ADFED1C0AB4EEE00AF1EE10FA02DD09
:1077300000201649087011480078401C0F49087055
:107740000E4800780328D7DB0021084807F064FCC6
:107750000021064807F0BEFB0721044807F0F3F8B4
:107760000621024807F044F900200CE7087D0020BC
:107770001D410020164100207C7D00201E4100207C
:107780001F410020707D0020887D00201C410020CA
:107790000000B4420080D44410B54FF4FA604B4965
:1077A000886200BF4A49494807F0E6F84748806ABE
:1077B000401E464988624648007818B90846806AE3
:1077C0000028EFD14148806A10B94FF0FF3010BD5A
:1077D00040493E4806F09CFD3F4800210160416061
:1077E000816000203D49087047E04FF4FA60374956
:1077F000886200BF3649354807F0BEF83348806AD2
:10780000401E324988623248007818B90846806ABA
:107810000028EFD12D48806A10B94FF0FF30D6E72D
:107820002C492A4806F074FD00202D4908701BE001
:1078300028492B4A127831F9120007F015F826482A
:107840002749097800EB8100D0ED000A30EE200ACC
:1078500021482349097800EB810080ED000A204887
:107860000078401C1E4908701D4800780328DFDBA3
:107870001A480078401C19490870184800780528F3
:10788000B3DB00201549087016E013481349097846
:1078900000EB810090ED000AF1EE040A80EE201A60
:1078A0000D480E49097800EB810080ED001A0B4865
:1078B0000078401C09490870084800780328E4DB78
:1078C0000121024807F0E3F8002080E7087D00204E
:1078D0001D41002016410020707D00201E41002027
:1078E0001F41002010B52DED048B8A480021016056
:1078F0004160816000208849087049E04FF4FA60D7
:107900008649886200BF8649844807F035F8834875
:10791000806A401E814988628148007818B908460B
:10792000806A0028EFD17D48806A20B94FF0FF308F
:10793000BDEC048B10BD7B49784806F0E9FC0020C3
:10794000794908701BE07749774A127831F91200BB
:1079500006F08AFF6F487449097800EB8100D0ED8A
:10796000000A30EE200A6B486F49097800EB81006D
:1079700080ED000A6C480078401C6B4908706A482A
:1079800000780328DFDB64480078401C62490870F7
:10799000614800780528B1DB00205F49087016E0D7
:1079A0005C485D49097800EB810090ED000AF1EE3A
:1079B000040A80EE201A57485749097800EB8100E5
:1079C00080ED001A54480078401C53490870524812
:1079D00000780328E4DB00204F4908702EE04D4872
:1079E0004D4A127800EB820090ED000A4F484A4A57
:1079F000127800EB8200D0ED000A30EE600A10EE43
:107A0000101A0846EEF77FFF41EC190BB0EE490A59
:107A1000F0EE690AF6F71CF8B0EE408AF0EE608AE4
:107A200051EC180BEEF79AFF41493B4A127841F8A6
:107A3000220039480078401C3749087036480078E1
:107A40000328CCDB00203449087023E03848324951
:107A5000097800EB810090ED000ADFED360AB4EE04
:107A6000E00AF1EE10FA0DD331482B49097800EB0A
:107A7000810090ED000ADFED300AB4EEE00AF1EE8D
:107A800010FA02DD00202D49087023480078401CC0
:107A900021490870204800780328D7DB00211F48BF
:107AA00006F0F5FF00211D4806F04DFF2348007841
:107AB000012814D122A10020F3F7FEF80121174874
:107AC00007F0B1F8FF2024490870144807F09AF82D
:107AD0002148007801281AD04FF0FF3028E71FA175
:107AE0000020F3F7E9F801210C4807F09CF8FF208B
:107AF00019490870094807F085F8174800780128E7
:107B000002D04FF0FF3013E74FF0FF3010E70020B6
:107B10000EE700007C7D00201E410020087D002033
:107B20001D410020164100201F410020707D0020D3
:107B3000887D0020007C124800E62A491C41002074
:107B40004C534D2053656C662054657374202D2072
:107B5000504153530D0A00001541002053656C66D7
:107B60002054657374202D204641494C0D0A0000B5
:107B700038B50446194890F84C00A0422BD014B1F7
:107B8000012C27D112E00021144807F0F5F96946CD
:107B9000124807F0C9F99DF8000010B14FF0FF300E
:107BA00038BD00210D4880F84C1013E001210B482E
:107BB00007F0E2F96946094807F0B6F99DF80000B8
:107BC000012802D04FF0FF30EAE70121034880F896
:107BD0004C1000BF00BF0020E2E70000087D00203D
:107BE00038B50446434890F84900A04279D0082CA3
:107BF0007DD2DFE804F004177C7C2B3F5367002123
